:100000000C94A3470C94C4470C9499D00C94C44707
:100010000C94C4470C94C4470C94C4470C94C44734
:100020000C94C4470C94C4470C94C4470C94C4D299
:100030000C94C4470C94C4470C94CEB40C94C4479D
:100040000C94C4470C94C4470C94C4470C94C44704
:100050000C94C4470C94C4470C94C4470C94C447F4
:100060000C94C4470C94B3D00C9442D00C94C44765
:100070000C9419CA0C94BBC90C94F7C90C94C447CE
:100080000C9464D10C94C4470C94C4470C94C4479A
:100090000C94C4470C94C4470C94C4470C94C447B4
:1000A0000C94C4470C94C4470C94C4470C94A7BB4D
:1000B0000C944BBC0C94C4470C94C4470C94BFB62E
:1000C0000C94C4470C94C4470C94C4470C94C44784
:1000D0000C94C4470C94C4470C94C4470C94C44774
:1000E0000C9465A60C94C4470C94C4470C94C44764
:1000F0000C94C4470C94C4470C94C4470C94C44754
:100100000C947EBB0C9422BC0C9455BB0C94F9BB94
:100110000C94C4470C94C4470C94C4470C94C44733
:100120000C94C4470C94C4470C94C4470C94C44723
:100130000C94C4470C9423B60C94C4470C94C44745
:100140000C94C4470C94C4470C94C4470C94C44703
:100150000C94C4470C94C4470C945BA60C94C447FD
:100160000C94C4470C94C4470C94C4470C94C447E3
:100170000C94C4470C94C4470C94C4470C94C447D3
:100180000C94C4470C94C4470C94C4470C94C447C3
:100190000C94C4470C94C4470C94C4470C94C447B3
:1001A0000C94D0BB0C9474BC0C94C4470C94C447FE
:1001B0000C9471B60C94C4470C94C4470C94C44777
:1001C0000C94C4470C94C4470C94C4470C94C44783
:1001D0000C94C4470C94C4470C94C4470C94C44773
:1001E0000C94C4470C94C447BA71C471CE71D871D1
:1001F000E371E977E977E977E977E977E971E97711
:10020000E977E977E977E977E977EB71F571FF71DC
:1002100009721372E977E977E977E977E977E9779E
:100220001D72E9777372E977E977E977E977E9771A
:10023000E977E977B272E977CE75E977E977E97717
:10024000E977E977E977E977E977CE75E977E977CB
:10025000E977DF72E472EE72F872FA7204730F7368
:10026000E9771A73E977E9775773E977E977E977F7
:10027000E977E977E977E977E977E977E977E9777E
:10028000E977E977E977E9776173E977E977E977FA
:10029000E977E977E977E977E977E9776B73A87325
:1002A000E5732E743874517451745B7465746F7493
:1002B00079748374887492749C74E777E777E7772E
:1002C000E777E777E777E777E777E777E777E7773E
:1002D000E777E777E777E777E777E777E777E7772E
:1002E000E7775B74E777E777E777E777E777E777AD
:1002F000E777E777E777E777E777E777E777E7770E
:10030000E777E777E777A674B074BA74C474E777D1
:10031000E777E777E777E777E777E777E777517486
:100320007477337737773F771B771F7727772B776C
:100330004B77607768776C777077CC7743773F75CA
:1003400050756175E977E977D974AB71E9777275A2
:1003500083759475CE754274B675E977EA74E9775A
:10036000A575FB74CE74E977E977E9770C751D758F
:100370002E75EEBAF6BAFEBA06BB0EBB16BB1EBB96
:1003800026BB06BE6ABD72BD7ABD82BD8ABD92BD66
:100390009ABDA2BDAABDB2BDBABDC2BDCABDD2BDC5
:1003A000EABDEABDEABDEABDEABDEABDEABDEABD15
:1003B000EABDEABDEABDEABDEABDEABDEABDEABD05
:1003C000EABDEABDEABDEABDEABDEABDEABDEABDF5
:1003D000EABDEABDEABDEABDEABDEABDEABDEABDE5
:1003E000EABDEABDEABDDABDE2BD084AD73B3BCE75
:1003F000016E84BCBFFDC12F3D6C74319ABD568324
:100400003DDA3D00C77F11BED9E4BB4C3E916BAADB
:10041000AABE000000803F05A84CCDB2D44EB9382A
:1004200036A9020C50B9918688083CA6AAAA2ABE11
:10043000000000803F07634236B79BD8A71A39688F
:100440005618AEBAAB558C1D3CB7CC5763BD6DED9D
:10045000FD753EF6177231BF000000803F080000B6
:1004600000BE922449123EABAAAA2ABECDCCCC4CE7
:100470003E00000080BEABAAAAAA3E00000000BF5A
:10048000000000803F0000000000084178D3BB431B
:1004900087D1133D190E3CC3BD4282AD2B3E68ECA3
:1004A0008276BED98FE1A93E4C80EFFFBE01C4FF2A
:1004B0007F3F0000000000000C94A8730C94BAA7C2
:1004C0000C946F740C9458BD0C9490BA0C94ACBA04
:1004D0000C94D8680C944B570C94D5630C94C96455
:1004E0000C9450C60C94A9790C9461750C9469C84D
:1004F0000C9478680C949C740C94C2CC0C941B776C
:100500000C94C6A70C94A1790C94D55A0C9456B9A6
:100510000C941A730C94CF5B0C94945E0C94555A03
:100520000C9458570C94A2BD0C94B7CD0C94B15AAE
:100530000C9492740C940C750C94C4740C943BBA87
:100540000C94E4790C94435B0C94B25D0C948CBADB
:100550000C9480670C94DA470C9474770C94D04711
:100560000C9464570C947B5E0C949ABD0C94CAADA9
:100570000C94E15A0C94FF710C94B6570C94C64736
:100580000C94BEA70C94B2AD0C943B780C94966876
:100590000C942E740C9451740C94726E0C94B55E81
:1005A0000C94FB740C9409720C9438740C94328281
:1005B0000C94CD630C94E5590C949EAD0C94C55AE3
:1005C0000C94D9630C94D15A0C9433630C94BB5B98
:1005D0000C94E9770C946C770C94A06B0C94765780
:1005E0000C9433770C948C840C9418AC0C945CCBE6
:1005F0000C94D9B90C94FA720C9494BA0C94FD5AD8
:100600000C942B770C94B0740C94B75B0C94B0548E
:100610000C94F55A0C945C590C9495570C94654BBA
:100620000C94F7C80C94CD5A0C941EC00C94D4575B
:100630000C94BABD0C942E750C9468770C9470775A
:100640000C94B4590C94C6AD0C94DD5A0C94B35B65
:100650000C9454580C941AAC0C945B740C946A5718
:100660000C949E800C94625E0C94DABD0C94F5712F
:100670000C94CEAD0C94E55A0C942ECD0C942B78A2
:100680000C947ABD0C9492BD0C9426BB0C94A75B81
:100690000C943F770C94F8720C94E9B90C94D55EE5
:1006A0000C94AEA70C94A0570C94F95A0C94815753
:1006B0000C94E5730C94CAA70C94F15A0C94D97459
:1006C0000C9419480C9443AC0C94175A0C941D7557
:1006D0000C9472BD0C94AABD0C94A5790C9446BDE3
:1006E0000C94746D0C94B2BD0C94E7770C94588004
:1006F0000C946ABD0C942A640C94FB4E0C945E64BA
:100700000C94FE5B0C948BAD0C9442740C94155FAE
:100710000C9437770C94F35B0C94B2720C944B6985
:100720000C94DE6E0C9473720C949CC00C941D5847
:100730000C9462B90C94A9640C9421790C94797A84
:100740000C94E75B0C94025A0C94C2A70C94EB71C6
:100750000C941D720C9427770C94576E0C94237A8A
:100760000C94B95A0C940EBB0C9488740C94BA7403
:100770000C94CEA70C9482BD0C94BF5B0C94AB710F
:100780000C94FB590C9413720C943C5F0C942A4803
:100790000C9494750C94C1920C94B6A70C942B5D98
:1007A0000C94B4BA0C9401BA0C94B2A70C94E472F1
:1007B0000C947E580C944E7A0C94EA740C94E37169
:1007C0000C949A800C94A8BA0C9460770C94D75B24
:1007D0000C94605E0C94054F0C94F4580C94CC77F8
:1007E0000C94645E0C94C3680C94CAC00C9483751A
:1007F0000C94D35B0C945CBD0C948B5D0C94226FB9
:100800000C940D610C94C15A0C9457730C941064A1
:100810000C940BC60C94A5750C94755F0C94EE7239
:100820000C9461730C9433C10C94C2BD0C94EABD5A
:100830000C9406BE0C9426AF0C940F730C94C471E8
:100840000C9403680C941CAC0C94095A0C9406BBD1
:100850000C94E9710C9479740C94875D0C9440BDF0
:100860000C9497CE0C9499790C94275E0C94BA71E1
:100870000C948ABD0C9433CE0C94E2BD0C94986B0E
:100880000C94EEBA0C94D95D0C94C1570C9441AC05
:100890000C94105A0C94F55E0C94F6BA0C946EC03D
:1008A0000C94205B0C9489640C9496800C9447AC57
:1008B0000C94365A0C94DB5B0C94B7580C94D8719A
:1008C0000C94B55A0C949FA80C94DF5B0C94B0BAAE
:1008D0000C94CABD0C947C630C949D790C94C95AF9
:1008E0000C94005E0C94D2AD0C94E95A0C947057A1
:1008F0000C948C570C9404730C94C35B0C94004FB1
:100900000C94E7580C9411630C94D6C80C945E5761
:100910000C9472750C9468C90C94D2BD0C9480CD63
:100920000C94D95A0C9416BB0C94B6750C94E2CF67
:100930000C9474790C9465740C944AB90C94FEBAB6
:100940000C9450750C9483740C9449680C9456C99B
:100950000C94DD630C9479790C942ECC0C94DE4EBF
:100960000C94CB5B0C94DF720C94625B0C943F5B39
:100970000C94BD5A0C94CE740C940A4F0C94ED5AFE
:100980000C94AB5B0C941EBB0C946B730C94C75B08
:100990000C944B770C94015B0C94CE710C94CE7537
:1009A0000C94D1630C94AB570C9443770C9499BA84
:1009B0000C94AF5B0C94AAA70C94E35B0C94E557E2
:1009C0000C9444640C94E0590C94A6740C945EBA94
:1009D0000C94FDAE0C941F770C943F755B2573252A
:1009E000735D20257320257320706F736974696FA0
:1009F0006E2531382E336625730A005B2573257307
:100A00005D202573202573206F666673657425321B
:100A1000302E336625730A005B257325735D202510
:100A200073207A65726F206261636B6F6666253131
:100A3000392E336625730A005B257325735D2025E7
:100A400073206C61746368206261636B6F666625F6
:100A500031382E336625730A005B257325735D20BC
:100A60002573206C617463682076656C6F636974AC
:100A7000792531332E306625732F6D696E0A005B40
:100A8000257325735D20257320736561726368206B
:100A900076656C6F636974792531322E3066257303
:100AA0002F6D696E0A005B257325735D2025732009
:100AB000737769746368206D617825313764205BD2
:100AC000303D6F66662C313D686F6D696E672C3204
:100AD0003D6C696D69742C333D6C696D69742B686C
:100AE0006F6D696E675D0A005B257325735D202558
:100AF0007320737769746368206D696E253137647C
:100B0000205B303D6F66662C313D686F6D696E67A6
:100B10002C323D6C696D69742C333D6C696D697460
:100B20002B686F6D696E675D0A005B257325735DC9
:100B3000202573207261646975732076616C756518
:100B40002532302E346625730A005B257325735DCC
:100B5000202573206A756E6374696F6E20646576F4
:100B6000696174696F6E2531342E346625732028CF
:100B70006C61726765722069732066617374657257
:100B8000290A005B257325735D202573206A657231
:100B90006B20686F6D696E672531362E3066257360
:100BA0002F6D696E5E33202A2031206D696C6C696F
:100BB0006F6E0A005B257325735D202573206A65BF
:100BC000726B206D6178696D756D2531352E3066DB
:100BD00025732F6D696E5E33202A2031206D696C7C
:100BE0006C696F6E0A005B257325735D2025732089
:100BF00074726176656C206D696E696D756D2531F5
:100C0000372E336625730A005B257325735D202517
:100C1000732074726176656C206D6178696D756D95
:100C20002531372E336625730A005B257325735DE6
:100C30002025732076656C6F63697479206D617807
:100C4000696D756D2531312E306625732F6D696E96
:100C50000A005B257325735D202573206665656436
:100C600072617465206D6178696D756D2531312E05
:100C7000306625732F6D696E0A005B257325735DE1
:100C80002025732061786973206D6F646525313884
:100C9000642025730A005B6D615D20206D696E2004
:100CA000617263207365676D656E742531382E330C
:100CB0006625730A005B736C5D2020736F66742079
:100CC0006C696D697420656E61626C652531326492
:100CD0000A005B63745D202063686F7264616C203E
:100CE000746F6C6572616E63652531372E346625CD
:100CF000730A005B6A615D20206A756E6374696FB8
:100D00006E20616363656C65726174696F6E25380E
:100D10002E306625730A005B6764695D2064656632
:100D200061756C742067636F6465206469737461B6
:100D30006E6365206D6F6465253264205B303D47CE
:100D400039302C313D4739315D0A005B6770615D98
:100D50002064656661756C742067636F64652070DC
:100D600061746820636F6E74726F6C253364205BEE
:100D7000303D4736312C313D4736312E312C323D16
:100D80004736345D0A005B67636F5D2064656661AA
:100D9000756C742067636F646520636F6F72642085
:100DA00073797374656D253364205B312D3620288B
:100DB0004735342D473539295D0A005B67756E5D0F
:100DC0002064656661756C742067636F6465207567
:100DD0006E697473206D6F6465253564205B303DEA
:100DE0004732302C313D4732315D0A005B67706C11
:100DF0005D2064656661756C742067636F6465204F
:100E0000706C616E6525313064205B303D47313751
:100E10002C313D4731382C323D4731395D0A0025B0
:100E20006320776F726B206F66667365743A253145
:100E3000322E336625730A002563206D616368696D
:100E40006E6520706F736E3A2531312E33662573CF
:100E50000A00256320706F736974696F6E3A2531DB
:100E6000352E336625730A00546F6F6C206E756DD6
:100E70006265722020202020202020202025640A66
:100E800000466565642072617465206D6F64653A23
:100E900020202020202025730A0044697374616E8D
:100EA0006365206D6F64653A202020202020202576
:100EB000730A0050617468204D6F64653A202020E9
:100EC000202020202020202025730A00506C616EF5
:100ED000653A2020202020202020202020202020B3
:100EE0002025730A004D6F74696F6E206D6F646505
:100EF0003A20202020202020202025730A00436F44
:100F00006F7264696E6174652073797374656D3A8C
:100F100020202025730A00556E6974733A20202022
:100F200020202020202020202020202025730A009F
:100F3000486F6D696E672073746174653A20202074
:100F4000202020202025730A0046656564686F6CA8
:100F5000642073746174653A20202020202025735A
:100F60000A004D6F74696F6E2073746174653A2066
:100F70002020202020202025730A004379636C65FF
:100F80002073746174653A202020202020202020C6
:100F900025730A00526177206D616368696E652070
:100FA00073746174653A20202025730A004D6163D3
:100FB00068696E652073746174653A202020202072
:100FC000202025730A004C696E65206E756D626580
:100FD000723A2531306C750A00466565642072618D
:100FE00074653A2531362E336625732F6D696E0A86
:100FF0000056656C6F636974793A2531372E336614
:1010000025732F6D696E0A005F102E100E10473980
:1010100035202D20756E6974732D7065722D726583
:10102000766F6C7574696F6E206D6F6465004739FB
:1010300034202D20756E6974732D7065722D6D6965
:101040006E757465206D6F64652028692E652E208D
:101050006665656472617465206D6F64652900471B
:101060003933202D20696E76657273652074696D41
:1010700065206D6F6465009B107B10473931202D12
:1010800020696E6372656D656E74616C206469734E
:1010900074616E6365206D6F646500473930202D83
:1010A000206162736F6C7574652064697374616E1E
:1010B0006365206D6F646500EC10D410BE10473678
:1010C00034202D20636F6E74696E756F7573206D9B
:1010D0006F6465004736312E31202D2065786163BD
:1010E000742073746F70206D6F6465004736312013
:1010F0002D2065786163742070617468206D6F6461
:101100006500261117110811473139202D20595A31
:1011100020706C616E6500473138202D20585A20B0
:10112000706C616E6500473137202D205859207052
:101130006C616E6500B211A011871166113F1147F5
:101140003830202D2063616E63656C206D6F74698B
:101150006F6E206D6F646520286E6F6E6520616311
:10116000746976652900473320202D20636F756EE2
:1011700074657220636C6F636B776973652061724D
:1011800063206665656400473220202D20636C6F04
:10119000636B7769736520617263206665656400BF
:1011A000473120202D206C696E656172206665656F
:1011B0006400473020202D206C696E6561722074B8
:1011C0007261766572736520287365656B29007995
:1011D000125F1245122B121112F711DD114735392A
:1011E000202D20636F6F7264696E6174652073795E
:1011F0007374656D203600473538202D20636F6F7E
:101200007264696E6174652073797374656D2035DD
:1012100000473537202D20636F6F7264696E6174EB
:10122000652073797374656D203400473536202D41
:1012300020636F6F7264696E617465207379737473
:10124000656D203300473535202D20636F6F726444
:10125000696E6174652073797374656D203200471F
:101260003534202D20636F6F7264696E6174652060
:1012700073797374656D203100473533202D206DEF
:10128000616368696E6520636F6F7264696E617413
:10129000652073797374656D00AC12A6129F1248B5
:1012A0006F6D696E6700486F6D6564004E6F7420E6
:1012B000486F6D656400E012DB12D612D012CB12BB
:1012C000C212456E6420486F6C6400486F6C640005
:1012D000446563656C00506C616E0053796E630009
:1012E0004F666600F312EF12EA12486F6C64005208
:1012F000756E0053746F70001D1313130D130613D6
:1013000002134A6F6700486F6D696E670050726F15
:101310006265004D616368696E696E67004F66665D
:101320000053134D13471342133E1338132F135317
:10133000687574646F776E004379636C6500456E01
:10134000640053746F7000416C61726D005265618E
:10135000647900496E697469616C697A696E6700C5
:10136000B613B013AA13A513A1139D1398139213C8
:101370008C1385138113781353687574646F776EBB
:10138000004A6F6700486F6D696E67004379636C50
:10139000650050726F626500486F6C640052756E34
:1013A00000456E640053746F7000416C61726D0093
:1013B000526561647900496E697469616C697A6922
:1013C0006E6700DD13C713473231202D206D696C25
:1013D0006C696D65746572206D6F646500473230AD
:1013E000202D20696E63686573206D6F646500173A
:1013F000140C140014F7135B7261646975735D005B
:101400005B696E686962697465645D005B737461D1
:101410006E646172645D005B64697361626C6564D3
:101420005D0031142D1428142064656700206D6D53
:101430000020696E002A2A2A204E4F544943452035
:101440002A2A2A20526573657474696E6720626166
:101450007564207261746520746F202573005B626F
:101460006175645D2055534220626175642072612C
:10147000746525313564205B313D393630302C328E
:101480003D31393230302C333D33383430302C3428
:101490003D35373630302C353D3131353230302C1A
:1014A000363D3233303430305D0A005B72786D5D2A
:1014B0002073657269616C205258206D6F646525D8
:1014C000313564205B303D636861725F6D6F6465C8
:1014D0002C313D6C696E655F6D6F64655D0A005B04
:1014E00065785D2020656E61626C6520666C6F7743
:1014F00020636F6E74726F6C25313064205B303DF9
:101500006F66662C313D584F4E2F584F46462C3251
:101510003D5254532F4354535D0A005B65655D2073
:1015200020656E61626C65206563686F2531386483
:10153000205B303D6F66662C313D6F6E5D0A005B4F
:1015400065635D2020657870616E64204C46207470
:101550006F2043524C46206F6E205458253664202D
:101560005B303D6F66662C313D6F6E5D0A00A115E4
:101570009C15961590158A1583157C1532333034D9
:1015800030300031313532303000353736303000D0
:101590003338343030003139323030003936303081
:1015A0000030007379730066620000000017029932
:1015B00079275E605E763C5C2FDC4373797300664E
:1015C000760000000017039D79275E605E7A3CEC90
:1015D00051783F737973006870000000000700A124
:1015E00079D95D645E7E3C0000803F73797300684A
:1015F00076000000001700A579275E79797F3C000E
:10160000000041737973006964000000000400A9C0
:10161000792179605E723C00000000000000006EDD
:1016200000000000000000B15AD95D945EED340066
:10163000000000000000006C696E6500000000B151
:101640005AD457945EED340000000000000000768C
:10165000656C0000001002175AE557605E723C008E
:10166000000000000000006665656400001002369E
:101670005A1D58605E723C000000000000000073BC
:1016800074617400000000B55A4B57605E723C00F4
:10169000000000000000006D61637300000000B9ED
:1016A0005A5857605E723C00000000000000006362
:1016B00079637300000000BD5A5E57605E723C00A3
:1016C000000000000000006D6F747300000000C196
:1016D0005A6457605E723C00000000000000006821
:1016E0006F6C6400000000C55A6A57605E723C006F
:1016F00000000000000000756E697400000000CD5D
:101700005A7657605E723C000000000000000063E3
:101710006F6F7200000000D15A8157605E723C000A
:10172000000000000000006D6F6D6F00000000D52C
:101730005A8C57605E723C00000000000000007090
:101740006C616E00000000D95A9557605E723C00D3
:10175000000000000000007061746800000000DDFF
:101760005AA057605E723C00000000000000006458
:1017700069737400000000E15AAB57605E723C0070
:101780000000000000000066726D6F00000000E5C0
:101790005AB657605E723C00000000000000007402
:1017A0006F6F6C00000000E95AC157605E723C0028
:1017B0000000006D706F006D706F7800001003F313
:1017C0005B7E58605E723C000000006D706F006DC3
:1017D000706F7900001003F35B7E58605E723C000E
:1017E0000000006D706F006D706F7A00001003F3E1
:1017F0005B7E58605E723C000000006D706F006D93
:10180000706F6100001003F35B7E58605E723C00F5
:101810000000006D706F006D706F6200001003F3C8
:101820005B7E58605E723C000000006D706F006D62
:10183000706F6300001003F35B7E58605E723C00C3
:10184000000000706F7300706F737800001003E782
:101850005B5458605E723C00000000706F73007053
:101860006F737900001003E75B5458605E723C00B0
:10187000000000706F7300706F737A00001003E750
:101880005B5458605E723C00000000706F73007023
:101890006F736100001003E75B5458605E723C0098
:1018A000000000706F7300706F736200001003E738
:1018B0005B5458605E723C00000000706F730070F3
:1018C0006F736300001003E75B5458605E723C0066
:1018D0000000006F6673006F66737800001003FEEF
:1018E0005BB758605E723C000000006F6673006F6B
:1018F00066737900001003FE5BB758605E723C00AF
:101900000000006F6673006F66737A00001003FEBC
:101910005BB758605E723C000000006F6673006F3A
:1019200066736100001003FE5BB758605E723C0096
:101930000000006F6673006F66736200001003FEA4
:101940005BB758605E723C000000006F6673006F0A
:1019500066736300001003FE5BB758605E723C0064
:10196000000000686F6D00686F6D6500000000C9C1
:101970005A7057E559723C00000000686F6D0068AE
:101980006F6D7800001000E75B8B5D605EC2340015
:10199000000000686F6D00686F6D7900001000E74F
:1019A0005B8B5D605EC33400000000686F6D006893
:1019B0006F6D7A00001000E75B8B5D605EC43400E1
:1019C000000000686F6D00686F6D6100001000E737
:1019D0005B8B5D605EC53400000000686F6D006861
:1019E0006F6D6200001000E75B8B5D605EC63400C7
:1019F000000000686F6D00686F6D6300001000E705
:101A00005B8B5D605EC73400000000707262007026
:101A1000726265000000001EC08B5D605EC834000D
:101A20000000007072620070726278000010031E85
:101A3000C0275E605EC934000000007072620070F2
:101A4000726279000010031EC0275E605ECD340014
:101A5000000000707262007072627A000010031E53
:101A6000C0275E605ED134000000007072620070BA
:101A7000726261000010031EC0275E605ED53400F4
:101A80000000007072620070726262000010031E3B
:101A9000C0275E605ED93400000000707262007082
:101AA000726263000010031EC0275E605EDD3400BA
:101AB0000000006A6F67006A6F6778000010001E00
:101AC000C0875DFB59E734000000006A6F67006A59
:101AD0006F6779000010001EC0875D025AE734006E
:101AE0000000006A6F67006A6F677A000010001ECE
:101AF000C0875D095AE734000000006A6F67006A1A
:101B00006F6761000010001EC0875D105AE7340047
:101B1000000000707772007077723100000000B42E
:101B2000BAE9B9605E723C00000000707772007024
:101B300077723200000000B4BAE9B9605E723C000E
:101B4000000000707772007077723300000000B4FC
:101B5000BAE9B9605E723C000000007077720070F4
:101B600077723400000000B4BAE9B9605E723C00DC
:101B700000000031000000316D61000000030090A2
:101B8000BA8B5D645EF05A00000000310000003145
:101B90007361000000130394BA275E4AB9FB5A66CA
:101BA00066E63F310000003174720000001B0499AA
:101BB000BA275E56B9FF5A000020423100000031BA
:101BC0006D690000000300A8BA8B5D62B9F15A008C
:101BD0000000413100000031706F0000000300ACD4
:101BE000BA8B5DB55EF55A0000803F3100000031D0
:101BF000706D0000000300B0BA8B5DD9B9F65A00D1
:101C000000004032000000326D61000000030090CF
:101C1000BA8B5D645E0F5B0000803F3200000032D3
:101C20007361000000130394BA275E4AB91A5B6619
:101C300066E63F320000003274720000001B049917
:101C4000BA275E56B91E5B00002042320000003207
:101C50006D690000000300A8BA8B5D62B9105B00DB
:101C60000000413200000032706F0000000300AC41
:101C7000BA8B5DB55E145B0000803F32000000321D
:101C8000706D0000000300B0BA8B5DD9B9155B0020
:101C900000004033000000336D610000000300903D
:101CA000BA8B5D645E2E5B0000803F330000003322
:101CB0007361000000130394BA275E4AB9395B666A
:101CC00066E63F330000003374720000001B049985
:101CD000BA275E56B93D5B00002042330000003356
:101CE0006D690000000300A8BA8B5D62B92F5B002C
:101CF0000000413300000033706F0000000300ACAF
:101D0000BA8B5DB55E335B0000000033000000332A
:101D1000706D0000000300B0BA8B5DD9B9345B0070
:101D200000004034000000346D61000000030090AA
:101D3000BA8B5D645E4D5B000000403400000034EF
:101D40007361000000130394BA275E4AB9585B66BA
:101D500066E63F340000003474720000001B0499F2
:101D6000BA275E56B95C5B607607403400000034E9
:101D70006D690000000300A8BA8B5D62B94E5B007C
:101D80000000413400000034706F0000000300AC1C
:101D9000BA8B5DB55E525B0000803F3400000034BA
:101DA000706D0000000300B0BA8B5DD9B9535B00C1
:101DB0000000407800000078616D000000030062C0
:101DC0005BE758F4587E330000803F7800000078CD
:101DD000766D0000001B00AB5B275E7C63833300E5
:101DE000007A46780000007866720000001B00A7A9
:101DF0005B275E7C637F3300007A467800000078C2
:101E0000746E0000001B03B35B275E7C638B3300A2
:101E10000000007800000078746D0000001B03AF24
:101E20005B275E7C63873300009143780000007875
:101E30006A6D0000001B00B75B275E5C598F3300A2
:101E4000409C4578000000786A680000001B00BBD9
:101E50005B275EB459933300401C4678000000783D
:101E60006A640000001B04BF5B275E7C639B330A2F
:101E7000D7233C7800000078736E0000000300C791
:101E80005B8B5D46BDA2320000803F780000007889
:101E900073780000000300CB5B8B5D46BDA332006E
:101EA000000000780000007873760000001B00CF6F
:101EB0005B275E7C63A33300803B4578000000789D
:101EC0006C760000001B00D35B275E7C63A73300A9
:101ED00000C84278000000786C620000001B03D745
:101EE0005B275E7C63AB3300002041780000007804
:101EF0007A620000001B03DB5B275E7C63AF33006C
:101F00000000407900000079616D0000000300626C
:101F10005BE758F458B3330000803F790000007944
:101F2000766D0000001B00AB5B275E7C63B833005E
:101F3000007A46790000007966720000001B00A755
:101F40005B275E7C63B43300007A46790000007939
:101F5000746E0000001B03B35B275E7C63C033001C
:101F60000000007900000079746D0000001B03AFD1
:101F70005B275E7C63BC330000A0437900000079DE
:101F80006A6D0000001B00B75B275E5C59C433001C
:101F9000409C4579000000796A680000001B00BB86
:101FA0005B275EB459C83300401C467900000079B5
:101FB0006A640000001B04BF5B275E7C63D0330AA9
:101FC000D7233C7900000079736E0000000300C73E
:101FD0005B8B5D46BDA4320000803F790000007934
:101FE00073780000000300CB5B8B5D46BDA532001B
:101FF000000000790000007973760000001B00CF1C
:102000005B275E7C63D83300803B45790000007914
:102010006C760000001B00D35B275E7C63DC330022
:1020200000C84279000000796C620000001B03D7F1
:102030005B275E7C63E0330000204179000000797B
:102040007A620000001B03DB5B275E7C63E43300E5
:102050000000407A0000007A616D00000003006219
:102060005BE758F458E8330000803F7A0000007ABC
:10207000766D0000001B00AB5B275E7C63ED3300D8
:10208000007A447A0000007A66720000001B00A704
:102090005B275E7C63E93300007A447A0000007AB3
:1020A000746E0000001B03B35B275E7C63F5330096
:1020B00000F0C27A0000007A746D0000001B03AFCC
:1020C0005B275E7C63F133000000007A0000007A39
:1020D0006A6D0000001B00B75B275E5C59F9330096
:1020E0000048427A0000007A6A680000001B00BBCA
:1020F0005B275EB459FD3300007A447A0000007A11
:102100006A640000001B04BF5B275E7C6305340A21
:10211000D7233C7A0000007A736E0000000300C7EA
:102120005B8B5D46BDA632000000007A0000007A9D
:1021300073780000000300CB5B8B5D46BDA73200C7
:1021400000803F7A0000007A73760000001B00CF09
:102150005B275E7C630D3400007A447A0000007ACD
:102160006C760000001B00D35B275E7C631134009B
:1021700000C8427A0000007A6C620000001B03D79E
:102180005B275E7C631534000020417A0000007AF2
:102190007A620000001B03DB5B275E7C631934005E
:1021A0000040406100000061616D000000030062BA
:1021B0005BE758F4581D34000040406100000061A6
:1021C000766D0000001300AB5B275E3C5F2234009D
:1021D00080CA46610000006166720000001300A71B
:1021E0005B275E3C5F1E3400804A46610000006150
:1021F000746E0000001303B35B275E7C632A340017
:102200000080BF6100000061746D0000001303AF27
:102210005B275E3C5F2634000080BF6100000061E8
:102220006A6D0000001300B75B275E5C592E340016
:10223000349E4861000000616A680000001300BB22
:102240005B275EB459323400349E4861000000615F
:102250006A640000001304BF5B275E3C5F3A34CD24
:10226000CCCC3D610000006172610000001B03C323
:102270005B275E3C5F3E34DFC3A940610000006124
:10228000736E0000000300C75B8B5D46BDA8320083
:1022900000803F610000006173780000000300CB04
:1022A0005B8B5D46BDA9320000000061000000614B
:1022B00073760000001300CF5B275E3C5F42340062
:1022C00000FA4461000000616C760000001300D346
:1022D0005B275E3C5F46340000FA44610000006109
:1022E0006C620000001303D75B275E3C5F4A34003A
:1022F00000A04061000000617A620000001303DB6F
:102300005B275E3C5F4E34000000406200000062CC
:10231000616D0000000300625BE758F4585234001E
:102320000000006200000062766D0000001300AB48
:102330005B275E3C5F57340000614562000000622D
:1023400066720000001300A75B275E3C5F533400F9
:102350000061456200000062746E0000001303B368
:102360005B275E7C635F34000080BF620000006218
:10237000746D0000001303AF5B275E3C5F5B3400AD
:102380000080BF62000000626A6D0000001300B7A9
:102390005B275E5C5963340000A04162000000626C
:1023A0006A640000001300BF5B275E3C5F6F340A65
:1023B000D7233C620000006272610000001B03C36F
:1023C0005B275E3C5F73340000803F630000006366
:1023D000616D0000000300625BE758F45887340029
:1023E0000000006300000063766D0000001300AB86
:1023F0005B275E3C5F8C3400006145630000006336
:1024000066720000001300A75B275E3C5F88340003
:102410000061456300000063746E0000001303B3A5
:102420005B275E7C639434000080BF630000006320
:10243000746D0000001303AF5B275E3C5F903400B7
:102440000080BF63000000636A6D0000001300B7E6
:102450005B275E5C5998340000A041630000006374
:102460006A640000001300BF5B275E3C5FA4340A6F
:10247000D7233C630000006372610000001B03C3AC
:102480005B275E3C5FA8340000803F703100007025
:1024900031667271001300AAA7275E3C5FCC590019
:1024A00000C84270310000703163736C001300AEDD
:1024B000A7275E3C5FD05900007A4470310000705D
:1024C00031637368001300B2A7275E3C5FD45900E4
:1024D00000FA4470310000703163706C001303B671
:1024E000A7275E3C5FD8590000003E7031000070A5
:1024F00031637068001303BAA7275E3C5FDC59CDD7
:10250000CC4C3E70310000703177736C001300BE0C
:10251000A7275E3C5FE05900007A447031000070EC
:1025200031777368001300C2A7275E3C5FE459004F
:1025300000FA4470310000703177706C001303C6EC
:10254000A7275E3C5FE8590000003E703100007034
:1025500031777068001303CAA7275E3C5FEC59CD42
:10256000CC4C3E703100007031706F66001303CEAA
:10257000A7275E3C5FF059CDCCCC3D673534006772
:1025800035347800001B03DF5B275E7C63EE32008E
:10259000000000673534006735347900001B03DF25
:1025A0005B275E7C63F23200000000673534006711
:1025B00035347A00001B03DF5B275E7C63F6320054
:1025C000000000673534006735346100001B03DF0D
:1025D0005B275E3C5FFA320000000067353400671D
:1025E00035346200001B03DF5B275E3C5FFE320078
:1025F000000000673534006735346300001B03DFDB
:102600005B275E3C5F0233000000006735350067E2
:1026100035357800001B03DF5B275E7C63063300E3
:10262000001143673535006735357900001B03DF3E
:102630005B275E7C630A3300002043673535006703
:1026400035357A00001B03DF5B275E7C630E3300A9
:10265000000000673535006735356100001B03DF7A
:102660005B275E3C5F123300000000673535006772
:1026700035356200001B03DF5B275E3C5F163300CD
:10268000000000673535006735356300001B03DF48
:102690005B275E3C5F1A3300000000673536006739
:1026A00035367800001B03DF5B275E7C631E33003A
:1026B000000000673536006735367900001B03DF00
:1026C0005B275E7C632233000000006735360067BD
:1026D00035367A00001B03DF5B275E7C6326330000
:1026E000000000673536006735366100001B03DFE8
:1026F0005B275E3C5F2A33000000006735360067C9
:1027000035366200001B03DF5B275E3C5F2E330023
:10271000000000673536006735366300001B03DFB5
:102720005B275E3C5F32330000000067353700678F
:1027300035377800001B03DF5B275E7C6336330090
:10274000000000673537006735377900001B03DF6D
:102750005B275E7C633A3300000000673537006713
:1027600035377A00001B03DF5B275E7C633E330056
:10277000000000673537006735376100001B03DF55
:102780005B275E3C5F42330000000067353700671F
:1027900035376200001B03DF5B275E3C5F4633007A
:1027A000000000673537006735376300001B03DF23
:1027B0005B275E3C5F4A33000000006735380067E6
:1027C00035387800001B03DF5B275E7C634E3300E7
:1027D000000000673538006735387900001B03DFDB
:1027E0005B275E7C6352330000000067353800676A
:1027F00035387A00001B03DF5B275E7C63563300AD
:10280000000000673538006735386100001B03DFC2
:102810005B275E3C5F5A3300000000673538006775
:1028200035386200001B03DF5B275E3C5F5E3300D0
:10283000000000673538006735386300001B03DF90
:102840005B275E3C5F62330000000067353900673C
:1028500035397800001B03DF5B275E7C636633003D
:10286000000000673539006735397900001B03DF48
:102870005B275E7C636A33000000006735390067C0
:1028800035397A00001B03DF5B275E7C636E330003
:10289000000000673539006735396100001B03DF30
:1028A0005B275E3C5F7233000000006735390067CC
:1028B00035396200001B03DF5B275E3C5F76330027
:1028C000000000673539006735396300001B03DFFE
:1028D0005B275E3C5F7A3300000000673932006797
:1028E00039327800001103DF5B275E605E5F3500E0
:1028F000000000673932006739327900001103DFC8
:102900005B275E605E633500000000673932006758
:1029100039327A00001103DF5B275E605E673500A5
:10292000000000673932006739326100001103DFAF
:102930005B275E605E6B3500000000673932006720
:1029400039326200001103DF5B275E605E6F350085
:10295000000000673932006739326300001103DF7D
:102960005B275E605E7335000000006732380067E9
:1029700032387800001103E35B275E605E77350034
:10298000000000673238006732387900001103E335
:102990005B275E605E7B35000000006732380067B1
:1029A00032387A00001103E35B275E605E7F3500FA
:1029B000000000673238006732386100001103E31D
:1029C0005B275E605E833500000000673238006779
:1029D00032386200001103E35B275E605E873500DA
:1029E000000000673238006732386300001103E3EB
:1029F0005B275E605E8B3500000000673330006748
:102A000033307800001103E35B275E605E8F350092
:102A1000000000673330006733307900001103E3B2
:102A20005B275E605E93350000000067333000670F
:102A300033307A00001103E35B275E605E97350058
:102A4000000000673330006733306100001103E39A
:102A50005B275E605E9B35000000006733300067D7
:102A600033306200001103E35B275E605E9F350038
:102A7000000000673330006733306300001103E368
:102A80005B275E605EA335000000006A6964006A2F
:102A9000696461000000001EC0005E155F923C008A
:102AA0000000006A6964006A696462000000001E38
:102AB000C0005E155F963C000000006A6964006A11
:102AC000696463000000001EC0005E155F9A3C0050
:102AD0000000006A6964006A696464000000001E06
:102AE000C0005E155F9E3C00000000737973006AB1
:102AF00061000000001F00015B275E7C63BC3200A8
:102B000024F449737973006374000000001F0420EB
:102B10005B275E7C63C0320AD7233C7379730073F2
:102B20006C0000000007003F5B8B5D645EC43200F8
:102B300000000073797300737400000000070058F0
:102B4000BD8B5D40BD97320000803F737973006D8F
:102B5000740000000017028CBA275E01BAEC5A001C
:102B6000000040000000006D650000000000006EE5
:102B7000C05EBA5EBA723C00000000000000006D4A
:102B8000640000000000006EC03BBA3BBA723C001B
:102B900000000073797300656A000000000700966A
:102BA000808B5DB55E843C0000803F737973006A62
:102BB000760000000007009A808B5D58805C3F0023
:102BC00000A040737973006A730000000007009E44
:102BD000808B5DB55E5D3F0000803F73797300744C
:102BE0007600000000070033C18B5DB55E5F5C00BE
:102BF00000803F737973007176000000000700D2F7
:102C0000AD8B5DF55E255A0000000073797300738B
:102C10007600000000070047AC8B5DD55E325A009D
:102C200000803F7379730073690000000007004360
:102C3000ACD95D1CAC335A00007A437379730065DC
:102C400063000000000700CD638B5DC9647432002F
:102C5000000000737973006565000000000700D173
:102C6000638B5DA9647532000000007379730065A1
:102C700078000000000700D5638B5D896476320020
:102C80000000407379730072786D0000000700D96E
:102C9000638B5DB55E77320000803F7379730062AD
:102CA00061756400000400DD638B5D336372320084
:102CB00000A040000000007372000000000000410E
:102CC000AC18AC1AAC723C000000000000000071AF
:102CD00072000000000000C6AD8BAD605E723C006B
:102CE000000000000000007169000000000000CA40
:102CF000AD9EAD605E723C000000000000000071FF
:102D00006F000000000000CEADB2AD605E723C000E
:102D10000000000000000065720000000000001EBE
:102D2000C09FA8605E723C000000000000000071BF
:102D3000660000000000001EC0875DE059723C0084
:102D40000000000000000072780000000000009CFD
:102D5000C01163605E723C00000000000000006D66
:102D6000736700000000006EC0875D605E723C000B
:102D700000000000000000636C6561720000001E2E
:102D8000C0DE4EDE4E723C00000000000000006815
:102D90006F6C64000000001EC0FB4EFB4E723C00D6
:102DA0000000000000000073746172740000001ED7
:102DB000C0004F004F723C000000000000000066A1
:102DC0006C7573680000001EC0054F054F723C0013
:102DD0000000000000000072657365740000001EB2
:102DE000C00A4F0A4F723C0000000000000000744F
:102DF000787400000000001EC0875D625E723C00B7
:102E00000000000000000074696400000001009CE4
:102E1000C0D95D945EA23C00000000000000007478
:102E2000657374000000001EC0237A5CBD723C0014
:102E30000000000000000064656661000000001EE4
:102E4000C04E7A2B5D723C00000000000000006262
:102E50006F6F74000000001EC0797A7479723C00B4
:102E60000000000000000068656C70000000001E9B
:102E7000C0E479605E723C00000000000000006861
:102E8000000000000000001EC0E479605E723C009B
:102E90000000007379730067706C0000000700ED9C
:102EA0005A8B5DD55ED232000000007379730067E3
:102EB000756E0000000700F15A8B5DB55ED33200DD
:102EC00000803F7379730067636F0000000700F5AF
:102ED0005A8B5D645ED1320000803F737973006766
:102EE00070610000000700F95A8B5DD55ED4320096
:102EF000000040737973006764690000000700FDFB
:102F00005A8B5DB55ED532000000000000000067FE
:102F1000630000000000001EC02B783B78723C006C
:102F2000000000000000006D61000000001B044371
:102F30005B275E7C63C932CDCCCC3D0000000066CF
:102F4000640000000003009CC08B5DB55E5E3F0026
:102F50000000007564610075646130000003009C2E
:102F6000C0005E155F2E3C000000007564610075B6
:102F7000646131000003009CC0005E155F323C00BC
:102F80000000007564610075646132000003009CFC
:102F9000C0005E155F363C0000000075646100757E
:102FA000646133000003009CC0005E155F3A3C0082
:102FB0000000007564620075646230000003009CCC
:102FC000C0005E155F3E3C00000000756462007545
:102FD000646231000003009CC0005E155F423C004B
:102FE0000000007564620075646232000003009C9A
:102FF000C0005E155F463C0000000075646200750D
:10300000646233000003009CC0005E155F4A3C0010
:103010000000007564630075646330000003009C69
:10302000C0005E155F4E3C000000007564630075D3
:10303000646331000003009CC0005E155F523C00D9
:103040000000007564630075646332000003009C37
:10305000C0005E155F563C0000000075646300759B
:10306000646333000003009CC0005E155F5A3C009F
:103070000000007564640075646430000003009C07
:10308000C0005E155F5E3C00000000756464007562
:10309000646431000003009CC0005E155F623C0068
:1030A0000000007564640075646432000003009CD5
:1030B000C0005E155F663C0000000075646400752A
:1030C000646433000003009CC0005E155F6A3C002E
:1030D0000000005F7465005F74657800001002CA2C
:1030E000C0275E605E9557000000005F7465005F5A
:1030F00074657900001002CAC0275E605E995700AF
:103100000000005F7465005F74657A00001002CAF9
:10311000C0275E605E9D57000000005F7465005F21
:1031200074656100001002CAC0275E605EA157008E
:103130000000005F7465005F74656200001002CAE1
:10314000C0275E605EA557000000005F7465005FE9
:1031500074656300001002CAC0275E605EA9570054
:103160000000005F7472005F74727800001002CA81
:10317000C0275E605EBA58000000005F7472005F96
:1031800074727900001002CAC0275E605EBE5800EB
:103190000000005F7472005F74727A00001002CA4F
:1031A000C0275E605EC258000000005F7472005F5E
:1031B00074726100001002CAC0275E605EC65800CB
:1031C0000000005F7472005F74726200001002CA37
:1031D000C0275E605ECA58000000005F7472005F26
:1031E00074726300001002CAC0275E605ECE580091
:1031F0000000005F7473005F74733100001002CA36
:10320000C0275E605E2558000000005F7073005F9D
:1032100070733100001002CAC0275E605E3558002E
:103220000000005F6373005F63733100001002CA27
:10323000C0275E605E4558000000005F6573005F58
:1032400065733100001002CAC0275E605E555800E9
:103250000000005F7873005F78733100001002CACD
:10326000C0275E605E875B000000005F6665005FF0
:1032700066653100001002CAC0275E605E655800B6
:103280000000005F7473005F74733200001002CAA4
:10329000C0275E605E2958000000005F7073005F09
:1032A00070733200001002CAC0275E605E39580099
:1032B0000000005F6373005F63733200001002CA96
:1032C000C0275E605E4958000000005F6573005FC4
:1032D00065733200001002CAC0275E605E59580054
:1032E0000000005F7873005F78733200001002CA3C
:1032F000C0275E605E9F5B000000005F6665005F48
:1033000066653200001002CAC0275E605E69580020
:103310000000005F7473005F74733300001002CA12
:10332000C0275E605E2D58000000005F7073005F74
:1033300070733300001002CAC0275E605E3D580003
:103340000000005F6373005F63733300001002CA04
:10335000C0275E605E4D58000000005F6573005F2F
:1033600065733300001002CAC0275E605E5D5800BE
:103370000000005F7873005F78733300001002CAAA
:10338000C0275E605EB75B000000005F6665005F9F
:1033900066653300001002CAC0275E605E6D58008B
:1033A0000000005F7473005F74733400001002CA81
:1033B000C0275E605E3158000000005F7073005FE0
:1033C00070733400001002CAC0275E605E4158006E
:1033D0000000005F6373005F63733400001002CA73
:1033E000C0275E605E5158000000005F6573005F9B
:1033F00065733400001002CAC0275E605E61580029
:103400000000005F7873005F78733400001002CA18
:10341000C0275E605ECF5B000000005F6665005FF6
:1034200066653400001002CAC0275E605E715800F5
:10343000000000000000005F64616D000000001EDD
:10344000C0555A555A723C0000000000000000733D
:10345000653030000002001EC0B25D7B5E3E5A0047
:103460000000000000000073653031000002001E03
:10347000C0B25D7B5E405A00000000000000007397
:10348000653032000002001EC0B25D7B5E425A0011
:103490000000000000000073653033000002001ED1
:1034A000C0B25D7B5E445A00000000000000007363
:1034B000653034000002001EC0B25D7B5E465A00DB
:1034C0000000000000000073653035000002001E9F
:1034D000C0B25D7B5E485A0000000000000000732F
:1034E000653036000002001EC0B25D7B5E4A5A00A5
:1034F0000000000000000073653037000002001E6D
:10350000C0B25D7B5E4C5A000000000000000073FA
:10351000653038000002001EC0B25D7B5E4E5A006E
:103520000000000000000073653039000002001E3A
:10353000C0B25D7B5E505A000000000000000073C6
:10354000653130000002001EC0B25D7B5E525A0041
:103550000000000000000073653131000002001E11
:10356000C0B25D7B5E545A00000000000000007392
:10357000653132000002001EC0B25D7B5E565A000B
:103580000000000000000073653133000002001EDF
:10359000C0B25D7B5E585A0000000000000000735E
:1035A000653134000002001EC0B25D7B5E5A5A00D5
:1035B0000000000000000073653135000002001EAD
:1035C000C0B25D7B5E5C5A0000000000000000732A
:1035D000653136000002001EC0B25D7B5E5E5A009F
:1035E0000000000000000073653137000002001E7B
:1035F000C0B25D7B5E605A000000000000000073F6
:10360000653138000002001EC0B25D7B5E625A0068
:103610000000000000000073653139000002001E48
:10362000C0B25D7B5E645A000000000000000073C1
:10363000653230000002001EC0B25D7B5E665A003B
:103640000000000000000073653231000002001E1F
:10365000C0B25D7B5E685A0000000000000000738D
:10366000653232000002001EC0B25D7B5E6A5A0005
:103670000000000000000073653233000002001EED
:10368000C0B25D7B5E6C5A00000000000000007359
:10369000653234000002001EC0B25D7B5E6E5A00CF
:1036A0000000000000000073653235000002001EBB
:1036B000C0B25D7B5E705A00000000000000007325
:1036C000653236000002001EC0B25D7B5E725A0099
:1036D0000000000000000073653237000002001E89
:1036E000C0B25D7B5E745A000000000000000073F1
:1036F000653238000002001EC0B25D7B5E765A0063
:103700000000000000000073653239000002001E56
:10371000C0B25D7B5E785A000000000000000073BC
:10372000797300000000001EC00D61755F723C00DF
:103730000000000000000070310000000000001ECA
:10374000C00D61755F723C00000000000000003198
:10375000000000000000001EC00D61755F723C009B
:103760000000000000000032000000000000001E09
:10377000C00D61755F723C00000000000000003366
:10378000000000000000001EC00D61755F723C006B
:103790000000000000000034000000000000001ED7
:1037A000C00D61755F723C000000000000000078F1
:1037B000000000000000001EC00D61755F723C003B
:1037C0000000000000000079000000000000001E62
:1037D000C00D61755F723C00000000000000007ABF
:1037E000000000000000001EC00D61755F723C000B
:1037F0000000000000000061000000000000001E4A
:10380000C00D61755F723C000000000000000062A6
:10381000000000000000001EC00D61755F723C00DA
:103820000000000000000063000000000000001E17
:10383000C00D61755F723C00000000000000006771
:10384000353400000000001EC00D61755F723C0041
:103850000000000000000067353500000000001E79
:10386000C00D61755F723C00000000000000006741
:10387000353600000000001EC00D61755F723C000F
:103880000000000000000067353700000000001E47
:10389000C00D61755F723C00000000000000006711
:1038A000353800000000001EC00D61755F723C00DD
:1038B0000000000000000067353900000000001E15
:1038C000C00D61755F723C000000000000000067E1
:1038D000393200000000001EC00D61755F723C00AF
:1038E0000000000000000067323800000000001EE9
:1038F000C00D61755F723C000000000000000067B1
:10390000333000000000001EC00D61755F723C0086
:10391000000000000000006D706F00000000001E3D
:10392000C00D61755F723C00000000000000007077
:103930006F7300000000001EC00D61755F723C00D7
:10394000000000000000006F667300000000001E11
:10395000C00D61755F723C0000000000000000684F
:103960006F6D00000000001EC00D61755F723C00AD
:103970000000000000000070726200000000001EE5
:10398000C00D61755F723C00000000000000007017
:10399000777200000000001EC00D61755F723C0070
:1039A000000000000000006A6F6700000000001EB9
:1039B000C00D61755F723C00000000000000006AED
:1039C000696400000000001EC00D61755F723C005C
:1039D0000000000000000075646100000000001E8F
:1039E000C00D61755F723C000000000000000075B2
:1039F000646200000000001EC00D61755F723C0033
:103A00000000000000000075646300000000001E5C
:103A1000C00D61755F723C00000000000000007581
:103A2000646400000000001EC00D61755F723C0000
:103A3000000000000000005F746500000000001E30
:103A4000C00D61755F723C00000000000000005F67
:103A5000747200000000001EC00D61755F723C00B2
:103A6000000000000000005F747300000000001EF2
:103A7000C00D61755F723C00000000000000005F37
:103A8000707300000000001EC00D61755F723C0085
:103A9000000000000000005F637300000000001ED3
:103AA000C00D61755F723C00000000000000005F07
:103AB000657300000000001EC00D61755F723C0060
:103AC000000000000000005F787300000000001E8E
:103AD000C00D61755F723C00000000000000005FD7
:103AE000666500000000001EC00D61755F723C003D
:103AF000000000000000006D000000000000001E3B
:103B0000C04464605E723C00000000000000007170
:103B1000000000000000001EC02A64605E723C00CD
:103B2000000000000000006F000000000000001E08
:103B3000C01064605E723C000000000000000024C1
:103B4000000000000000001EC05E64605E723C0069
:103B5000000000486F6D696E67206572726F722099
:103B60002D20256320617869732073657474696EF4
:103B70006773206D6973636F6E66696775726564DC
:103B80000050726F62696E67206572726F72202DCD
:103B900020256320617869732063616E6E6F7420E5
:103BA0006D6F766520647572696E672070726F62E2
:103BB000696E67005B69645D202054696E794720F7
:103BC0004944253330730A005B68765D20206861C4
:103BD0007264776172652076657273696F6E2531E4
:103BE000362E32660A005B68705D20206861726460
:103BF0007761726520706C6174666F726D25313209
:103C0000640A005B66765D20206669726D7761727A
:103C1000652076657273696F6E2531362E32660ABD
:103C2000005B66625D20206669726D776172652057
:103C30006275696C642531382E32660A00456E74EF
:103C400065722024626F6F743D3120746F20656E41
:103C50007465722074686520626F6F74206C6F6188
:103C60006465722E0A000A0A0A2323232054696E0F
:103C7000794720424F4F54204C4F414445522048F1
:103C8000656C70202323230A00456E74657220241E
:103C9000646566613D3120746F20726573657420C0
:103CA0007468652073797374656D20746F2074680F
:103CB0006520666163746F72792064656661756CF6
:103CC000742076616C7565732E0A54686973207769
:103CD000696C6C206F766572777269746520616EAD
:103CE00079206368616E67657320796F75206861FC
:103CF0007665206D6164652E0A000A0A0A23232373
:103D00002054696E794720524553544F5245204400
:103D1000454641554C54532048656C70202323235D
:103D20000A00496E766F6B652073656C662074655A
:103D3000737420627920656E746572696E672024E1
:103D4000746573743D4E207768657265204E2069F6
:103D500073206F6E65206F663A0A202024746573A5
:103D6000743D312020736D6F6B6520746573740A28
:103D7000202024746573743D322020686F6D696E55
:103D800067207465737420202028796F75206D7505
:103D90007374207472697020686F6D696E67207328
:103DA00077697463686573290A20202474657374C5
:103DB0003D332020737175617265207465737420C2
:103DC0002020286120736572696573206F662073F7
:103DD000717561726573290A202024746573743DBE
:103DE00034202061726320746573742020202020A9
:103DF0002028736F6D65206C61726765206369723E
:103E0000636C6573290A202024746573743D352022
:103E1000206477656C6C20746573742020202028E2
:103E20006D6F7665732073706163656420627920BD
:103E300031207365636F6E64206477656C6C7329E1
:103E40000A202024746573743D36202066656564FD
:103E5000686F6C6420746573742028656E74657275
:103E6000202120616E64207E20746F20686F6C6456
:103E700020616E6420726573746172742C207265A7
:103E800073706563746976656C79290A20202474DF
:103E90006573743D3720204D20636F646573207413
:103EA0006573742020284D20636F64657320696EEC
:103EB0007465726D696E676C6564207769746820DB
:103EC0006D6F766573290A202024746573743D38FC
:103ED00020204A534F4E20746573742020202020E8
:103EE000286D6F74696F6E20746573742072756EBF
:103EF000207573696E67204A534F4E20636F6D6D56
:103F0000616E6473290A202024746573743D39201E
:103F100020696E76657273652074696D65207465BD
:103F200073740A202024746573743D313020726FDD
:103F300074617279206D6F74696F6E20746573742B
:103F40000A202024746573743D313120736D616CD7
:103F50006C206D6F76657320746573740A2020245D
:103F6000746573743D313220736C6F77206D6F769A
:103F7000657320746573740A202024746573743D1E
:103F8000313320636F6F7264696E61746520737979
:103F90007374656D206F66667365742074657374E1
:103FA00020284739322C204735342D473539290A06
:103FB0000A546573747320617373756D6520612095
:103FC00063656E7465726564205859206F72696705
:103FD000696E20616E64206174206C656173742069
:103FE00038306D6D20636C656172616E6365206948
:103FF0006E20616C6C20646972656374696F6E73A6
:104000000A546573747320617373756D65205A204B
:10401000686173206174206C656173742034306D45
:104020006D20706F7369697469766520636C656172
:1040300072616E63650A5465737473207374617280
:1040400074207769746820612047302058302059E7
:1040500030205A30206D6F76650A486F6D696E6743
:104060002069732074686520657863657074696F72
:104070006E2E204E6F20696E697469616C20706FBE
:10408000736974696F6E206F7220636C6561726111
:104090006E636520697320617373756D65640A00D2
:1040A0000A0A0A2323232054696E79472053454C7A
:1040B0004620544553542048656C70202323230A1E
:1040C0000045616368202420636F6D6D616E64201C
:1040D00061626F766520616C736F20646973706CC8
:1040E0006179732074686520746F6B656E20666FEC
:1040F0007220656163682073657474696E672069F6
:104100006E205B205D20627261636B6574730A547C
:104110006F20766965772073657474696E677320A4
:10412000656E746572206120746F6B656E3A0A0A61
:104130002020243C746F6B656E3E0A0A466F722025
:104140006578616D706C65202479667220746F20CB
:10415000646973706C6179207468652059206D61A1
:1041600078206665656420726174650A0A546F2060
:104170007570646174652073657474696E6773200B
:10418000656E74657220746F6B656E206571756104
:104190006C732076616C75653A0A0A2020243C74A1
:1041A0006F6B656E3E3D3C76616C75653E0A0A46F6
:1041B0006F72206578616D706C6520247966723D40
:1041C00038303020746F207365742074686520590E
:1041D000206D617820666565642072617465207465
:1041E0006F20383030206D6D2F6D696E7574650AE3
:1041F000466F7220636F6E66696775726174696F6E
:104200006E2064657461696C73207365653A20681B
:10421000747470733A2F2F6769746875622E636FB8
:104220006D2F73796E746865746F732F54696E792E
:10423000472F77696B692F54696E79472D436F6EED
:1042400066696775726174696F6E0A005468657398
:104250006520636F6D6D616E6473206172652061AE
:10426000637469766520666F7220636F6E66696736
:1042700075726174696F6E3A0A2020247379732015
:1042800053686F772073797374656D202867656E46
:104290006572616C292073657474696E67730A2096
:1042A00020243120202053686F77206D6F746F7247
:1042B00020312073657474696E677320286F7220D3
:1042C0007768617465766572206D6F746F7220799E
:1042D0006F752077616E7420312C322C332C342989
:1042E0000A2020247820202053686F7720582061EE
:1042F0007869732073657474696E677320286F72B0
:1043000020776861746576657220617869732079B9
:104310006F752077616E7420782C792C7A2C612C43
:10432000622C63290A2020246D20202053686F7797
:1043300020616C6C206D6F746F722073657474698A
:104340006E67730A2020247120202053686F772025
:10435000616C6C20617869732073657474696E6731
:10436000730A2020246F20202053686F7720616C0F
:104370006C206F66667365742073657474696E670C
:10438000730A2020242420202053686F7720616C3A
:104390006C2073657474696E67730A20202468202A
:1043A000202053686F7720746869732068656C708B
:1043B0002073637265656E0A0A000A0A0A232323C2
:1043C0002054696E794720434F4E46494755524124
:1043D00054494F4E2048656C70202323230A000A5D
:1043E000466F722064657461696C65642054696EFF
:1043F000794720696E666F207365653A206874742A
:1044000070733A2F2F6769746875622E636F6D2F12
:1044100073796E746865746F732F54696E79472F62
:1044200077696B692F0A466F7220746865206C612A
:1044300074657374206669726D7761726520736547
:10444000653A2068747470733A2F2F6769746875C1
:10445000622E636F6D2F73796E746865746F732F3E
:1044600054696E79470A506C65617365206C6F679B
:1044700020616E792069737375657320617420689B
:104480007474703A2F2F7777772E73796E7468650E
:10449000746F732E636F6D2F666F72756D730A483C
:1044A0006176652066756E0A000A4E6F74653A2063
:1044B00054696E79472067656E6572617465732013
:1044C0006175746F6D617469632073746174757361
:1044D000207265706F727473206279206465666102
:1044E000756C740A546869732063616E206265207C
:1044F00064697361626C656420627920656E7465BD
:1045000072696E67202473763D300A5365652074A6
:1045100068652077696B692062656C6F7720666FCC
:1045200072206D6F72652064657461696C732E0A08
:1045300000546865736520636F6D6D616E647320F0
:10454000617265206163746976652066726F6D20A3
:1045500074686520636F6D6D616E64206C696E6553
:104560003A0A205E782020202020202020202020B1
:10457000202052657365742028636F6E74726F6CAF
:10458000207829202D20736F667477617265207200
:10459000657365740A20203F2020202020202020E1
:1045A00020202020204D616368696E6520706F7344
:1045B0006974696F6E20616E642067636F64652043
:1045C0006D6F64656C2073746174650A202024200B
:1045D00020202020202020202020202053686F77BA
:1045E00020616E642073657420636F6E6669677501
:1045F000726174696F6E2073657474696E67730A93
:1046000020202120202020202020202020202020A9
:1046100046656564686F6C64202D2073746F70202C
:104620006D6F74696F6E20776974686F7574206C34
:104630006F73696E6720706F736974696F6E0A209B
:10464000207E2020202020202020202020202043E9
:1046500079636C65205374617274202D20726573C8
:10466000746172742066726F6D2066656564686F30
:104670006C640A2020682020202020202020202078
:1046800020202053686F7720746869732068656CF8
:10469000702073637265656E0A20202468202020D4
:1046A00020202020202020202053686F7720636F57
:1046B0006E66696775726174696F6E2068656C708B
:1046C0002073637265656E0A2020247465737420FC
:1046D00020202020202020204C6973742073656CDA
:1046E000662D74657374730A202024746573743D99
:1046F0004E2020202020202052756E2073656C668D
:104700002D74657374204E0A202024686F6D653DFA
:10471000312020202020202052756E206120686FDB
:104720006D696E67206379636C650A202024646577
:1047300066613D3120202020202020526573746F57
:10474000726520616C6C2073657474696E67732088
:10475000746F2022666163746F72792220646566CB
:1047600061756C74730A000A0A0A232323205469B2
:104770006E79472048656C70202323230A002200AD
:104780007B2272223A7B226D7367223A22007B726F
:104790003A7B6D73673A22005B6A735D20206A730F
:1047A0006F6E2073657269616C697A6520737479C4
:1047B0006C65253964205B303D72656C6178656499
:1047C0002C313D7374726963745D0A005B6A765DB7
:1047D00020206A736F6E20766572626F73697479D8
:1047E00025313564205B303D73696C656E742C3106
:1047F0003D666F6F7465722C323D6D6573736167D2
:1048000065732C333D636F6E666967732C343D6C42
:10481000696E656E756D2C353D766572626F736578
:104820005D0A005B656A5D2020656E61626C6520D3
:104830006A736F6E206D6F646525313364205B3061
:104840003D746578742C313D4A534F4E5D0A009D8E
:1048500059975990598B59825977596C59605954C5
:104860005946592F59205913590759F358E658D129
:1048700058BD58BA58B758A85893587E586F585FC3
:10488000584D5836581958FC57E357CD57BC57AABE
:10489000579D578B5771576E576B576857655762BF
:1048A000575F575C5759575657535750574D574AAC
:1048B000574757445741573E573B5738573557325C
:1048C000572F572C5729572657235720571D571A0C
:1048D000571757145711570E570B570857055702BC
:1048E00057FF56FC56F956F656F356F056ED56EA73
:1048F00056E756E456E156DE56DB56D856D556D224
:1049000056AB56875667564D5633561956F555D8F9
:1049100055C055AA5590556C554F553D551D5506DA
:1049200055ED54CB54B2549454785460544E543092
:10493000541B54FA53F653F253EE53EA53E653E240
:1049400053DE53DA53D653D253CE53CA53C653C24F
:1049500053BE53A4538A5377535B53495332531175
:10496000530053E052C052A6528C52755242521517
:1049700052F551D351AD5186516A514B51315117B6
:1049800051F250C950B15086505A502450EF4FDD6B
:104990004FCB4FBC4FA94F904F6E4F5C4F4A4F3893
:1049A0004F264F144F024FF04EDE4ECC4EBA4EA85B
:1049B0004E964E844E724E6E4E6A4E664E624E5EFD
:1049C0004E5A4E564E524E4E4E4A4E464E424E3E17
:1049D0004E3A4E364E324E2E4E2A4E264E224E0E17
:1049E0004EF04DD44DA94D844D5F4D5B4D574D5309
:1049F0004D4F4D4B4D474D434D3F4D3B4D374D3347
:104A00004D2F4D2B4D274D134DF74CDB4CBF4CA379
:104A10004C874C6B4C4F4C334C174CFB4BDF4BC310
:104A20004BBF4BBB4BB74BB34BAF4BAB4BA74B93B6
:104A30004B6B4B444B1E4BF14ACB4A9E4A9A4A96CB
:104A40004A924A7F4A5E4A494A4A6F6767696E6777
:104A5000206379636C65206661696C6564005072DF
:104A60006F626520656E64706F696E742069732073
:104A70007374617274696E6720706F696E74005030
:104A8000726F6265206379636C65206661696C652D
:104A90006400323439003234380032343700486F21
:104AA0006D696E67204572726F72202D20486F6DA0
:104AB000696E67207377697463686573206D6973C5
:104AC000636F6E6669677572656400486F6D696EC5
:104AD00067204572726F72202D204E656761746980
:104AE0007665206C61746368206261636B6F6666D3
:104AF00000486F6D696E67204572726F72202D20BD
:104B000054726176656C206D696E2026206D617827
:104B100020617265207468652073616D6500486F5F
:104B20006D696E67204572726F72202D204C617422
:104B300063682076656C6F63697479206973207A85
:104B400065726F00486F6D696E67204572726F7293
:104B5000202D205365617263682076656C6F6369F0
:104B60007479206973207A65726F00486F6D696E81
:104B700067204572726F72202D20426164206F722F
:104B8000206E6F2061786973207370656369666950
:104B9000656400486F6D696E67206379636C65209A
:104BA0006661696C65640032333900323338003233
:104BB000333700323336003233350032333400328B
:104BC000333300536F6674206C696D6974206578A7
:104BD000636565646564202D2043206D6178005312
:104BE0006F6674206C696D697420657863656564AF
:104BF0006564202D2043206D696E00536F6674201C
:104C00006C696D6974206578636565646564202DE1
:104C10002042206D617800536F6674206C696D6965
:104C200074206578636565646564202D2042206D7D
:104C3000696E00536F6674206C696D6974206578C5
:104C4000636565646564202D2041206D61780053A3
:104C50006F6674206C696D6974206578636565643E
:104C60006564202D2041206D696E00536F667420AD
:104C70006C696D6974206578636565646564202D71
:104C8000205A206D617800536F6674206C696D69DD
:104C900074206578636565646564202D205A206DF5
:104CA000696E00536F6674206C696D697420657855
:104CB000636565646564202D2059206D617800531B
:104CC0006F6674206C696D697420657863656564CE
:104CD0006564202D2059206D696E00536F66742025
:104CE0006C696D6974206578636565646564202D01
:104CF0002058206D617800536F6674206C696D696F
:104D000074206578636565646564202D2058206D86
:104D1000696E00536F6674206C696D6974206578E4
:104D200063656564656400323139003231380032C0
:104D30003137003231360032313500323134003211
:104D40003133003231320032313100323130003211
:104D500030390032303800323037003230360054CB
:104D6000726170657A6F696420706C616E6E6572D5
:104D7000206661696C656420746F20636F6E766570
:104D8000726765004C696D69742073776974636834
:104D900020686974202D2053687574646F776E20C5
:104DA0006F63637572726564004D616368696E65F7
:104DB00020697320616C61726D6564202D20436FE2
:104DC0006D6D616E64206E6F742070726F636573B9
:104DD000736564004D6F7665206C6573732074682D
:104DE000616E206D696E696D756D2074696D650009
:104DF0004D6F7665206C657373207468616E206DED
:104E0000696E696D756D206C656E677468004765C5
:104E10006E657269632054696E7947206572726F9E
:104E200072003139390031393800313937003139C0
:104E300036003139350031393400313933003139F8
:104E400032003139310031393000313839003138F0
:104E500038003138370031383600313835003138D4
:104E600034003138330031383200313831003138D4
:104E700030005420776F726420697320696E766108
:104E80006C6964005420776F7264206973206D69C7
:104E90007373696E67005220776F726420697320A4
:104EA000696E76616C6964005220776F7264206964
:104EB00073206D697373696E67005120776F726438
:104EC00020697320696E76616C6964005120776F88
:104ED0007264206973206D697373696E67004C207A
:104EE000776F726420697320696E76616C69640003
:104EF0004C20776F7264206973206D697373696EDB
:104F000067004820776F726420697320696E76614C
:104F10006C6964004820776F7264206973206D6942
:104F20007373696E67004520776F72642069732020
:104F3000696E76616C6964004520776F72642069E0
:104F400073206D697373696E67004420776F7264B4
:104F500020697320696E76616C6964004420776F04
:104F60007264206973206D697373696E67005020E5
:104F7000776F7264206973206E6F74206120766190
:104F80006C696420746F6F6C206E756D6265720061
:104F90005020776F7264206973206E6F7420616E89
:104FA00020696E7465676572005020776F726420A7
:104FB0006973206E65676174697665005020776F4C
:104FC0007264206973207A65726F005020776F7267
:104FD0006420697320696E76616C69640050207783
:104FE0006F7264206973206D697373696E67004125
:104FF00072632073706563696669636174696F6E5B
:10500000206572726F72202D20656E64706F696EFC
:1050100074206973207374617274696E6720706F95
:10502000696E7400417263207370656369666963B9
:105030006174696F6E206572726F72202D207261CB
:105040006469757320617263206F7574206F6620C8
:10505000746F6C6572616E6365004172632073707A
:105060006563696669636174696F6E206572726FEA
:1050700072202D206D697373696E67206F66667389
:1050800065742873290041726320737065636966D3
:1050900069636174696F6E206572726F72202D2072
:1050A0006D697373696E6720617869732865732908
:1050B0000041726320737065636966696361746936
:1050C0006F6E206572726F72005370696E646C65EA
:1050D000206D757374206265207475726E696E67D9
:1050E00020666F72207468697320636F6D6D616EE6
:1050F00064005370696E646C65206D757374206212
:1051000065206F666620666F72207468697320631D
:105110006F6D6D616E64005370696E646C652053D1
:1051200020776F726420697320696E76616C6964A0
:10513000005370696E646C65205320776F72642031
:105140006973206D697373696E67005370696E646B
:105150006C6520737065656420657863656564655A
:1051600064206D6178696D756D005370696E646C53
:10517000652073706565642062656C6F77206D696A
:105180006E696D756D0050726F6772616D6D6564EB
:1051900020706F696E742073616D65206173206388
:1051A000757272656E7420706F696E7400437574E9
:1051B00074657220636F6D70656E736174696F6E74
:1051C0002063616E6E6F7420626520656E61626C33
:1051D0006564005265717565737465642076656CED
:1051E0006F636974792065786365656473206C69A1
:1051F0006D697473004730206F72204731206D75E0
:1052000073742062652061637469766520666F72CD
:105210002047353300526F7461727920617865736D
:105220002063616E6E6F7420626520757365642003
:1052300077697468207468697320636F6D6D616E3F
:105240006400496E76657273652074696D65206DC2
:105250006F64652063616E6E6F7420626520757384
:1052600065642077697468207468697320636F6D62
:105270006D616E64004665656472617465206E6F71
:1052800074207370656369666965640053656C6555
:105290006374656420706C616E6520697320696E4B
:1052A00076616C69640053656C6563746564207035
:1052B0006C616E65206973206D697373696E670038
:1052C000417869732074617267657420706F7369C7
:1052D00074696F6E20697320696E76616C69640011
:1052E000417869732074617267657420706F7369A7
:1052F00074696F6E206973206D697373696E6700DE
:10530000417869732069732064697361626C6564B4
:10531000004178697320697320696E76616C6964F5
:1053200020666F72207468697320636F6D6D616EA3
:105330006400417869732063616E6E6F74206265EA
:105340002070726573656E74004178697320776FA1
:105350007264206D697373696E670047636F64657B
:10536000206D6F64616C2067726F75702076696F55
:105370006C6174696F6E004D20636F646520756E9B
:10538000737570706F727465640047636F64652035
:10539000636F6D6D616E6420756E737570706F7282
:1053A0007465640047656E657269632047636F6466
:1053B0006520696E707574206572726F720031328B
:1053C0003900313238003132370031323600313273
:1053D0003500313234003132330031323200313273
:1053E0003100313230003131390031313800313162
:1053F000370031313600313135004A534F4E207479
:105400007874206669656C64732063616E6E6F7476
:10541000206265206E6573746564004A534F4E20A8
:10542000737472696E6720746F6F206C6F6E6700A3
:105430004A534F4E20696E707574206861732074F2
:105440006F6F206D616E79207061697273004A53CD
:105450004F4E2073796E746178206572726F72009E
:10546000496E7075742076616C75652072616E6727
:1054700065206572726F7200496E70757420657870
:105480006365656473206D6178696D756D20766103
:105490006C756500496E707574206C65737320744B
:1054A00068616E206D696E696D756D2076616C75D1
:1054B0006500496E70757420657863656564732056
:1054C0006D6178206C656E67746800436F6D6D6107
:1054D0006E64206E6F742061636365707465642010
:1054E000617420746869732074696D65005061721D
:1054F000616D657465722063616E6E6F74206265A4
:10550000207265616400506172616D65746572201E
:10551000697320726561642D6F6E6C7900556E73CE
:105520007570706F72746564206E756D626572203F
:105530006F72204A534F4E20747970650042616447
:10554000206E756D62657220666F726D61740049C0
:105550006E76616C6964206F72206D616C666F722B
:105560006D656420636F6D6D616E6400556E72656C
:10557000636F676E697A656420636F6D6D616E64D9
:10558000206F7220636F6E666967206E616D6500C3
:1055900047656E6572696320617373657274696FC4
:1055A0006E206661696C757265004D656D6F72790C
:1055B000206661756C74206465746563746564004D
:1055C000537461636B206F766572666C6F772064CD
:1055D0006574656374656400436F6E74726F6C6CA0
:1055E000657220617373657274696F6E206661699C
:1055F0006C7572650043616E6F6E6963616C206DDE
:10560000616368696E6520617373657274696F6E3A
:10561000206661696C75726500506C616E6E6572B2
:1056200020617373657274696F6E206661696C7551
:105630007265005374657070657220617373657272
:1056400074696F6E206661696C75726500456E6382
:105650006F64657220617373657274696F6E206622
:1056600061696C75726500494F207375622D73799D
:105670007374656D20617373657274696F6E2066F3
:1056800061696C75726500436F6E6669672073753A
:10569000622D73797374656D2061737365727469BB
:1056A0006F6E206661696C75726500494F206D658B
:1056B0006D6F727920616C6C6F636174696F6E20BD
:1056C000617373657274696F6E206661696C75725F
:1056D000650038380038370038360038350038343F
:1056E00000383300383200383100383000373900A4
:1056F0003738003737003736003735003734003752
:105700003300373200373100373000363900363851
:105710000036370036360036350036340036330072
:105720003632003631003630003539003538003534
:105730003700353600353500353400353300353225
:10574000003531003530003439003438003437004A
:10575000343600343500343400343300343200340D
:1057600031003430003339003338003337003336FA
:105770000042616420737461747573207265706F88
:1057800072742073657474696E6700506572736912
:105790007374656E6365206572726F7200466C6F1C
:1057A0006174206973204E414E00466C6F61742015
:1057B000697320696E66696E697465004D6F766500
:1057C0002074696D65206973204E414E004D6F76DF
:1057D000652074696D6520697320696E66696E69FC
:1057E00074650047656E65726963206578636570EE
:1057F00074696F6E207265706F7274004661696CB7
:10580000656420746F2067657420706C616E6E65CE
:1058100072206275666665720053797374656D20D7
:10582000616C61726D202D207368757474696E6788
:1058300020646F776E00496E697469616C697A6182
:1058400074696F6E206661696C757265005265617E
:10585000642D6F6E6C7920616464726573730049A6
:105860006E76616C69642041646472657373004490
:105870006976696465206279207A65726F00466C8A
:105880006F6174696E6720706F696E7420657272E3
:105890006F7200496E7465726E616C2072616E6722
:1058A00065206572726F7200496E7465726E616C0C
:1058B000206572726F720031390031380046756EA2
:1058C0006374696F6E2069732073747562626564B6
:1058D00000456E746572696E6720626F6F74206C2C
:1058E0006F6164657200496E697469616C697A6997
:1058F0006E67004275666665722066756C6C202D59
:1059000020666174616C004275666665722066751A
:105910006C6C0042756666657220656D7074790006
:105920004E6F207375636820646576696365004D0A
:1059300061782066696C652073697A652065786393
:1059400065656465640046696C65206E6F74206FE0
:1059500070656E00456E64206F662066696C650038
:10596000456E64206F66206C696E650048617264E4
:10597000207265736574005465726D696E6174653B
:105980006400436F6D706C657465004E6F6F7000DE
:1059900045616761696E004572726F72004F4B001E
:1059A0005B7031706F665D2070776D207068617319
:1059B00065206F66662020202531352E3366205BFA
:1059C000302E2E315D0A005B70317770685D20707B
:1059D000776D20636377207068617365206869253F
:1059E00031352E3366205B302E2E315D0A005B7020
:1059F0003177706C5D2070776D20636377207068FD
:105A0000617365206C6F2531352E3366205B302E37
:105A10002E315D0A005B70317773685D2070776DA1
:105A2000206363772073706565642068692531356C
:105A30002E30662052504D0A005B703177736C5DDA
:105A40002070776D20636377207370656564206CC8
:105A50006F2531352E30662052504D0A005B703173
:105A60006370685D2070776D206377207068617364
:105A700065206869202531352E3366205B302E2E57
:105A8000315D0A005B703163706C5D2070776D2052
:105A90006377207068617365206C6F202531352E27
:105AA0003366205B302E2E315D0A005B70316373EC
:105AB000685D2070776D2063772073706565642062
:105AC0006869202531352E30662052504D0A005B22
:105AD000703163736C5D2070776D20637720737015
:105AE000656564206C6F202531352E30662052505C
:105AF0004D0A005B70316672715D2070776D2066B3
:105B000072657175656E63792020202531352E30E0
:105B10006620487A0A0053595354454D2052454156
:105B20004459004C6F6164696E6720636F6E6669EB
:105B300067732066726F6D20454550524F4D004986
:105B40006E697469616C697A696E6720636F6E66ED
:105B500069677320746F2053686170656F6B6F3273
:105B6000203530306D6D2070726F66696C65007B1A
:105B7000226572223A7B226662223A25302E3266F4
:105B80002C227374223A25642C226D7367223A22E8
:105B90002573227D7D0A007B65723A7B66623A2519
:105BA000302E32662C73743A25642C6D73673A225A
:105BB0002573227D7D0A005B71765D2020717565FD
:105BC0007565207265706F727420766572626F738E
:105BD000697479253764205B303D6F66662C313DF2
:105BE00073696E676C652C323D747269706C655DAB
:105BF0000A00716F3A25640A0071693A25640A0047
:105C000071723A25640A005B73765D2020737461BB
:105C1000747573207265706F727420766572626F2E
:105C200073697479253664205B303D6F66662C316C
:105C30003D66696C74657265642C323D766572628E
:105C40006F73655D0A005B73695D20207374617416
:105C5000757320696E74657276616C2531342E30EF
:105C600066206D730A004D6F746F7220256320707B
:105C70006F77657220656E61626C65642073746114
:105C800074653A25322E30660A005B257325735DF4
:105C9000206D257320706F776572206D616E61676E
:105CA000656D656E7425313064205B303D646973C9
:105CB00061626C65642C313D616C77617973206F32
:105CC0006E2C323D696E206379636C652C333D77B1
:105CD00068656E206D6F76696E675D0A005B25737F
:105CE00025735D206D257320706F6C617269747906
:105CF00025313864205B303D6E6F726D616C2C31E4
:105D00003D726576657273655D0A005B2573257368
:105D10005D206D2573206D6963726F737465707398
:105D200025313664205B312C322C342C385D0A004E
:105D30005B257325735D206D257320747261766514
:105D40006C20706572207265766F6C7574696F6E09
:105D50002531302E346625730A005B257325735D6B
:105D6000206D2573207374657020616E676C6525E6
:105D700032302E336625730A005B257325735D2050
:105D80006D2573206D617020746F206178697325B3
:105D9000313564205B303D582C313D592C323D5A11
:105DA0002E2E2E5D0A005B6D745D20206D6F746F6A
:105DB000722069646C652074696D656F7574253136
:105DC000342E3266205365630A00D95DD55DD05DFF
:105DD0002064656700206D6D0020696E005B737440
:105DE0005D2020737769746368207479706525314C
:105DF0003864205B303D4E4F2C313D4E435D0A00F0
:105E00005465737420232564206E6F7420666F754B
:105E10006E640A004E312054314D360A4E3220470E
:105E200031370A4E33204732310A4E382046313856
:105E300030300A4E392047310A4E31303020473950
:105E40003220582D32352E313737592D33342E30FC
:105E50003732205A2D312E303030202854454D50C5
:105E60002C2052454D4F5645204C41544552290A4D
:105E70004E33343320582D32352E353935592D33A4
:105E8000342E3334390A4E33343420582D32352EE3
:105E9000373031592D33342E3433360A4E333435BE
:105EA00020582D32352E373931592D33342E353295
:105EB000300A4E33343620582D32352E3836345988
:105EC0002D33342E3630310A4E33343720582D32AC
:105ED000352E393230592D33342E3637390A4E3378
:105EE000343820582D32352E393630592D33342E52
:105EF0003735340A4E33343920582D32352E39385F
:105F000032592D33342E3832360A4E33353020583C
:105F10002D32352E393837592D33342E3839350A4C
:105F20004E33353120582D32352E393736592D33F1
:105F3000342E3936310A4E33353220582D32352E33
:105F4000393438592D33352E3032330A4E33353308
:105F500020582D32352E393033592D33352E3038E7
:105F6000320A4E33353420582D32352E38343159DB
:105F70002D33352E3133380A4E33353520582D32F6
:105F8000352E373633592D33352E3139300A4E33CD
:105F9000353620582D32352E363639592D33352E9B
:105FA0003233390A4E33353720582D32352E3535B8
:105FB00039592D33352E3238340A4E33353820587E
:105FC0002D32352E343333592D33352E3332350AB5
:105FD0004E33353920582D32352E323931592D3343
:105FE000352E3336330A4E33363020582D32352E87
:105FF000313334592D33352E3339370A4E33363158
:1060000020582D32342E393633592D33352E343233
:10601000380A4E33363220582D32342E373737591E
:106020002D33352E3435350A4E33363320582D3244
:10603000342E353737592D33352E3437370A4E3312
:10604000363420582D32342E333637592D33352EF1
:106050003439360A4E33363520582D32342E313409
:1060600034592D33352E3531310A4E3336362058DA
:106070002D32332E393039592D33352E3532320AFF
:106080004E33363720582D32332E363631592D3394
:10609000352E3532390A4E33363820582D32332ECC
:1060A000343033592D33352E3533320A4E333639A9
:1060B00020582D32332E313333592D33352E35338D
:1060C000320A4E33373020582D32322E383533597C
:1060D0002D33352E3532370A2F4E323531382047A1
:1060E0003058302E333237592D33332E3532315A22
:1060F0002D312E3030300A4E32353139204D33308B
:10610000004E31204732300A4E3520473430204788
:1061100031370A4E3130205431204D30360A284E66
:106120003135204739302047302058302059302031
:106130005A30290A4E3230205335303030204D301D
:1061400033200A4E32352058302E30363420593024
:106150002E333236205A300A4E3430204730312028
:106160004631362E300A4E35302058302E303634F7
:106170002059302E3332360A4E35352058302E30E5
:1061800036302059302E3239330A4E3630205830CE
:106190002E3037372059302E3236370A4E363520DA
:1061A00058302E3131312059302E3235370A4E37A2
:1061B000302058302E3134392059302E3235320AC1
:1061C0004E37352058302E3138382059302E323560
:1061D000350A4E38302058302E3232372059302E82
:1061E0003236380A4E38352058302E32353720595D
:1061F000302E3237310A4E39302058302E33333575
:106200002059302E3236350A4E39352058302E344A
:1062100031322059302E3237310A4E313030205849
:10622000302E3437342059302E3238370A4E313040
:10623000352058302E3439312059302E3238390A31
:106240004E3131302058302E3531372059302E32F2
:1062500037330A4E3131352058302E3534342059F9
:10626000302E3236330A4E3132302058302E353807
:10627000302059302E3236310A4E313235205830E6
:106280002E3539352059302E3236330A4E313330DF
:106290002058302E3632312059302E3237340A4EC3
:1062A0003133352058302E3635392059302E3330A1
:1062B000360A4E3134302058302E3637332059309C
:1062C0002E3333350A4E3134352058302E36373997
:1062D0002059302E3336310A4E3135302058302E89
:1062E0003637382059302E3338390A4E313535207B
:1062F00058302E3637302059302E3432300A4E3155
:1063000036302058302E3637302059302E3434363F
:106310000A4E3136352058302E3638302059302E3E
:106320003437340A4E3137302058302E373034204D
:1063300059302E3439370A4E3137352058302E3700
:1063400033322059302E3531350A4E31383020580D
:10635000302E3739342059302E3533350A4E313806
:10636000352058302E3837322059302E3536370AFE
:106370004E3139302058302E3935302059302E36B4
:1063800030340A4E3139352058312E3033312059CE
:10639000302E3634370A4E3230302058312E3134D8
:1063A000392059302E3732320A4E323035205831AA
:1063B0002E3330382059302E3835340A4E323130B1
:1063C0002058312E3433302059302E3938340A4E8B
:1063D0003231352058312E3434372059302E393867
:1063E000360A4E3232302058312E3632382059306B
:1063F0002E3832320A4E3232352058312E3733326F
:106400002059302E3731340A4E3233302058322E54
:106410003030392059302E3338310A4E323335205E
:1064200058322E3131362059302E3236360A4E321D
:1064300034302058322E3232382059302E31353710
:106440000A4E3234352058322E3238302059302E10
:106450003132330A4E3235302058322E3333322027
:1064600059302E3039340A4E3235352058322E34D8
:1064700032332059302E3037300A4E3236302058E1
:10648000322E3438392059302E3036350A4E3236D5
:10649000352058322E3535372059302E3036360AD1
:1064A0004E3237302058322E3632372059302E3087
:1064B00038340A4E3237352058322E363933205987
:1064C000302E3130390A4E3238302058322E3733A0
:1064D000302059302E3133330A4E3238352058327D
:1064E0002E3830352059302E3139300A4E3239307D
:1064F0002058322E3832392059302E3231360A4E59
:106500003239352058322E3838302059302E323931
:10651000310A4E3330302058322E3838342059303A
:106520002E3330300A4E3330352058322E38393839
:106530002059302E3333320A4E3331302058322E28
:106540003930352059302E3336370A4E3331352025
:1065500058322E3931302059302E3430370A4E33EC
:1065600032302058322E3930382059302E343436DB
:106570000A4E3332352058322E3930312059302EE0
:106580003439350A4E3333302058322E38393720DB
:1065900059302E3439350A4E3333352058322E389F
:1065A00039302059302E3532340A4E3334302058A9
:1065B000322E3834322059302E3630340A4E3334AD
:1065C000352058322E3831342059302E3636350A9F
:1065D0004E3335302058322E3739342059302E374B
:1065E00035300A4E3335352058322E37393120595F
:1065F000302E3833380A4E3336302058322E383168
:10660000392059302E3937360A4E33363520583234
:106610002E3833372059312E3034340A4E33373048
:106620002058322E3836322059312E3131320A4E2E
:106630003337352058322E3837372059312E313400
:10664000350A4E3338302058322E39313220593104
:106650002E3231370A4E3338352058322E39313701
:106660002059312E3232360A4E3339302058322EEC
:106670003935312059312E3238310A4E33393520EF
:1066800058322E3937302059312E3239350A4E34AE
:1066900030302058322E3939362059312E323935A2
:1066A0000A4E3430352058332E3031332059312EB4
:1066B0003237350A4E3431302058332E30323420C0
:1066C00059312E3235340A4E3431352058332E307C
:1066D00037302059312E3135310A4E34323020587E
:1066E000332E3037372059312E3133340A4E34327D
:1066F000352058332E3132352059312E3033390A76
:106700004E3433302058332E3133382059312E3027
:1067100031390A4E3433352058332E323035205932
:10672000302E3930380A4E3434302058332E323837
:10673000322059302E3739370A4E34343520583309
:106740002E3336312059302E3639310A4E34353019
:106750002058332E3432362059302E3539320A4EF5
:106760003435352058332E3435362059302E3534D3
:10677000330A4E3436302058332E343739205930CE
:106780002E3439330A4E3436352058332E343934CA
:106790002059302E3437320A4E3437302058332EB9
:1067A0003530352059302E3434360A4E34373520C2
:1067B00058332E3531382059302E3431370A4E3483
:1067C00038302058332E3533302059302E3339317C
:1067D0000A4E3438352058332E3536342059302E71
:1067E0003330300A4E3439302058332E3537372085
:1067F00059302E3235330A4E3439352058332E3540
:1068000036382059302E3231320A4E353030205849
:10681000332E3534342059302E3137360A4E353048
:10682000352058332E3534312059302E3134360A44
:106830004E3531302058332E3535332059302E31F6
:1068400031390A4E3531352058332E3537362059F7
:10685000302E3130360A4E3532302058332E35390D
:10686000372059302E3130320A4E353235205833E8
:106870002E3631382059302E3130390A4E353330EA
:106880002058332E3633392059302E3132390A4EC2
:106890003533352058332E3635302059302E3135AA
:1068A000390A4E3534302058332E3636332059309D
:1068B0002E3137380A4E3534352058332E36373896
:1068C0002059302E3139320A4E3535302058332E8A
:1068D0003639392059302E3139370A4E3535352081
:1068E00058332E3732332059302E3139360A4E354F
:1068F00036302058332E3736342059302E31373940
:106900000A4E3536352058332E3830352059302E42
:106910003136350A4E3537302058332E383834204A
:1069200059302E3135390A4E3537352058332E3906
:1069300034392059302E3136350A4E35383020580A
:10694000332E3936362059302E3137350A4E353808
:10695000352058332E3937382059302E3139340A02
:106960004E3539302058332E3937382059302E32B1
:1069700032330A4E3539352058332E3936302059C6
:10698000302E3234350A4E3630302058332E3833DC
:10699000342059302E3331310A4E363035205833B9
:1069A0002E3736322059302E3334350A4E363130B8
:1069B0002058332E3732362059302E3338390A4E8C
:1069C0003631352058332E3730332059302E343578
:1069D000380A4E3632302058332E3638322059306D
:1069E0002E3533300A4E3632352058332E3637396D
:1069F0002059302E3533340A4E3633302058332E5A
:106A00003632362059302E3638310A4E363335205C
:106A100058332E3536382059302E3832380A4E3613
:106A200034302058332E3434342059312E3038301D
:106A30000A4E3634352058332E3430352059312E15
:106A40003136370A4E3635302058332E3430342024
:106A500059312E3136370A4E3635352058332E33DC
:106A600038372059312E3230380A4E3636302058D9
:106A7000332E3338342059312E3230380A4E3636E0
:106A8000352058332E3336352059312E3236350ADB
:106A90004E3637302058332E3335352059312E328B
:106AA00038350A4E3637352058332E33343820598E
:106AB000312E3330380A4E3638302058332E3333A7
:106AC000332059312E3335300A4E3638352058337D
:106AD0002E3332312059312E3339310A4E36393086
:106AE0002058332E3331312059312E3432380A4E6A
:106AF0003639352058332E3333392059312E34323C
:106B0000330A4E3730302058332E34343020593148
:106B10002E3430360A4E3730352058332E3531304A
:106B20002059312E3430380A4E3731302058332E28
:106B30003538352059312E3432310A4E373135202F
:106B400058332E3631312059312E3433390A4E37ED
:106B500032302058332E3631312059312E343431F1
:106B60000A4E3732352058332E3631352059312EE2
:106B70003434310A4E3733302058332E36333620F2
:106B800059312E3438380A4E3733352058332E36A3
:106B900033342059312E3531370A4E3734302058AE
:106BA000332E3632322059312E3534330A4E3734B3
:106BB000352058332E3630352059312E3536330AAC
:106BC0004E3735302058332E3537362059312E3553
:106BD00037350A4E3735352058332E353434205961
:106BE000312E3538310A4E3736302058332E34376F
:106BF000392059312E3539320A4E3736352058333F
:106C00002E3435312059312E3539380A4E37373048
:106C10002058332E3338372059312E3632360A4E2B
:106C20003737352058332E3339302059312E36330B
:106C3000360A4E3738302058332E3533322059310A
:106C40002E3630320A4E3738352058332E36303112
:106C50002059312E3539370A4E3739302058332EE6
:106C60003636382059312E3539380A4E37393520E5
:106C700058332E3738322059312E3631320A4E38B9
:106C800030302058332E3739342059312E363138B0
:106C90000A4E3830352058332E3836382059312EA8
:106CA0003633360A4E3831302058332E39313820B9
:106CB00059312E3635350A4E3831352058332E3974
:106CC00034352059312E3636370A4E383230205876
:106CD000332E3936342059312E3638350A4E383273
:106CE000352058332E3936372059312E3638350A6B
:106CF0004E3833302058332E3937342059312E3620
:106D000039390A4E3833352058332E393834205922
:106D1000312E3732350A4E3834302058332E393838
:106D2000342059312E3735380A4E3834352058330F
:106D30002E3937302059312E3739300A4E38353018
:106D40002058332E3934352059312E3831370A4EF8
:106D50003835352058332E3931382059312E3832D4
:106D6000360A4E3836302058332E383931205931D2
:106D70002E3832370A4E3836352058332E383432D2
:106D80002059312E3830390A4E3837302058332EBA
:106D90003739382059312E3738340A4E38373520B4
:106DA00058332E3734362059312E3737320A4E3881
:106DB00038302058332E3639382059312E37363472
:106DC0000A4E3838352058332E3633352059312E77
:106DD0003736360A4E3839302058332E3535332081
:106DE00059312E3738350A4E3839352058332E343C
:106DF00037382059312E3832300A4E393030205849
:106E0000332E3430392059312E3836340A4E393049
:106E1000352058332E3334352059312E3931380A44
:106E20004E3931302058332E3236342059322E30FC
:106E300032330A4E3931352058332E323438205906
:106E4000322E3035310A4E3932302058332E32341A
:106E5000302059322E3038310A4E393235205833ED
:106E60002E3331362059322E3038360A4E393330EF
:106E70002058332E3339302059322E3130340A4ED7
:106E80003933352058332E3431342059322E3132B3
:106E9000310A4E3934302058332E343331205932B0
:106EA0002E3135330A4E3934352058332E343333AE
:106EB0002059322E3138300A4E3935302058332E91
:106EC0003432372059322E3230350A4E393535209A
:106ED00058332E3431332059322E3232340A4E395F
:106EE00036302058332E3339322059322E32343254
:106EF0000A4E3936352058332E3333352059322E49
:106F00003234340A4E3937302058332E3237382055
:106F100059322E3233360A4E3937352058332E3215
:106F200035362059322E3234320A4E393830205814
:106F3000332E3233392059322E3235310A4E393818
:106F4000352058332E3231312059322E3238300A22
:106F50004E3939302058332E3137342059322E33C0
:106F600035360A4E3939352058332E3135392059C6
:106F7000322E3339370A4E313030302058332E31EB
:106F800035302059322E3433380A4E3130303520E6
:106F900058332E3134302059322E3438310A4E31A4
:106FA0003031302058332E3133322059322E3531A2
:106FB000300A4E313031352058332E313138205996
:106FC000322E3534330A4E313032302058332E30A1
:106FD00039392059322E3537360A4E313032352084
:106FE00058332E3035312059322E3633310A4E3156
:106FF0003033302058332E3030332059322E36364D
:10700000360A4E313033352058322E393537205933
:10701000322E3638350A4E313034302058322E393F
:1070200030372059322E3639390A4E313034352036
:1070300058322E3836302059322E3731310A4E31FF
:107040003035302058322E3831392059322E3732EF
:10705000370A4E313035352058322E3736382059E0
:10706000322E3734350A4E313036302058322E37F2
:1070700031362059322E3735370A4E3130363520E9
:1070800058322E3637352059322E3735370A4E31A1
:107090003037302058322E3537392059322E373399
:1070A000310A4E313037352058322E35373020599D
:1070B000322E3732330A4E313038302058322E35A6
:1070C00035392059322E3732300A4E31303835209A
:1070D00058322E3533302059322E3730310A4E3166
:1070E0003039302058322E3530312059322E363951
:1070F000330A4E313039352058322E343731205949
:10710000322E3638330A4E313130302058322E3458
:1071100034332059322E3636380A4E31313035204C
:1071200058322E3339362059322E3633340A4E3106
:107130003131302058322E3335342059322E353902
:10714000310A4E313131352058322E333532205903
:10715000322E3539310A4E313132302058322E3309
:1071600032352059322E3534330A4E313132352002
:1071700058322E3331352059322E3532310A4E31C4
:107180003133302058322E3330372059322E3439B3
:10719000380A4E313133352058322E3239362059A3
:1071A000322E3436340A4E313134302058322E32B9
:1071B00039332059322E3432370A4E3131343520AA
:1071C00058322E3239352059322E3336360A4E3166
:1071D0003135302058322E3332312059322E33306F
:1071E000330A4E313135352058322E333538205957
:1071F000322E3234370A4E313136302058322E3466
:1072000031392059322E3230330A4E313136352061
:1072100058322E3431392059322E3137390A4E3115
:107220003137302058322E3430352059322E313516
:10723000380A4E313137352058322E333632205904
:10724000322E3132330A4E313138302058322E331B
:1072500035342059322E3130340A4E313138352010
:1072600058322E3335342059322E3039310A4E31CE
:107270003139302058322E3338302059322E3036C2
:10728000350A4E313139352058322E3431302059BB
:10729000322E3035310A4E313230302058322E34D1
:1072A00031302059322E3034370A4E3132303520C9
:1072B00058322E3430352059322E3032380A4E3181
:1072C0003231302058322E3430382059322E30317D
:1072D000300A4E313231352058322E343136205971
:1072E000312E3939350A4E313232302058322E346F
:1072F00033332059312E3938320A4E31323235206B
:1073000058322E3433382059312E3936330A4E3123
:107310003233302058322E3434372059312E39341C
:10732000380A4E313233352058322E343631205916
:10733000312E3933380A4E313234302058322E341F
:1073400038302059312E3933310A4E31323435201C
:1073500058322E3437382059312E3839390A4E31C7
:107360003235302058322E3438372059312E3837C4
:10737000350A4E313235352058322E3530342059C9
:10738000312E3835340A4E313236302058322E35CF
:1073900032372059312E3834380A4E3132363520C2
:1073A00058322E3534392059312E3834390A4E317D
:1073B0003237302058322E3537372059312E383673
:1073C000310A4E313237352058322E36303420597A
:1073D000312E3836360A4E313238302058322E3679
:1073E00033312059312E3835340A4E313238352078
:1073F00058322E3634302059312E3832370A4E3139
:107400003239302058322E3634302059312E373927
:10741000320A4E313239352058322E36323920591F
:10742000312E3735390A4E313330302058322E362E
:1074300031322059312E3732370A4E313330352030
:1074400058322E3537362059312E3639340A4E31DE
:107450003331302058322E3533362059312E3636DE
:10746000320A4E313331352058322E3437302059DC
:10747000312E3631360A4E313332302058322E33E7
:1074800034352059312E3535310A4E3133323520DD
:1074900058322E3330372059312E3532310A4E31A1
:1074A0003333302058322E3236302059312E343892
:1074B000320A4E313333352058322E32343320598C
:1074C000312E3437370A4E313334302058322E3291
:1074D00032382059312E3436390A4E313334352082
:1074E00058322E3232322059312E3434380A4E314D
:1074F0003335302058322E3232382059312E343242
:10750000350A4E313335352058322E323534205934
:10751000312E3430350A4E313336302058322E3247
:1075200036382059312E3337330A4E313336352031
:1075300058322E3237392059312E3334320A4E31F7
:107540003337302058322E3330382059312E3238EC
:10755000370A4E313337352058322E3334302059E4
:10756000312E3235340A4E313338302058322E34F1
:1075700030372059312E3230310A4E3133383520F0
:1075800058322E3434312059312E3135360A4E31AD
:107590003339302058322E3435342059312E31339E
:1075A000310A4E313339352058322E343630205995
:1075B000312E3130360A4E313430302058322E34AC
:1075C00036342059312E3130320A4E3134303520A4
:1075D00058322E3437312059312E3033360A4E315D
:1075E0003431302058322E3436362059302E393747
:1075F000310A4E313431352058322E34353120594C
:10760000302E3839370A4E313432302058322E3449
:1076100031352059302E3739310A4E313432352048
:1076200058322E3430332059302E3736370A4E3107
:107630003433302058322E3338382059302E3736F4
:10764000350A4E313433352058322E3330362059F6
:10765000302E3834310A4E313434302058322E3204
:1076600032322059302E3931310A4E3134343520FE
:1076700058322E3131342059302E3939350A4E31B5
:107680003435302058322E3030322059312E3037B8
:10769000360A4E313435352058312E39303520599F
:1076A000312E3133390A4E313436302058312E37AD
:1076B00035342059312E3232330A4E3134363520AA
:1076C00058312E3633372059312E3237380A4E3161
:1076D0003437302058312E3538322059312E33305E
:1076E000310A4E313437352058312E35353820594E
:1076F000312E3331350A4E313438302058312E3462
:1077000036302059312E3335320A4E313438352057
:1077100058312E3339392059312E3336300A4E3113
:107720003439302058312E3333382059312E333507
:10773000340A4E313439352058312E3238372059F9
:10774000312E3332390A4E313530302058312E3215
:1077500034382059312E3239340A4E313530352003
:1077600058312E3231372059312E3235340A4E31CC
:107770003531302058312E3231342059312E3235C6
:10778000320A4E313531352058312E3137322059B9
:10779000312E3139350A4E313532302058312E31C3
:1077A00032382059312E3133390A4E3135323520B5
:1077B00058312E3131302059312E3131370A4E3186
:1077C0003533302058302E3935382059302E393461
:1077D000310A4E313533352058302E383931205961
:1077E000302E3837330A4E313534302058302E3869
:1077F00032352059302E3830380A4E313534352064
:1078000058302E3735352059302E3734370A4E311F
:107810003535302058302E3631392059302E363318
:10782000330A4E313535352058302E34373720590C
:10783000302E3532360A4E313536302058302E341F
:1078400037372059302E3532340A4E31353635200F
:1078500058302E3431312059302E3437360A4E31DB
:107860003537302058302E3333312059302E3435CF
:10787000340A4E313537352058302E3237382059BA
:10788000302E3432370A4E313538302058302E32CF
:1078900033312059302E3339370A4E3135383520BF
:1078A00058302E3138332059302E3337390A4E3183
:1078B0003539302058302E3133352059302E33367B
:1078C000350A4E313539352058302E30373620596B
:1078D000302E3334310A4E313630352047303020A7
:1078E0004633302E300A4E31363130204D3035207F
:1078F0000A4E313631352047393020583020593042
:10790000205A300A4E31363135204D33300A284561
:107910006E64206F6620434E432050726F67726121
:107920006D2900284D53472A2A2A2A204D6963725F
:107930006F737465702054657374205B76315D20BD
:107940002A2A2A2A290A473030204731372047324D
:1079500031204734302047343920473830204739E8
:10796000300A6730783079307A300A7B22316D699D
:10797000223A317D0A7B22326D69223A317D0A7BBF
:1079800022336D69223A317D0A7B22346D69223AB5
:10799000317D0A6730207831300A7B22316D6922CF
:1079A0003A327D0A78300A7B22316D69223A347D81
:1079B0000A7831300A7B22316D69223A387D0A78A3
:1079C000300A6730207931300A7B22326D69223AE1
:1079D000327D0A79300A7B22326D69223A347D0A7F
:1079E0007931300A7B22326D69223A387D0A79304A
:1079F0000A6730207A31300A7B22336D69223A32AD
:107A00007D0A7A300A7B22336D69223A347D0A7A04
:107A100031300A7B22336D69223A387D0A7A300A86
:107A20006730206131300A7B22346D69223A327D21
:107A30000A61300A7B22346D69223A347D0A613151
:107A4000300A7B22346D69223A387D0A61300A6D32
:107A50003200284D53472A2A2A2A20436F6F726426
:107A6000696E617465206F666673657473207465F2
:107A70007374205B76315D202A2A2A2A290A67300E
:107A800030673137673231673430673439673830BF
:107A90006739300A6735340A673932783079307A95
:107AA000300A663630300A284D53472A2A2A2A20BF
:107AB0007465737420473932206F6666736574731A
:107AC0002A2A2A2A290A286D73675374657020317F
:107AD0003A204D6F76652066726F6D20302C302015
:107AE000746F2033302C30206D6D20696E20706FE4
:107AF0007369746976652058206469726563746976
:107B00006F6E290A286D73675374657020323A20AE
:107B10005265736574206F726967696E20746F2097
:107B2000302E30207573696E6720473932290A2854
:107B30006D73675374657020333A204D6F766520FE
:107B4000746F2032302C302E2053686F756C642097
:107B50006D6F7665203230206D6D20696E20706FFC
:107B60007369746976652058206469726563746905
:107B70006F6E20616E64207374617475732072651A
:107B8000706F72742073686F756C642073746172A7
:107B9000742066726F6D20302C30290A286D73674F
:107BA0005374657020343A204D6F766520746F20D1
:107BB000302E3020202053686F756C64206D6F76F6
:107BC00065203230206D6D20696E206E65676174AE
:107BD000697665205820646972656374696F6E20E8
:107BE000616E6420737461747573207265706F7256
:107BF000742073686F756C6420737461727420668E
:107C0000726F6D2032302C30290A67317833300A98
:107C100067393278300A67317832300A6731783024
:107C200079300A2473720A67393278300A673470FF
:107C3000302E350A284D53472A2A2A2A2074657384
:107C40007420473535206F6666736574732A2A2A57
:107C50002A290A286D73675374657020313A2053BE
:107C6000657420436F6F7264696E61746520737907
:107C70007374656D2032205B6735355D20746F202D
:107C80006F6666736574206F662035302C35302939
:107C90000A286D73675374657020323A2053656CFF
:107CA0006563742047353520636F6F7264696E6158
:107CB00074652073797374656D290A286D73675331
:107CC00074657020333A204D6F766520746F2030D4
:107CD0002C302E20486561642073686F756C6420B9
:107CE0006D6F766520646961676F6E616C6C792079
:107CF000696E202B5820616E64202B5920616E64C0
:107D000020737461747573207265706F7274207360
:107D1000686F756C642073746172742066726F6D25
:107D200020302C30290A6731304C327032783530AF
:107D30007935300A6735350A6730783079300A6727
:107D40003470302E350A284D53472A2A2A2A2074A7
:107D500065737420473533206162736F6C75746589
:107D6000206F7665727269646573202A2A2A2A292F
:107D70000A286D73675374657020313A2052756E0E
:107D800020612073717561726520696E20473535F9
:107D90002073797374656D290A286D736753746550
:107DA0007020323A2052756E2061207371756172B5
:107DB0006520772F473533206F7665727269646569
:107DC000290A6730783079300A6730783230793074
:107DD0000A67307832307932300A67307830793259
:107DE000300A6730783079300A673470302E350ABF
:107DF0006735336730783079300A673533673078E4
:107E0000323079300A673533673078323079323042
:107E10000A673533673078307932300A673533672F
:107E200030783079300A6730783079300A673470CA
:107E3000302E350A284D53472A2A2A2A2074657382
:107E4000742052657475726E20746F20686F6D6552
:107E5000202A2A2A2A290A286D73675374657020FC
:107E6000313A2052657475726E20746F20686F6DA0
:107E700065207573696E6720473238290A286D734B
:107E8000675374657020323A2052657365742074AC
:107E90006F2047353420636F6F7264207379737479
:107EA000656D290A6732380A6735340A6D33300048
:107EB000284D53472A2A2A2A205465737420616367
:107EC000637572616379206F6620736C6F77206DC4
:107ED0006F766573205B76315D202A2A2A2A290A6B
:107EE0006735350A6730783079300A673470302E5C
:107EF000350A673470302E350A6731783130663292
:107F0000320A6735340A6730783079300A6D333099
:107F100000284D53472A2A2A2A2054657374207654
:107F20006572792073686F7274206D6F7665732047
:107F30005B76315D202A2A2A2A290A67307830792F
:107F4000300A673470302E350A673178302E31664A
:107F5000313030300A78300A78302E310A78300AE1
:107F600078302E310A78300A78302E310A78300A8B
:107F700078302E310A78300A78302E310A78300A7B
:107F800078302E310A78300A78302E310A78300A6B
:107F900078302E310A78300A78302E310A78300A5B
:107FA00078302E310A78300A78302E310A78300A4B
:107FB00078302E310A78300A78302E310A78300A3B
:107FC00078302E310A673470302E350A78300A78CE
:107FD000302E30310A78300A78302E30310A78303D
:107FE0000A78302E30310A78300A78302E30310A53
:107FF00078300A78302E30310A78300A78302E30D6
:10800000310A78300A78302E30310A78300A7830E8
:108010002E30310A78300A78302E30310A78300A22
:1080200078302E30310A78300A78302E30310A78A4
:10803000300A78302E30310A78300A78302E3031DC
:108040000A78300A78302E30310A6730783079304B
:108050000A6D3200284D53472A2A2A2A20526F746B
:108060006172792041786973204D6F74696F6E2059
:1080700054657374205B76315D202A2A2A2A290AE6
:10808000673030673137673231673430673439678A
:1080900038306739300A6730783079307A3061307B
:1080A000623063300A6735350A6730783079300AD4
:1080B0006633363030300A6730613336300A623327
:1080C00036300A633336300A61300A62300A633070
:1080D0000A673161313434300A62313434300A6332
:1080E000313434300A61300A62300A63300A673151
:1080F000613134343062373230633336300A7830AD
:1081000079307A306130623063300A6731783630E6
:10811000613134343062373230633336300A78308C
:1081200079307A306130623063300A6731783630C6
:108130007935306131343430623732306333363040
:108140000A783079307A306130623063300A6731D2
:1081500078363079353078323561313434306237C1
:108160003230633336300A783079307A30613062B9
:108170003063300A6735340A6730783079300A6DF9
:10818000333000284D53472A2A2A2A20496E766523
:108190007273652054696D65204D6F74696F6E2030
:1081A00054657374205B76315D202A2A2A2A290AB5
:1081B0006730306731376732316734306734396759
:1081C00038306739300A6735350A673078307930AA
:1081D0000A6739330A66302E30310A673178313018
:1081E0000A7931300A7A31300A6131300A78300A3E
:1081F00079300A7A300A61300A6731783130793162
:10820000307A2D31306131300A6730783079307A08
:108210003061300A66302E310A6732783130792D7C
:1082200031307A2D32306931300A67307830793028
:108230007A300A6733783130792D31307A2D323007
:108240006931300A6730783079307A300A673278AD
:10825000323079307A2D32306931300A67307830F7
:1082600079307A300A673378323079306931300AC0
:108270006730783079307A300A6732783079307AFE
:108280002D33306931300A6733783079307A30698C
:1082900031300A6730783079307A300A6732783096
:1082A00079306932302028435720333630206465D6
:1082B0006772656573290A673378307930693230BF
:1082C0002028434357203336302064656772656544
:1082D00073290A6739340A6735340A673078307988
:1082E000300A6D3330007B226763223A22673030D8
:1082F0006731376732316734306734396738306710
:108300003930227D0A7B226763223A226735352283
:108310007D0A7B226763223A2267307830793022E7
:108320007D0A7B226763223A2266353030227D0A3D
:108330007B226763223A22284D534773717561721D
:10834000657329227D0A7B226763223A226730788F
:108350003230227D0A7B226763223A227932302230
:108360007D0A7B226763223A227830227D0A7B22B3
:108370006763223A227930227D0A7B226763223AA0
:10838000226731783130227D0A7B226763223A22CC
:10839000793130227D0A7B226763223A22783022AB
:1083A0007D0A7B226763223A227930227D0A7B2272
:1083B0006763223A22284D5347636972636C657381
:1083C00029227D0A7B226763223A22673278313084
:1083D000792D3130693130227D0A7B226763223A60
:1083E00022673078307930227D0A7B226763223A17
:1083F000226733783130792D3130693130227D0A6E
:108400007B226763223A22673078307930227D0AF6
:108410007B226763223A22673278323079306931C1
:1084200030227D0A7B226763223A226730783079D6
:1084300030227D0A7B226763223A2267337832300A
:108440007930693130227D0A7B226763223A2267C4
:108450003078307930227D0A7B226763223A2267A6
:108460003278307930693130227D0A7B226763228D
:108470003A22673378307930693130227D0A7B22A5
:108480006763223A22673534227D0A7B22676322A2
:108490003A22673078307930227D0A7B2267632266
:1084A0003A226D3330227D00284D53472A2A2A2A4A
:1084B000204D636F6465732074657374205B76313F
:1084C0005D202A2A2A2A290A6735350A673078303A
:1084D00079300A6D330A673470310A6D350A6734B2
:1084E00070310A6D340A673470310A6D350A6734A9
:1084F00070310A6D370A673470310A6D390A673492
:1085000070310A6D380A673470310A6D390A663580
:1085100030300A67307832300A7932300A6D330AE7
:1085200078300A6D340A79300A6D350A673178314E
:10853000300A6D370A7931300A6D380A78300A6DA1
:10854000390A79300A6732783130792D3130693122
:10855000300A6D330A6730783079300A6D340A6733
:1085600033783130792D31306931300A6D350A6711
:1085700030783079300A6D370A67327832307930A6
:108580006931300A6D380A6730783079300A6D39D0
:108590000A673378323079306931300A67307830A1
:1085A00079300A6732783079306931300A67337848
:1085B0003079306931300A6735340A67307830797C
:1085C000300A6D333000284D53472A2A2A2A204684
:1085D000656564686F6C642054657374205B7631E4
:1085E0005D202A2A2A2A290A284D53472A2A2A2A7C
:1085F000204D616E75616C6C7920656E74657220BA
:108600002120616E64207E20647572696E67206D22
:108610006F76656D656E7420746F20746573742059
:108620002A2A2A2A290A6735350A673078307930AC
:108630000A673470330A6730306731376732316721
:1086400034306734396738306739300A663630304D
:108650000A6730783130307637362E3736350A783B
:108660003079300A6735340A6730783079300A6DEE
:10867000333000284D53472A2A2A2A204477656C34
:108680006C2054657374205B76315D202A2A2A2A77
:10869000290A6730306731376732316739300A6706
:1086A00035350A6730783079300A663530300A67F8
:1086B000307831300A673470310A67307832300AE6
:1086C000673470310A67307831300A673470310AA4
:1086D00067307830300A673470310A79350A673587
:1086E000340A6730783079300A6D330A6734703174
:1086F0000A67307831307931300A6D350A67347065
:10870000310A67307832307932300A6D340A673492
:1087100070310A67307833307933300A6D380A6740
:108720003470310A67307834307934300A6D390A60
:10873000673470310A67307835307935300A673000
:10874000783079300A6D3330004E31206730306731
:1087500031376732316734306734396738306739D9
:10876000300A4E3130206730783079300A4E32305E
:1087700020663530300A4E33302067327831307918
:108780002D31306931302028435720323730206472
:10879000656772656573290A4E343020673078301A
:1087A00079300A4E3530206733783130792D3130C9
:1087B000693130202843435720393020646567727F
:1087C000656573290A4E3630206730783079300A73
:1087D0004E38302067327832307930693130202895
:1087E0004357203138302064656772656573290A04
:1087F0004E3730206730783079300A4E3830206775
:108800003378323079306931302028434357203172
:1088100038302064656772656573290A4E393020E7
:108820006730783079300A4E39392046313230306D
:108830000A4E31303020673278307930693230205A
:108840002843572033363020646567726565732985
:108850000A4E313130206732783079306932302039
:108860002843572033363020616761696E290A4EEC
:10887000313230206637303020284368616E6765BA
:1088800020666565642072617465207768696C652F
:1088900020696E204732206D6F74696F6E206D6F96
:1088A0006465290A4E313330206732783079306977
:1088B00032302028435720333630203372642074FE
:1088C000696D65290A4E313430206732783079304D
:1088D00069323020284357203336302034746820E2
:1088E00074696D65290A4E31353020663530300A9D
:1088F0004E313630206733783079307A343069320F
:108900003020284343572033363020646567726532
:1089100065732077697468206C696E656172207474
:10892000726176656C290A4E3137302067337830B2
:1089300079307A306932302028434357203336303B
:1089400020616761696E290A4E3138302066373000
:108950003020286D73672A2A2A2A4368616E67656A
:1089600020666565642072617465207768696C654E
:1089700020696E204733206D6F74696F6E206D6FB4
:1089800064652A2A2A2A290A4E3139302067337829
:108990003079306932302028434357203336302035
:1089A0003372642074696D65290A4E323030206755
:1089B00033783079306932302028434357203336BA
:1089C00030203474682074696D65290A4E32313064
:1089D00020286D73672A2A2A2A4731382045766174
:1089E0006C20746573742A2A2A2A290A4E3232307E
:1089F000204731205833302E373037205A35302E2B
:108A000037323720463530300A4E32333020473146
:108A10003820473032205836372E373338205A32F4
:108A2000332E3631372052323520463235300A4E19
:108A3000323430206738300A4E3235302067307893
:108A40003079307A300A4E323630206D333000289B
:108A50004D53472A2A2A2A20537175617265732063
:108A60004D6F74696F6E2054657374205B76315D51
:108A7000202A2A2A2A290A6730306731376732319B
:108A80006734306734396738306739300A6730788F
:108A90003079300A67307832302028747261766518
:108AA00072736520612032306D6D20737175617253
:108AB0006520696E205820616E642059290A793238
:108AC000300A78300A79300A6731783130663530CB
:108AD0003020286472617720612031306D6D207301
:108AE000717561726520696E205820616E6420592D
:108AF0002061742046353030290A7931300A7830C7
:108B00000A79300A67307A323020287472617665CB
:108B100072736520612032306D6D207371756172E2
:108B20006520696E205820616E64205A290A7832C7
:108B3000300A7A300A78300A673178323079323048
:108B40007A323066353030202866656564206120D1
:108B500032306D6D20646961676F6E616C20696E83
:108B600020582C205920616E64205A290A783079C7
:108B7000307A300A7834307934307A3430202874BE
:108B80007261766572736520612034306D6D20638B
:108B900075626520696E20582C205920616E642012
:108BA0005A290A78343079307A300A78307934307A
:108BB0007A34300A7834307934307A300A7830793F
:108BC000307A34300A78307934307A300A78343078
:108BD00079307A34300A783079307A300A67383030
:108BE0000A6730783079300A673078310A67307830
:108BF000300A6D333000284D53472A2A2A2A20484C
:108C00006F6D696E672054657374205B76315D20EB
:108C10002A2A2A2A290A6732382E32783079307A7D
:108C2000300A6D333000284D53472A2A2A2A205310
:108C30006D6F6B652054657374205B76315D202AFF
:108C40002A2A2A290A473030204731372047323133
:108C500020473430204734392047383020473930D6
:108C60000A6D33673470310A6D35673470310A6DBF
:108C700034673470310A6D33673470310A6D35678B
:108C80003470310A6D37673470310A6D396734706A
:108C9000310A6D38673470310A6D390A67307830BF
:108CA00079307A300A673030207832300A78300AEA
:108CB0007932300A79300A7A32300A7A300A6132EF
:108CC000300A61300A473030207832302079323033
:108CD000207A3230206132300A473030207830201C
:108CE0007930207A302061300A47303120663330C5
:108CF000207832207932207A322061320A7830208E
:108D00007930207A302061300A673078310A673054
:108D100078300A6D32005B74765D2020746578745B
:108D200020766572626F7369747925313564205BD2
:108D3000303D73696C656E742C313D766572626F7F
:108D400073655D0A0025660A00256C750A002573A7
:108D50000A0074696E7967205B25735D2065727205
:108D60003A2025733A202573200074696E796720B4
:108D70005B25735D206F6B3E2000456E64206F663F
:108D800020636F6D6D616E642066696C650A0069B1
:108D9000C80BC6D6C8F7C856C950C62ECC0BC6C21B
:108DA000CC2ECD5CCB50C60000400640061040B82B
:108DB00000B82ECC0BC6C2CC2ECD5CCB50C600006A
:108DC000400620060840B800B897CE0BC6B7CD3392
:108DD000CEE2CF80CDA0084006050609010897CE57
:108DE0000BC6B7CD33CE68C950C6B00840060540A3
:108DF000B030800000000000F0E0D0C0100100CFD3
:108E0000673322211F1B1301016E616E00696E66BC
:108E1000004E414E494E495459494E46CDCCCC3D69
:108E20000AD7233C17B7D13877CC2B329595E62457
:108E30001FB14F0A000020410000C84200401C46FC
:108E400020BCBE4CCA1B0E5AAEC59D7400407A10A1
:108E5000F35A00A0724E18090010A5D4E80000E8EB
:108E60007648170000E40B54020000CA9A3B000049
:108E700000E1F505000080969800000040420F00D8
:108E80000000A08601000000102700000000E80399
:108E9000000000006400000000000A000000000064
:108EA0000100000000002C76D888DC674F0823DF23
:108EB000C1DFAE59E1B1B796E5E3E453C63AE651F6
:108EC000997696E8E6C28426EB898C9B62ED407C1D
:108ED0006FFCEFBC9C9F40F2BAA56FA5F490055AB9
:108EE0002AF75C936B6CF9676DC11BFCE0E40D47DE
:108EF000FEF520E6B500D0ED902E03009435770501
:108F00000080841E080000204E0A000000C80C33B8
:108F10003333330F986E12831141EF8D2114893B47
:108F2000E65516CFFEE6DB18D1844B381BF77C1DC7
:108F3000901DA4BBE424203284725E228100C9F11A
:108F400024ECA1E53D2711241FBECFEFCDBFDFE507
:108F5000DEBF00E00CBF13E2A0E0B0E2E8E0F7EC17
:108F600001E00BBF02C007900D92AA38B107D9F7F4
:108F70002CE5AAE8B3E201C01D92A237B207E1F7DF
:108F80000E9440810C9482E30C940000FC016081FB
:108F90007181828193810E9430D560933F3508951D
:108FA000FC0160817181828193810E9430D5609340
:108FB0003E350895AF92BF92CF92DF92EF92FF922B
:108FC0000F931F93CF93DF937B018C0182ECC82E0C
:108FD00084E3D82EE601AA24A394BC2EBC18F70182
:108FE00061917191819191917F012CEA35EC47E279
:108FF00057E30E94BFD618164CF4F8014081518106
:10900000628173818B2D0E946F82A8820C5F1F4F3B
:109010002196F4E3C83CDF0701F7DF91CF911F9160
:109020000F91FF90EF90DF90CF90BF90AF900C9496
:109030007A82FC0160817181828193810E9430D5A6
:1090400060934035613019F481E00E94407881E0FE
:109050000C946178CF93DF93CDB7DEB76897CDBF1F
:10906000DEBFFC0160817181828193810E9430D5D5
:109070006093413581E0613019F40E9440780CC062
:109080000E946178CE01019628E1FC0111922A9597
:10909000E9F7BC010E9419486896CDBFDEBFDF9199
:1090A000CF9108950F931F93CF93DF93CDB7DEB782
:1090B0002D97CDBFDEBF27E0E8EDF0E28E010F5F18
:1090C0001F4FD80101900D922A95E1F7BC01660F60
:1090D000771F680F791F660F771F660F771F660F60
:1090E000771F69557A4E45E050E0CE0108960E9400
:1090F000F6E0688570E0C8010E9424E1009739F429
:109100006B8570E0C8010E9424E1009711F0801B7C
:1091100001C08FEF2D96CDBFDEBFDF91CF911F91A4
:109120000F9108950F931F93CF93DF93CDB7DEB7C1
:10913000C058D109CDBFDEBFFC010D9624852F9309
:1091400023852F9322852F9321852F939F938F9390
:109150007196FF93EF939F938F937F936F938E01FD
:109160000F5F1F4F1F930F930E94ADE2C8010E9433
:109170001FC0CDBFDEBFC058DF4FCDBFDEBFDF9108
:10918000CF911F910F910895EF92FF920F931F932C
:10919000CF93DF93CDB7DEB7C058D109CDBFDEBFC7
:1091A0008C01F62EE72EFC01848195810E945248A5
:1091B00083309CF58F3F09F03BC02FC09801235F9F
:1091C0003F4F9F938F93F80184858F9383858F936F
:1091D00082858F9381858F933F932F930F5E1F4FCF
:1091E0001F930F933F932F93EF92FF928E010F5F88
:1091F0001F4F1F930F930E94ADE2C8010E941FC032
:10920000CDBFDEBFC058DF4FCDBFDEBFDF91CF91F6
:109210001F910F91FF90EF900895E6E2F4E16591C0
:1092200074914FE450E086E69FE30E94F6E0C6CFDB
:10923000E0913835F0E0EE0FFF1FEE5DFB4E6591DB
:1092400074914FE450E086E69FE30E94F6E0B6CFCB
:10925000EF92FF920F931F93CF93DF93CDB7DEB7BB
:10926000C058D109CDBFDEBF8C01F62EE72EFC0120
:10927000848195810E9452488330B4F58F3F09F074
:109280003EC032C0A8014F5E5F4F9801235F3F4F41
:109290009F938F93F80184858F9383858F93828525
:1092A0008F9381858F935F934F933F932F935F931A
:1092B0004F933F932F93EF92FF928E010F5F1F4FBB
:1092C0001F930F930E94ADE2C8010E941FC0CDBF43
:1092D000DEBFC058DF4FCDBFDEBFDF91CF911F9102
:1092E0000F91FF90EF900895E6E2F4E1659174919B
:1092F0004FE450E086E69FE30E94F6E0C3CFE091A2
:109300003835F0E0EE0FFF1FEE5DFB4E6591749176
:109310004FE450E086E69FE30E94F6E0B3CFDF9291
:10932000EF92FF920F931F93CF93DF93CDB7DEB7EA
:10933000C858D109CDBFDEBF8B01E42ED52E37E052
:10934000EFEDF0E2DE01AF57BF4F01900D923A957D
:10935000E1F7C857DF4F2883C858D0400E945248D1
:10936000F82EC857DF4F2881C858D04082E08F15AB
:1093700018F0E22FF0E002C0E2E0F0E0EE0FFF1F95
:10938000EE5DFB4E659174914FE450E086E69FE3FD
:109390000E94F6E09F938F93F80183818F938281DF
:1093A0008F9381818F9380818F93E1E8F0E0EC0FC0
:1093B000FD1FEF0DF11D80811F928F93DF92EF92C1
:1093C0008E010F5F1F4F1F930F930E94ADE2C801E4
:1093D0000E941FC0CDBFDEBFC857DF4FCDBFDEBF6D
:1093E000DF91CF911F910F91FF90EF90DF90089543
:1093F0004F925F926F927F92AF92BF92CF92DF9225
:10940000EF92FF920F931F93CF93DF93C2ECD4E3BD
:1094100007E813E35C018991813009F042C0F8014B
:10942000C480D580E680F780408051806280738060
:10943000A3019201C701B6010E9413D39F772CEAC2
:1094400035EC47E257E30E94BCD487FD2AC020E0F8
:1094500034E244E759ECC701B6010E94BFD61816A2
:109460005CF4F5012081318142815381C701B6014D
:109470000E94BFD6181604F120E034E244E759EC0C
:10948000C301B2010E94BFD618165CF4F501208119
:10949000318142815381C301B2010E94BCD487FD56
:1094A0000BC00B5C1F4FF4E0AF0EB11C84E3C83C53
:1094B000D80709F0B0CF02C08CED01C080E0DF9189
:1094C000CF911F910F91FF90EF90DF90CF90BF90C1
:1094D000AF907F906F905F904F9008958091BE34D1
:1094E000811105C08091BD348093BC3429C0823085
:1094F00031F487E08093BC348091BD3421C0833047
:1095000031F489E08093BC348091BD3419C084303B
:1095100031F48AE08093BC348091BD3411C08091D5
:10952000BF34813031F485E08093BC348091BD3408
:1095300007C0823019F486E08093BC348091BD343A
:10954000863019F08091BC3408958BE08093BC3450
:1095500008958091BD3408958093BF34813059F0CF
:1095600018F0823041F008958DEE94E38093EB344F
:109570009093EC34089585EB98E58093EB349093C9
:10958000EC340895FC0184810895845B9F4FFC01B5
:1095900080810895855B9F4FFC0180810895825BE7
:1095A0009F4FFC0180810895815B9F4FFC0180816A
:1095B0000895875B9F4FFC01808108950C947097FC
:1095C000CD96FC0160817181828193810895FC01B7
:1095D000648308958B5A9F4FFC01608308958F5BCD
:1095E0009F4FFC014083518362837383089560938E
:1095F000ED347093EE348093EF349093F03488EE32
:1096000091E20C949C62BF92CF92DF92EF92FF9214
:109610000F931F93CF93DF93D0903A357C010FE5E2
:1096200015E38091393590E0EC01CC0FDD1FC80FB8
:10963000D91FCC0FDD1FCC0FDD1FCC0FDD1FCA5291
:10964000DD4C81E0D816A9F0B881A981CA80BB8021
:109650004091B235413091F4F8012081318142814D
:1096600053816B2F7A2F8C2D9B2D0E9414D39B013D
:1096700009C020E030E080E090E004C02B2F3A2FBA
:109680008C2D9B2DA901BC01F701458F568F678F4B
:1096900070A3F4E0EF0EF11C0C5F1F4F249685E3DE
:1096A0000737180771F6DF91CF911F910F91FF9047
:1096B000EF90DF90CF90BF900895835B9F4FFC01A8
:1096C00060838DEE94E30C94034B4F925F926F9204
:1096D0007F928F929F92AF92BF92CF92DF92EF9242
:1096E000FF920F931F93CF93DF93CDB7DEB76897A9
:1096F000CDBFDEBF8C016091B23570E080E090E0BC
:109700000E945ED52B013C01F8016081718182814C
:1097100093810E9430D570E05B01AA0CBB1CA60EA1
:10972000B71EAA0CBB1CAA0CBB1CAA0CBB1CC501F7
:109730008A529D4C5C010FE515E3FE0131964F0105
:10974000F501C190D190E190F1905F01F801619134
:109750007191819191918F01A30192010E9461D732
:109760009B01AC01C701B6010E9414D3F4016193BF
:109770007193819391934F01F5E307371F0701F729
:10978000CE0101960E9453978DEE94E30E94034B05
:109790006896CDBFDEBFDF91CF911F910F91FF90F3
:1097A000EF90DF90CF90BF90AF909F908F907F9081
:1097B0006F905F904F9008958D5E944369F4E62F0B
:1097C000F0E0EE0FFF1FEE0FFF1FE95BFA4C608128
:1097D0007181828193810895862F0C944897CF924E
:1097E000DF92EF92FF920F931F93CF93DF93EC01E1
:1097F00084E3CD3ED80709F04AC070E0FB01EE0FCC
:10980000FF1FEE0FFF1FE95BFA4CC080D180E280A2
:10981000F38080913A35813059F18091393590E06B
:10982000FC01EE0FFF1FE80FF91FEE0FFF1FE60F01
:10983000F71FEE0FFF1FEE0FFF1FEA52FD4C0081D6
:109840001181B281A3812091B2352130B1F4FB01A5
:10985000EE0FFF1FEE0FFF1FE15AFA4C20813181FE
:1098600042815381B8018B2F9A2F0E9414D308C0D4
:1098700060E070E080E090E003C0B8018B2F9A2F89
:109880009B01AC01C701B6010E9413D303C0862F10
:109890000E945C97C55BDF4F2881211106C023E33E
:1098A00033E34BEC51E40E94C3D4DF91CF911F917D
:1098B0000F91FF90EF90DF90CF90089588E1E2EF55
:1098C000F4E3A7E4B5E301900D928A95E1F7809166
:1098D000363581110CC08091F134813041F4109201
:1098E0002A3510922B3510922C3510922D35089573
:1098F0004F925F926F927F928F929F92AF92BF92A0
:10990000CF92DF92EF92FF920F931F93CF93DF934B
:10991000CDB7DEB76997CDBFDEBF8091BE34811170
:1099200055C08091E334813009F050C00E94AAC52F
:1099300081114CC01092E3349EEE692E92E3792E91
:1099400026E3822E912C8E010E5E1F4F36EEA32E43
:1099500030E2B32E33C0F70181917F011F928F93C4
:109960005F924F92BF92AF921F930F930E9484E237
:10997000B80187E493E20E94BE5F8D839E83F60167
:1099800081919191A191B1916F018A879B87AC8759
:10999000BD87CE0101960E94865CCDBFDEBF9EEDE5
:1099A000E91690E2F906B9F6E8E16E0E711CFFEFD8
:1099B0008F1A9F0A8CE38816910441F0240189EDE7
:1099C000E82E80E2F82E630188E7C8CF80E0699630
:1099D000CDBFDEBFDF91CF911F910F91FF90EF9030
:1099E000DF90CF90BF90AF909F908F907F906F90BF
:1099F0005F904F9008952F923F924F925F926F9297
:109A00007F928F929F92AF92BF92CF92DF92EF920E
:109A1000FF920F931F93CF93DF93CDB7DEB72997B4
:109A2000CDBFDEBF4C015B0140903C3550903A35D4
:109A3000209039356090B235709038356B0182EFE7
:109A400094E3888799875EE7E52E53E3F52E98E146
:109A5000299E100111248401D6016D917D918D9173
:109A60009D916D012CEA35EC47E257E30E94BCD48E
:109A700087FD80C0F70180818150823008F07AC074
:109A800041104CC0F1E05F1609F1E885F985E20D5F
:109A9000F31DEC51F2408081898391819D83B281D5
:109AA000A381E1E06E1217C0E885F985E359FF4F05
:109AB0002081318142815381BC018B2F9A2F0E94DA
:109AC00014D369837D838E839F8307C019821D828F
:109AD0001E821F8202C0BE83AF8371100CC023E3BD
:109AE00033E34BEC51E4D8016D917D918D919C91C4
:109AF0000E9461D705C0F8016081718182819381E4
:109B000029813D814E815F810E9414D3A885B9854A
:109B10006D937D938D939C9313972CC0A885B985E5
:109B20008D919D910D90BC91A02D89839A83AB83DB
:109B3000BC8371100EC023E333E34BEC51E4F80116
:109B400060817181828193810E9461D79B01AC0108
:109B500005C0D8012D913D914D915C9169817A812B
:109B60008B819C810E9414D3E885F9856083718381
:109B7000828393838885998504968887998795E35E
:109B8000E90EF11C0C5F1F4FA885B985AE5FB44389
:109B900009F062CF6090383570903C35F0913A35DD
:109BA000F983C09039352091B2352D838CE0A80E11
:109BB000B11CADE1B4E3A887B9874EEFE42E44E3CE
:109BC000F42EB8E1CB9E600111248401F50161916E
:109BD0007191819191915F012CEA35EC47E257E355
:109BE0000E94BCD487FD8CC0A885B9858C91882340
:109BF00009F486C08150823030F4F8012484358421
:109C0000468457843BC0611016C023E333E34BEC1A
:109C100051E4D8011C966D917D918D919C911F9777
:109C20000E9461D720E030E044EB53E40E9461D70A
:109C30001B012C010DC020E030E044EB53E4F8019F
:109C400064857585868597850E9461D71B012C01E7
:109C50002BED3FE049EC50E4A885B98591966D91D4
:109C60007D918D919C9194970E9461D79B01AC014D
:109C7000C201B1010E94C3D41B012C01711031C07B
:109C8000B981B130E1F0F701EC0DFD1DEC51F2406E
:109C9000A081B18192808380ED81E130A1F4F70150
:109CA000E359FF4F2081318142815381BD01892DCC
:109CB000982D0E9414D3DB01982E892E04C0A0E0B9
:109CC000B0E0912C812CA2019101BD01892D982D2C
:109CD0000E9414D3D7016D937D938D939C9313971A
:109CE0000FC0A2019101F70160817181828193818E
:109CF0000E9414D3D7016D937D938D939C931397FA
:109D0000E885F985F596E887F987F4E0EF0EF11C10
:109D10000C5F1F4F888599858C5B944309F056CF63
:109D20002996CDBFDEBFDF91CF911F910F91FF909C
:109D3000EF90DF90CF90BF90AF909F908F907F90EB
:109D40006F905F904F903F902F9008958091BA321E
:109D50009091BB328F3E924111F08FE50895809132
:109D60007136909172368F3E9241B9F780914335AA
:109D7000909144358F3E924181F78091B935909111
:109D8000BA358F3E924149F780910D5990910E5905
:109D90008F3E924111F78091CA599091CB598F3ED5
:109DA0009241D9F680E00895CF93C82F0E945FA812
:109DB00082E08093BD348C2FCF9108958091BE3482
:109DC000811104C083E08093BD3403C085E080939B
:109DD000BD3480E00895CF93C82F0E94A3B380E0E4
:109DE0000E9438AF8C2F0E945FA886E08093BD341C
:109DF0008C2FCF91089581E08093E43480E0089522
:109E000081E08093E63480E0089581E08093E5343A
:109E100080E008950E94FA7880E0089580933735B5
:109E200080E008958093383580E0089580933C3534
:109E300080E008954F925F926F927F929F92AF92CF
:109E4000BF92CF92DF92EF92FF920F931F93CF9327
:109E5000DF93C82FB62E8A01F22ED32F8FEF8C0FEF
:109E6000863008F082C06091453670E080E090E076
:109E70000E945ED52CEA35EC47E257E30E94BCD441
:109E800087FD75C082E0B81619F0E4E1BE1271C01A
:109E900090903835CF2CDD2E8C2F90E0EC01CC0F3C
:109EA000DD1FC80FD91FCC0FDD1FCC0FDD1FCC0F5E
:109EB000DD1FCA52DD4C780107E415E3AA24A39400
:109EC000F60161917191819191916F012CEA35ECCC
:109ED00047E257E30E94BFD61816DCF5F2E0BF1246
:109EE00014C091100CC023E333E34BEC51E4F701B1
:109EF00060817181828193810E9461D724C0F701C2
:109F000060817181828193811EC0F80140805180FF
:109F10006280738091100EC023E333E34BEC51E475
:109F2000F70160817181828193810E9461D79B01D9
:109F3000AC0105C0F7012081318142815381C30109
:109F4000B2010E9413D3688379838A839B83A09292
:109F5000E3342496F4E0EF0EF11C0C5F1F4F85E311
:109F60000F35180709F0ACCF06C081EA05C08CEAAE
:109F700003C08DEA01C080E0DF91CF911F910F9166
:109F8000FF90EF90DF90CF90BF90AF909F907F9029
:109F90006F905F904F900895CF93DF93CDB7DEB76A
:109FA0006897CDBFDEBF80933935682F70E080E0C1
:109FB00090E00E945CD569837A838B839C831D82A9
:109FC0001E821F82188619861A861B861C861D868D
:109FD0001E861F86188A198A1A8A1B8A1C8A1D8A5D
:109FE0001E8A1F8A188EAE014F5F5F4FBA0185E649
:109FF0009BE40E94B18380E06896CDBFDEBFDF9115
:10A00000CF910895CF93DF93EDEEF4E386E5DF0182
:10A010001D928A95E9F78BE5ABEBB5E3ED01982F3F
:10A0200019929A95E9F7A6E1B6E3ED0119928A959E
:10A03000E9F78FEE92E18093BA329093BB3280932E
:10A040007136909372368093433590934435809364
:10A05000B9359093BA3580930D5990930E598093EA
:10A06000CA599093CB59E093EB34F093EC34809140
:10A07000D332809338358091D1320E94CC4F809179
:10A08000D232809337358091D43280933B358091A2
:10A09000D53280933C3581E0809336358093B3355B
:10A0A00094E09093F1341092E4341092E5341092DD
:10A0B000E6348093BD348093BC340E94D6ADDF91EA
:10A0C000CF910C94F384CF92DF92EF92FF92CF93D3
:10A0D000C82F6A017B01E82FF0E0DF01AA0FBB1F48
:10A0E000AA0FBB1FA95BBA4C4D935D936D937C93F4
:10A0F0001397EE0FFF1FEE0FFF1FEE50FB4C408338
:10A100005183628373838C2F0E946482B701A601FE
:10A110008C2F0E946F82CF91FF90EF90DF90CF90B5
:10A120000C947A829F92AF92BF92CF92DF92EF927D
:10A13000FF920F931F93CF93DF93CDB7DEB768974E
:10A14000CDBFDEBF962EA72EC62ED72E7C0100E0F7
:10A1500010E0B12CF60161917191819191916F01A3
:10A160002CEA35EC47E257E30E94BFD61816A4F557
:10A170008091383581110EC023E333E34BEC51E479
:10A18000F70160817181828193810E9461D7AB0167
:10A19000BC0105C0F7014081518162817381E1E01A
:10A1A000F0E0EC0FFD1FE00FF11F4083518362834D
:10A1B0007383C80186549D4CFC01E357FD4F4083D7
:10A1C000518362837383E555F10940835183628330
:10A1D00073838B2D0E946482B3940C5F1F4FF4E055
:10A1E000EF0EF11C0831110509F0B4CF492D5A2D9D
:10A1F000BE016F5F7F4F8AED97E40E94B18380E0DC
:10A200006896CDBFDEBFDF91CF911F910F91FF9078
:10A21000EF90DF90CF90BF90AF909F9008954F92B6
:10A220005F926F927F928F929F92AF92BF92CF92E6
:10A23000DF92EF92FF920F931F93CF93DF93CDB7EF
:10A24000DEB76897CDBFDEBF21E02093B2358090A6
:10A250003935909038355B016C0107E415E3882DA2
:10A2600090E07C01EE0CFF1CE80EF91EEE0CFF1CCA
:10A27000EE0CFF1CEE0CFF1CC7018A529D4C7C01AA
:10A28000F50161917191819191915F012CEA35EC19
:10A2900047E257E30E94BFD6181664F5F701208104
:10A2A000318142815381F801608171818281938182
:10A2B0000E9413D32B013C0191100EC023E333E322
:10A2C0004BEC51E4F60160817181828193810E949F
:10A2D00061D79B01AC0105C0F6012081318142812B
:10A2E0005381C301B2010E9413D3F801608F718FB3
:10A2F000828F938FF4E0CF0ED11C0C5F1F4F84E050
:10A30000E80EF11C95E30F35190709F0B9CF682D58
:10A3100070E080E090E00E945CD569837A838B8353
:10A320009C831D821E821F82188619861A861B86B0
:10A330001C861D861E861F86188A198A1A8A1B8A01
:10A340001C8A1D8A1E8A1F8A188EAE014F5F5F4FBE
:10A35000BA0185E69BE40E94B18380E06896CDBF98
:10A36000DEBFDF91CF911F910F91FF90EF90DF90B3
:10A37000CF90BF90AF909F908F907F906F905F90A5
:10A380004F900895CF93DF93CDB7DEB76897CDBFD9
:10A39000DEBF1092B23510925F3510926035109288
:10A3A00061351092623510926335109264351092C7
:10A3B00065351092663510926735109268351092A7
:10A3C000693510926A3510926B3510926C35109287
:10A3D0006D3510926E3510926F3510927035109267
:10A3E0007135109272351092733510927435109247
:10A3F0007535109276356091393570E080E090E0E7
:10A400000E945CD569837A838B839C831D821E8224
:10A410001F82188619861A861B861C861D861E8634
:10A420001F86188A198A1A8A1B8A1C8A1D8A1E8A04
:10A430001F8A188EAE014F5F5F4FBA0185E69BE41D
:10A440000E94B18380E06896CDBFDEBFDF91CF91DF
:10A450000895CF93DF93CDB7DEB76897CDBFDEBF4A
:10A460001092B2356091393570E080E090E00E9442
:10A470005CD569837A838B839C831D821E821F82B5
:10A48000188619861A861B861C861D861E861F86C0
:10A49000188A198A1A8A1B8A1C8A1D8A1E8A1F8A90
:10A4A000188EAE014F5F5F4FBA0185E69BE40E94B4
:10A4B000B18380E06896CDBFDEBFDF91CF91089574
:10A4C000CF93DF93CDB7DEB76897CDBFDEBF81E016
:10A4D0008093B2356091393570E080E090E00E9461
:10A4E0005CD569837A838B839C831D821E821F8245
:10A4F000188619861A861B861C861D861E861F8650
:10A50000188A198A1A8A1B8A1C8A1D8A1E8A1F8A1F
:10A51000188EAE014F5F5F4FBA0185E69BE40E9443
:10A52000B18380E06896CDBFDEBFDF91CF91089503
:10A53000CF931092F1340E94FB4C8091C432813051
:10A5400069F482EF94E30E94F849C82F882331F020
:10A550000E945FA882E08093BD3417C08DEE94E323
:10A560000E94034B85E08093BD348091BE348111FD
:10A5700005C081E08093BE340E944BAC8DEE94E325
:10A580000E947D970E945E4CC0E08C2FCF91089571
:10A5900088E1E7E4F5E3A7E7B5E301900D928A953A
:10A5A000E1F780E008950F931F93CF93DF93CDB72A
:10A5B000DEB76A97CDBFDEBF8C0181E080933A356C
:10A5C0008DEE94E3698F7A8F0E94034B698D7A8DAB
:10A5D000C8010E9498520E94EB828823E1F388E12F
:10A5E000E0E0F0E2DE01119601900D928A95E1F72C
:10A5F000BE016F5F7F4F87E795E30E9498526A968E
:10A60000CDBFDEBFDF91CF911F910F91089588E1FB
:10A61000E7E4F5E3AFE8B5E301900D928A95E1F741
:10A6200080E008950F931F93CF93DF93CDB7DEB7EC
:10A630006A97CDBFDEBF8C0181E080933A358DEE05
:10A6400094E3698F7A8F0E94034B698D7A8DC801DC
:10A650000E9498520E94EB828823E1F388E1E0E0B7
:10A66000F0E2DE01119601900D928A95E1F7BE01AC
:10A670006F5F7F4F8FE895E30E9498526A96CDBF37
:10A68000DEBFDF91CF911F910F910895FB01DC0197
:10A6900080913635811111C09B01AD0160E070E001
:10A6A00080E89FE30E94C3D460932A3570932B35D2
:10A6B00080932C3590932D3518C0809138358111B9
:10A6C00009C023E333E34BEC51E4CD010E9461D791
:10A6D000FB0101C0CD01AF01BC0140932A3550936D
:10A6E0002B3560932C3570932D3580E00895809341
:10A6F000363580E0089580933B3580E0089560937F
:10A7000032357093333580933435909335350E94CC
:10A71000098480E008950F931F93CF93DF93EC019A
:10A720008B0180913635882399F080912A3590915C
:10A730002B35A0912C35B0912D35BC01CD019F77E3
:10A740002CEA35EC47E257E30E94BCD487FD30C0C9
:10A7500081E08093F134B801CE010E94FB4C8091DE
:10A76000C432813069F482EF94E30E94F849C82F23
:10A77000882331F00E945FA882E08093BD3419C025
:10A780008DEE94E30E94034B85E08093BD3480916D
:10A79000BE34811105C081E08093BE340E944BAC71
:10A7A0008DEE94E30E947D97C82F0E945E4C01C0FD
:10A7B000CEE88C2FDF91CF911F910F910895CF9309
:10A7C000DF93CDB7DEB76897CDBFDEBF682F70E0EF
:10A7D00080E090E00E945CD569837A838B839C83C0
:10A7E0001D821E821F82188619861A861B861C8669
:10A7F0001D861E861F86188A198A1A8A1B8A1C8A39
:10A800001D8A1E8A1F8A188EAE014F5F5F4FBA01E4
:10A8100086EC97E40E94B18380E06896CDBFDEBFEE
:10A82000DF91CF910895CF93DF93CDB7DEB76897CF
:10A83000CDBFDEBF60913F3570E080E090E00E94C8
:10A840005CD569837A838B839C831D821E821F82E1
:10A85000188619861A861B861C861D861E861F86EC
:10A86000188A198A1A8A1B8A1C8A1D8A1E8A1F8ABC
:10A87000188EAE014F5F5F4FBA0180ED97E40E94E2
:10A88000B18380E06896CDBFDEBFDF91CF910895A0
:10A89000CF93DF93CDB7DEB76897CDBFDEBF682F0C
:10A8A00070E080E090E00E945CD569837A838B83BE
:10A8B0009C831D821E821F82188619861A861B861B
:10A8C0001C861D861E861F86188A198A1A8A1B8A6C
:10A8D0001C8A1D8A1E8A1F8A188EAE014F5F5F4F29
:10A8E000BA0189E198E40E94B18380E06896CDBF07
:10A8F000DEBFDF91CF910895CF93DF93CDB7DEB761
:10A900006897CDBFDEBF682F70E080E090E00E94C6
:10A910005CD569837A838B839C831D821E821F8210
:10A92000188619861A861B861C861D861E861F861B
:10A93000188A198A1A8A1B8A1C8A1D8A1E8A1F8AEB
:10A94000188EAE014F5F5F4FBA018AE298E40E9411
:10A95000B18380E06896CDBFDEBFDF91CF910895CF
:10A96000CF93FC0160817181828193810E9430D5F7
:10A970006093BD341092BF348DEE94E38093EB343A
:10A980009093EC348091BE34813011F41092BE3437
:10A990001092C0341092E6340E943697C091BD34B4
:10A9A000C430C9F40E94C2518091D1320E94CC4F70
:10A9B0008091D232809337358091D53280933C3567
:10A9C00080E00E9438AF80E00E947C5481E0809358
:10A9D0003635C093F13481E0CF910C9429AB80934C
:10A9E000AF358093B0358093B83580E008952CEA78
:10A9F00035EC47E257E360915D3670915E368091A9
:10AA00005F36909160360E94BFD61816B4F48091DC
:10AA1000023690910336A0910436B0910536BC0100
:10AA2000CD019F772CEA35EC47E257E30E94BCD476
:10AA300087FF03C01092AF3503C081E08093AF352C
:10AA400080E008958093AF3580910236909103366F
:10AA5000A0910436B09105368093A7359093A83520
:10AA6000A093A935B093AA3580E008952CEA35EC7F
:10AA700047E257E360915D3670915E3680915F36B4
:10AA8000909160360E94BFD61816B4F480910236B9
:10AA900090910336A0910436B0910536BC01CD01EA
:10AAA0009F772CEA35EC47E257E30E94BCD487FF3E
:10AAB00003C01092B03503C081E08093B03580E0D0
:10AAC00008958093B0358091023690910336A0911D
:10AAD0000436B09105368093AB359093AC35A09396
:10AAE000AD35B093AE3580E008952CEA35EC47E201
:10AAF00057E360915D3670915E3680915F3690913C
:10AB000060360E94BFD61816B4F480910236909138
:10AB10000336A0910436B0910536BC01CD019F7774
:10AB20002CEA35EC47E257E30E94BCD487FF03C010
:10AB30001092B83503C081E08093B83580E0089565
:10AB40008093B8358091023690910336A0910436F7
:10AB5000B09105368093B4359093B535A093B63552
:10AB6000B093B73580E00895BC018DEE90E20C946F
:10AB7000BF6281E08093E434089581E08093E534FE
:10AB8000089581E08093E63408951F93CF93DF9377
:10AB9000CDB7DEB76897CDBFDEBF0E94709781301A
:10ABA000C9F10E945AD10E945EC80E946E8380E063
:10ABB0000E9460AC10E0812F0E944897AB01BC015D
:10ABC000812F0E9463501F5F1630A9F780E090E04C
:10ABD000A0E4B0E489839A83AB83BC831D821E8288
:10ABE0001F82188619861A861B861C861D861E865D
:10ABF0001F86188A198A1A8A1B8A1C8A1D8A1E8A2D
:10AC00001F8A188EBE016F5F7F4FCB010E94B05428
:10AC100080E001C08AE66896CDBFDEBFDF91CF91AC
:10AC20001F9108958091E4348130A9F42091BF34BC
:10AC3000213079F48091C03481110BC082E080937F
:10AC4000BF3485EB98E58093EB349093EC342093FC
:10AC5000C0341092E4348091E534813091F48091D5
:10AC6000BF34882331F0823061F49091C034943045
:10AC700051F40E947097811104C01092E5340E9433
:10AC8000C5559091C0348091E6348130C1F4209153
:10AC9000E534211114C09150933088F01092E634BD
:10ACA00095E09093C0349093BD349091BE3491114F
:10ACB00004C08093BE340E944BAC0E94E29F80E0AF
:10ACC000089585E08093BD348091BE34811105C024
:10ACD00081E08093BE340C944BAC0895CF93DF9306
:10ACE000CDB7DEB76897CDBFDEBF8091BE34882375
:10ACF00011F180E090E0A0E4B0E489839A83AB8313
:10AD0000BC831D821E821F82188619861A861B86A6
:10AD10001C861D861E861F86188A198A1A8A1B8A17
:10AD20001C8A1D8A1E8A1F8A188EBE016F5F7F4F84
:10AD3000CB010E94B0546896CDBFDEBFDF91CF91AA
:10AD40000895CF93DF93CDB7DEB76897CDBFDEBF51
:10AD500080E090E0A0E4B0E489839A83AB83BC8375
:10AD60001D821E821F82188619861A861B861C86E3
:10AD70001D861E861F86188A198A1A8A1B8A1C8AB3
:10AD80001D8A1E8A1F8A188EAE014F5F5F4FBA015F
:10AD900080EB94E50E94B1836896CDBFDEBFDF9162
:10ADA000CF910895CF93DF93CDB7DEB76897CDBF2E
:10ADB000DEBF80E090E0A0E8B0E489839A83AB83B3
:10ADC000BC831D821E821F82188619861A861B86E6
:10ADD0001C861D861E861F86188A198A1A8A1B8A57
:10ADE0001C8A1D8A1E8A1F8A188EAE014F5F5F4F14
:10ADF000BA0180EB94E50E94B1836896CDBFDEBFB7
:10AE0000DF91CF910895CF93DF93CDB7DEB727972A
:10AE1000CDBFDEBF97E0EFEDF0E2DE0111960190CD
:10AE20000D929A95E1F7873050F4E1E0F0E0EC0FF5
:10AE3000FD1FE80FF11D87FDFA95808101C080E2BA
:10AE40002796CDBFDEBFDF91CF9108950F931F935B
:10AE5000CF93DF93EC01042F10E020E030E009876E
:10AE60001A872B873C8782E08F8350E0440F551F61
:10AE7000640F751FFB01659174914FE450E086E605
:10AE80009FE30E94F6E0BC01CE01DF91CF911F91BC
:10AE90000F910C946162CF93DF93EC010E946E4A94
:10AEA000482F60E673E1CE01DF91CF910C942657D5
:10AEB0004091BD3461E273E10C9426574091BE3459
:10AEC00068EF72E10C9426574091BF3464EE72E152
:10AED0000C9426574091C03466EB72E10C942657CF
:10AEE0004091C13469E972E10C942657E091EB344A
:10AEF000F091EC34E55BFF4F408163EC73E10C941F
:10AF00002657E091EB34F091EC34E45BFF4F408145
:10AF10006FEC71E10C942657E091EB34F091EC3436
:10AF2000448165E371E10C942657E091EB34F09194
:10AF3000EC34E65BFF4F408162E071E10C942657F0
:10AF4000E091EB34F091EC34E25BFF4F408168EB31
:10AF500070E10C942657E091EB34F091EC34E15B16
:10AF6000FF4F408167E770E10C942657E091EB3486
:10AF7000F091EC34E75BFF4F408168E070E10C94A6
:10AF80002657E091EB34F091EC34EF5AFF4F4081BB
:10AF900050E060E070E0FC0141875287638774876E
:10AFA00022E0278380E00895E091EB34F091EC34C7
:10AFB0004081518162817381FC014187528763879F
:10AFC000748722E0278380E00895CF93DF93EC011C
:10AFD0008091BF34811105C019861A861B861C8694
:10AFE00014C00E943F9769877A878B879C8720913E
:10AFF000005921110AC025E832E441E25DE30E94D4
:10B0000061D769877A878B879C878C819D81FC01BA
:10B01000EE0FFF1FE80FF91FEE0FFF1FEE0FFF1FD0
:10B02000EE0FFF1FE255FA4E85919491888784E0D8
:10B030008F8380E0DF91CF910895CF93DF93EC0170
:10B040002091EB343091EC34F901FD9660817181EF
:10B050008281938169877A878B879C873E9620813E
:10B0600021110AC025E832E441E25DE30E9461D784
:10B0700069877A878B879C878C819D81FC01EE0F85
:10B08000FF1FE80FF91FEE0FFF1FEE0FFF1FEE0F60
:10B09000FF1FE255FA4E85919491888784E08F8353
:10B0A00080E0DF91CF910895CF93DF93EC018C8105
:10B0B0009D810E945248682F8091EB349091EC342E
:10B0C0000E94EF4B69877A878B879C878C819D8153
:10B0D000FC01EE0FFF1FE80FF91FEE0FFF1FEE0F31
:10B0E000FF1FEE0FFF1FE255FA4E8591949188875E
:10B0F00084E08F8380E0DF91CF910895CF93DF9339
:10B10000EC018C819D810E9452482091EB3430915A
:10B11000EC342D5E344369F4E82FF0E0EE0FFF1FAE
:10B12000EE0FFF1FE95BFA4C608171818281938190
:10B1300002C00E94489769877A878B879C878C8199
:10B140009D81FC01EE0FFF1FE80FF91FEE0FFF1F9F
:10B15000EE0FFF1FEE0FFF1FE255FA4E85919491FF
:10B16000888784E08F8380E0DF91CF910895CF932B
:10B17000DF93EC018C819D810E945248E091EB3479
:10B18000F091EC3494E0899FE00DF11D1124458D80
:10B19000568D678D70A149875A876B877C878C8114
:10B1A0009D81FC01EE0FFF1FE80FF91FEE0FFF1F3F
:10B1B000EE0FFF1FEE0FFF1FE255FA4E859194919F
:10B1C000888784E08F8380E0DF91CF910895CF93CB
:10B1D000DF93EC010E948B5D49856FEE73E1CE0138
:10B1E000DF91CF910C942657CF93DF93EC018C81A4
:10B1F0009D810E945248833054F48F3F91F407C0E0
:10B20000CE010E94645E80E016C08DE614C04985C0
:10B210005A856B857C854430510561057105A8F719
:10B22000EFCF49855A856B857C8543305105610593
:10B23000710558F7E5CFDF91CF91089595E3899F88
:10B24000F0011124E157FC4C60817181828193816E
:10B250000895CF92DF92EF92FF92CF93DF936A012E
:10B260007B0125E3829FC001112486549D4CFC0183
:10B27000EB52FF4F4083518362837383EC01C352CF
:10B28000DF4F20E034E244E759E4C701B6010E94F1
:10B2900061D79B01AC0160E070E080E89FE30E9411
:10B2A000C3D4688379838A839B83DF91CF91FF9096
:10B2B000EF90DF90CF900895CF92DF92EF92FF92C0
:10B2C000CF93DF93EC01C984DA84EB84FC8420E023
:10B2D00034E244E759E4C701B6010E94BFD618160C
:10B2E00064F420E034E244E759E4C701B6010E9467
:10B2F000C3D469877A878B879C87CE010E947C6341
:10B30000C984DA84EB84FC848C819D810E9452483C
:10B3100025E3829FC001112486549D4CFC01EB5211
:10B32000FF4FC082D182E282F382EC01C352DF4F31
:10B3300020E034E244E759E4C701B6010E9461D736
:10B340009B01AC0160E070E080E89FE30E94C3D401
:10B35000688379838A839B8380E0DF91CF91FF901C
:10B36000EF90DF90CF900895CF92DF92EF92FF920F
:10B37000CF93DF93EC01C984DA84EB84FC8420E072
:10B3800034E244E759E4C701B6010E94BFD618165B
:10B3900064F420E034E244E759E4C701B6010E94B6
:10B3A000C3D469877A878B879C87CE010E947C6390
:10B3B00080E0DF91CF91FF90EF90DF90CF900895E4
:10B3C00081E08093E53480E00895FC0181859285D9
:10B3D000A385B4850197A105B10511F40E94366BD0
:10B3E00080E008956091E7347091E8348091E93409
:10B3F0009091EA3408950E943C5F80E00E94B96D0C
:10B4000080E008950E943C5F81E00E94B96D80E079
:10B4100008950E943C5F82E00E94B96D80E008952B
:10B420000E943C5F83E00E94B96D80E00895CF9355
:10B43000DF93EC01E091EB34F091EC34E55BFF4FEE
:10B44000E081F0E0EE0FFF1FEE5DFB4E6591749121
:10B450004FE450E086E69FE30E94F6E0AC0161EF26
:10B460007FE0CE01DF91CF910C94CEC0CF93DF93DC
:10B47000EC01E091EB34F091EC34E55BFF4FE081BF
:10B48000F0E0EE0FFF1FEE5DFB4E659174914FE40F
:10B4900050E086E69FE30E94F6E0AC0169ED7FE0B4
:10B4A000CE01DF91CF910C94CEC0CF93DF93EC010E
:10B4B00081EF90E20E9457E2CE010E94175ACE011E
:10B4C0000E94365A66EC7FE0CE010E94FAC06DEA17
:10B4D0007FE0CE010E9444C064E97FE0CE010E947B
:10B4E00044C06BE77FE0CE010E9444C062E67FE08B
:10B4F000CE010E9444C069E47FE0CE010E9444C0B6
:10B5000060E37FE0CE010E9444C067E17FE0CE01AE
:10B510000E9444C06EEF7EE0CE010E9444C065EE02
:10B520007EE0CE010E9444C06CEC7EE0CE010E9421
:10B5300044C063EB7EE0CE010E9444C06AE97EE035
:10B54000CE010E9444C061E87EE0CE010E9444C06A
:10B5500068E67EE0CE010E9472C080E0DF91CF916C
:10B56000089566EC7FE00C94FAC06DEA7FE00C94DD
:10B5700044C064E97FE00C9444C06BE77FE00C9426
:10B5800044C062E67FE00C9444C069E47FE00C9420
:10B5900044C060E37FE00C9444C067E17FE00C941A
:10B5A00044C06EEF7EE00C9444C065EE7EE00C94E7
:10B5B00044C06CEC7EE00C9444C063EB7EE00C94E1
:10B5C00044C06AE97EE00C9444C061E87EE00C94DB
:10B5D00044C068E67EE00C9472C06CEE7DE00C9492
:10B5E00072C06BEB7DE00C9472C066E87DE00C9459
:10B5F00072C06BE47DE00C9472C067E17DE00C9456
:10B6000072C0CF93DF93EC01E091EB34F091EC3416
:10B61000E55BFF4FE081F0E0EE0FFF1FEE5DFB4EBC
:10B62000659174914FE450E086E69FE30E94F6E056
:10B63000AC0163EF7CE0CE01DF91CF910C94CEC0E2
:10B64000CF93DF93EC01E091EB34F091EC34E55BC8
:10B65000FF4FE081F0E0EE0FFF1FEE5DFB4E6591C6
:10B6600074914FE450E086E69FE30E94F6E0AC015F
:10B6700062ED7CE0CE01DF91CF910C94CEC065EB02
:10B680007CE00C94FAC0CF93DF93EC01E091EB34B3
:10B69000F091EC34E55BFF4FE081F0E0EE0FFF1F2F
:10B6A000EE5DFB4E659174914FE450E086E69FE3BA
:10B6B0000E94F6E0AC0166E97CE0CE01DF91CF911B
:10B6C0000C94CEC00F931F93CF93DF93CDB7DEB70B
:10B6D000C058D109CDBFDEBF8C01DC011996EC91B9
:10B6E000F0E0EE0FFF1FE151FC4E659174914FE4C5
:10B6F00050E086E69FE30E94F6E09801235F3F4F0B
:10B700009F938F93F80181851F928F933F932F937F
:10B710000F5E1F4F1F930F933F932F938AE79CE079
:10B720009F938F938E010F5F1F4F1F930F930E9464
:10B73000ADE2C8010E941FC0CDBFDEBFC058DF4FC1
:10B74000CDBFDEBFDF91CF911F910F91089562E5CC
:10B750007CE00C94C4486AE27CE00C94C44868E045
:10B760007CE00C94C44866EE7BE00C94C44864EB27
:10B770007BE00C94C44863E87BE00C94C4486AE422
:10B780007BE00C94C4486AE27BE00C94C44868EE09
:10B790007AE00C94924866EA7AE00C9492486FE75B
:10B7A0007AE00C94C44869E57AE00C94C44868E3F4
:10B7B0007AE00C94C44868E17AE00C94C4486BEFDA
:10B7C00079E00C9428496CED79E00C942849BC018F
:10B7D000675F7F4F2091383542E55EE0FC01848150
:10B7E00095810C948F49BC01675F7F4F21E048E34E
:10B7F0005EE0FC01848195810C948F49BC01675FF8
:10B800007F4F21E04FE15EE0FC01848195810C9443
:10B810008F490F931F93CF93DF93EC010C811D8110
:10B820000E94E96408171907C4F48C819D81FC010A
:10B83000EE0FFF1FE80FF91FEE0FFF1FEE0FFF1FA8
:10B84000EE0FFF1FED54FA4E25913491CE01F90110
:10B85000DF91CF911F910F91199485E1DF91CF91E5
:10B860001F910F9108950F931F93CF93DF93EC01D6
:10B870000C811D810E94E96408171907C4F48C81AA
:10B880009D81FC01EE0FFF1FE80FF91FEE0FFF1F58
:10B89000EE0FFF1FEE0FFF1FEF54FA4E259134916C
:10B8A000CE01F901DF91CF911F910F91199485E19C
:10B8B000DF91CF911F910F9108950F931F93CF9315
:10B8C000DF93EC010C811D810E94E96408171907C0
:10B8D000C4F48C819D81FC01EE0FFF1FE80FF91F5E
:10B8E000EE0FFF1FEE0FFF1FEE0FFF1FE155FA4E89
:10B8F00025913491CE01F901DF91CF911F910F91E4
:10B900001994DF91CF911F910F910895CF93DF93F9
:10B91000EC018C819D810E94FC648823C9F08C819C
:10B920009D81FC01EE0FFF1FE80FF91FEE0FFF1FB7
:10B93000EE0FFF1FEE0FFF1FE355FA4EE491E1FFFC
:10B9400005C0CE01DF91CF910C94C98180E001C088
:10B9500085E1DF91CF910895AF92BF92CF92DF92B0
:10B96000EF92FF920F931F93CF93DF93EC0181E04F
:10B970000E94124F1C821D8280E090E07E0121E136
:10B98000E20EF11C54E0A52E62E0B62E51C00C81EF
:10B990001D816801CC0CDD1C9601200F311F220F88
:10B9A000331F220F331F220F331F23553A4EF90145
:10B9B000849180FF38C0F601E00FF11FEE0FFF1FEA
:10B9C000EE0FFF1FEE0FFF1FE954FA4E65917591C0
:10B9D0008591949169877A878B879C87F901249157
:10B9E00024FD08C00E9430D569877A878B879C87A1
:10B9F000BF8201C0AF82B601600F711F660F771F53
:10BA0000660F771F660F771F69557A4E45E050E045
:10BA1000C7010E94F6E0CE010E94095CCE010E949F
:10BA2000865C0C811D810F5F1F4F0C831D83C80135
:10BA30000E94EC648111ABCF81E00E94E7A8DF9106
:10BA4000CF911F910F91FF90EF90DF90CF90BF901B
:10BA5000AF900C94CFA8CF92DF92EF92FF92CF934A
:10BA6000DF93EC01C984DA84EB84FC8481E0C8169E
:10BA7000D104E104F10449F0CE01DF91CF91FF90B0
:10BA8000EF90DF90CF900C944E7ACE010E94AC5C88
:10BA900082E08F83C986DA86EB86FC8680E0DF91C0
:10BAA000CF91FF90EF90DF90CF90089580912C3C44
:10BAB00090912D3C8F3E924111F08AE5089580913E
:10BAC0006E3C90916F3C8F3E9241B9F78091FE366B
:10BAD0009091FF368F3E924181F78091243A909168
:10BAE000253A8F3E924149F78091263A9091273A24
:10BAF0008F3E924111F780912A3C90912B3C8F3ED2
:10BB00009241D9F68091B53F8111D7CF0895FC01BC
:10BB1000178289E60895CF93DF93DC0114968D9107
:10BB20009C911597FC01EE0FFF1FE80FF91FEE0F18
:10BB3000FF1FEE0FFF1FEE0FFF1FEB54FA4EC591D4
:10BB4000D491488150E060E070E019964D935D9388
:10BB50006D937C931C9782E017968C9380E0DF9125
:10BB6000CF910895CF93DF93DC0114968D919C9132
:10BB70001597FC01EE0FFF1FE80FF91FEE0FFF1FD7
:10BB8000EE0FFF1FEE0FFF1FEB54FA4EC591D4913D
:10BB90004881598160E070E019964D935D936D93F3
:10BBA0007C931C9782E017968C9380E0DF91CF9175
:10BBB0000895CF93DF93DC0114968D919C91159796
:10BBC000FC01EE0FFF1FE80FF91FEE0FFF1FEE0F36
:10BBD000FF1FEE0FFF1FEB54FA4EC591D491488121
:10BBE00059816A817B8119964D935D936D937C9306
:10BBF0001C9782E017968C9380E0DF91CF91089597
:10BC0000CF93DF93DC0114968D919C911597FC01E5
:10BC1000EE0FFF1FE80FF91FEE0FFF1FEE0FFF1FC4
:10BC2000EE0FFF1FEB54FA4EC591D4914881598114
:10BC30006A817B8119964D935D936D937C931C97DC
:10BC400083E017968C9380E0DF91CF910895CF9396
:10BC5000DF93DC0114968D919C911597FC01EE0FFA
:10BC6000FF1FE80FF91FEE0FFF1FEE0FFF1FEE0F74
:10BC7000FF1FEB54FA4EC591D491488159816A81D6
:10BC80007B8119964D935D936D937C931C97FC017A
:10BC9000EE0FFF1FE80FF91FEE0FFF1FEE0FFF1F44
:10BCA000EE0FFF1FE255FA4E8591949118968C93F2
:10BCB000189784E017968C9380E0DF91CF910895D8
:10BCC00088E6089580E00895FC0124813581F9011A
:10BCD000EE0FFF1FE20FF31FEE0FFF1FEE0FFF1F10
:10BCE000EE0FFF1FEB54FA4EA591B491FC01818534
:10BCF0008C9380E00895FC0124813581F901EE0FD9
:10BD0000FF1FE20FF31FEE0FFF1FEE0FFF1FEE0FDF
:10BD1000FF1FEB54FA4EA591B491FC0181859285E9
:10BD20008D939C9380E00895CF93DF93FC01248151
:10BD30003581F901EE0FFF1FE20FF31FEE0FFF1F1A
:10BD4000EE0FFF1FEE0FFF1FEB54FA4EC591D4917B
:10BD5000FC0181859285A385B48588839983AA8314
:10BD6000BB8380E0DF91CF910895FC01418552852E
:10BD7000638574854230510561057105A0F48481A5
:10BD80009581FC01EE0FFF1FE80FF91FEE0FFF1F5B
:10BD9000EE0FFF1FEE0FFF1FEB54FA4EA591B4916B
:10BDA0004C9380E008958EE60895FC01418552850C
:10BDB000638574854330510561057105A0F4848164
:10BDC0009581FC01EE0FFF1FE80FF91FEE0FFF1F1B
:10BDD000EE0FFF1FEE0FFF1FEB54FA4EA591B4912B
:10BDE0004C9380E008958EE60895FC0141855285CC
:10BDF000638574854430510561057105A0F4848123
:10BE00009581FC01EE0FFF1FE80FF91FEE0FFF1FDA
:10BE1000EE0FFF1FEE0FFF1FEB54FA4EA591B491EA
:10BE20004C9380E008958EE60895CF93DF93DC0174
:10BE300014968D919C911597FC01EE0FFF1FE80F52
:10BE4000F91FEE0FFF1FEE0FFF1FEE0FFF1FEB544A
:10BE5000FA4EC591D49119964D915D916D917C9159
:10BE60001C97488359836A837B8383E017968C935E
:10BE700080E0DF91CF910895CF93DF93DC0114969A
:10BE80008D919C911597FC01EE0FFF1FE80FF91F94
:10BE9000EE0FFF1FEE0FFF1FEE0FFF1FEB54FA4ECA
:10BEA000C591D49119964D915D916D917C911C979E
:10BEB000488359836A837B83FC01EE0FFF1FE80FE1
:10BEC000F91FEE0FFF1FEE0FFF1FEE0FFF1FE255D2
:10BED000FA4E8591949118968C93189784E0179652
:10BEE0008C9380E0DF91CF9108951F93CF93DF93E0
:10BEF000EC018091843C8823D1F01DE10A80DB8134
:10BF0000C02D209711F480E013C08F818F3FD9F3AB
:10BF1000811104C0CE010E94335C06C0CE010E9494
:10BF2000095CCE010E94865C115041F7ECCF85E69A
:10BF3000DF91CF911F910895CF93DF93EC01BC0166
:10BF40008FEF90E20E942FE1892B41F0BE0182E049
:10BF500091E20E942FE121E0892B09F420E0822F59
:10BF6000DF91CF91089541E0209100373091013762
:10BF70002817390709F040E0842F08950F931F9385
:10BF8000CF93DF93CDB7DEB72997CDBFDEBF8B014F
:10BF900044E050E0BC01CE0101960E944FE146E032
:10BFA00050E0B801CE0101960E943FE10E94E96491
:10BFB000181619060CF03FC07981AA81BB811C813B
:10BFC0000D8127EA35E140E050E0F9016491671303
:10BFD00027C03196E491E11103C0A11121C029C00D
:10BFE000EA131EC0F9013296E491E11103C0B111C8
:10BFF00017C01FC0EB1314C0F9013396E491E1118F
:10C0000003C011110DC015C0E1130AC0F901349627
:10C01000E491E11103C0011103C00BC0E01749F026
:10C020004F5F5F4F285E3F4F4817590709F0CDCF4C
:10C0300002C0CA0102C08FEF9FEF2996CDBFDEBFBD
:10C04000DF91CF911F910F910895CF93DF93FC0162
:10C050002189222371F1EC016196BE0186E091E213
:10C060000E942FE1892B39F1BE018FEF90E20E94EF
:10C070002FE1892B11F1BE0189E091E20E942FE1AD
:10C08000892BD9F0BE018DEE90E20E942FE1892B21
:10C09000B1F0BE018CE091E20E942FE1892B79F092
:10C0A000BE0188EE91E20E942FE1892B51F485E0D8
:10C0B00009C080E007C082E005C083E003C084E0DF
:10C0C00001C081E0DF91CF910895FC018FEF87835C
:10C0D0001482158211861286138614861086118AA0
:10C0E0001586178A108EA081B181109711F41682DF
:10C0F0000DC017968C911797873029F416968C915E
:10C100008F5F868303C016968C918683CF01089536
:10C11000EF92FF920F931F93CF93DF93EC010C816B
:10C120001D810E94E964081719070CF06FC00C818B
:10C130001D81CE010E9465600C831D837E0181E11B
:10C14000E80EF11CB801660F771F600F711F660FB4
:10C15000771F660F771F660F771F69557A4EC701E5
:10C160000E94D7E08E01035F1F4F2C813D81B901F2
:10C17000660F771F620F731F660F771F660F771F9B
:10C18000660F771F6D557A4EC8010E94D7E08D85E6
:10C19000882311F18C819D81FC01EE0FFF1FE80FB8
:10C1A000F91FEE0FFF1FEE0FFF1FEE0FFF1FE355EE
:10C1B000FA4EE491E2FF02C01D8610C0F801019022
:10C1C0000020E9F7BF01601B710B605F7F4F6C0FB0
:10C1D0007D1FC7010E9438E18C819D81FC01EE0F1B
:10C1E000FF1FE80FF91FEE0FFF1FEE0FFF1FEE0FEF
:10C1F000FF1FEF54FA4E25913491CE01F901DF91E2
:10C20000CF911F910F91FF90EF901994DF91CF91F3
:10C210001F910F91FF90EF9008958F929F92AF9290
:10C22000BF92CF92DF92EF92FF920F931F93CF9323
:10C23000DF9300D01F92CDB7DEB76C015C0181E1C6
:10C24000A80EB11C87E0F601878363EAE62E65E15C
:10C25000F62E00E010E01DC0B701CE0101960E944D
:10C26000D7E0BE016F5F7F4FC5010E942FE1892B90
:10C2700059F44601F9E18F0E911CF601058F168FD6
:10C28000C4010E94886064010F5F1F4FF8E1EF0E48
:10C29000F11CC8010E94EC648111DECF2496CDBF51
:10C2A000DEBFDF91CF911F910F91FF90EF90DF9054
:10C2B000CF90BF90AF909F908F900895CF93DF93D2
:10C2C0001092283A1092293A21E0FC013081311174
:10C2D00001C020E0ABEEB6E3E4E0F7E33FEFA0837C
:10C2E000B18379965B96ED93FC935C975D961D9276
:10C2F0001C925E97EF0163972883229618822197FC
:10C3000038832A96188259964AE3E432F40739F7BB
:10C3100010920D3A10920E3A10920437109205378F
:10C32000FC012081222369F010920A3727E0209334
:10C330000B37BC0185E197E30E9438E18DE197E37B
:10C3400002C084E097E3DF91CF910895EF92FF92CE
:10C350000F931F93CF93DF938AE091E20E945E6177
:10C36000EC018FEE92E180932C3C90932D3C8093D6
:10C370006E3C90936F3C8093FE369093FF36809393
:10C38000243A9093253A8093263A9093273A8093C3
:10C390002A3C90932B3C81E00E94124F1C821D820C
:10C3A000CE010E94A0812091763C3091773C409153
:10C3B000783C5091793C69857A858B859C850E9473
:10C3C00013D39F772CEA35EC47E257E30E94BFD6A0
:10C3D000181624F4CE010E94AC5C58C00E94D4A868
:10C3E0001C821D8280E090E08E010F5E1F4F42E0B4
:10C3F000E42E54E0F52E44C06C817D81CB01880F82
:10C40000991FFC01E60FF71FEE0FFF1FEE0FFF1F36
:10C41000EE0FFF1FE355FA4EE491E0FF2CC0680FCA
:10C42000791F660F771F660F771F660F771F695595
:10C430007A4E45E050E0C8010E94F6E0CE010E942D
:10C44000A0818C819D81FC01EE0FFF1FE80FF91F79
:10C45000EE0FFF1FEE0FFF1FEE0FFF1FE355FA4E0B
:10C46000E491E4FF02C0FF8201C0EF82CE010E948E
:10C47000095C6C817D816F5F7F4F6C837D83CB0115
:10C480000E94EC648111B8CF0E94E7A860E171E2DC
:10C4900087E493E20E94BE5F809300379093013758
:10C4A00064E171E287E493E20E94BE5F8093023709
:10C4B00090930337DF91CF911F910F91FF90EF90F1
:10C4C0000895EF92FF920F931F93CF93DF938C0108
:10C4D0002091283A3091293AEB0109900020E9F7A0
:10C4E0002197C61BD70BAE01420F531F413052405C
:10C4F000D8F4F901E65DF54C7F01AE014F5F5F4F67
:10C50000CF010E9410E14091283A5091293A4F5FA3
:10C510005F4F4C0F5D1F4093283A5093293AF80122
:10C52000E78AF08E80E001C08DE0DF91CF911F910E
:10C530000F91FF90EF900895CF93DF932EE1CDE11F
:10C54000D7E33F813F3F59F00A80DB81C02D209720
:10C5500019F480E090E010C0215099F7FACFBC01A7
:10C5600087E493E20E94BE5F8C839D83019689F3EA
:10C57000CE010E948860CE01DF91CF910895EF92A5
:10C58000FF920F931F93CF93DF938B012EE1CDE1A9
:10C59000D7E33F813F3F59F00A80DB81C02D2097D0
:10C5A00019F480E090E01DC0215099F7FACF7E0188
:10C5B00021E1E20EF11C45E050E0BC01C7010E9400
:10C5C0004FE1B801CE010E9461628111EACFB7014B
:10C5D00087E493E20E94BE5F8C839D8385E08F8316
:10C5E000CE01DF91CF911F910F91FF90EF900895B1
:10C5F0002091843C213021F42091623F213029F4A4
:10C60000BC018DEE90E20C94BF6280E090E0089552
:10C610009091843C913019F4642F0C944D800C94CB
:10C6200017C0CF93DF93EC018091773281110BC05B
:10C630000E9452D1482F50E060E070E049875A874D
:10C640006B877C870AC00E9460C8482F50E060E07A
:10C6500070E049875A876B877C8782E08F8380E010
:10C66000DF91CF9108950F931F93CF93DF93CDB7B1
:10C67000DEB7C058D109CDBFDEBFDC011996EC9101
:10C680008FEF8E0F863030F088E491E20E94F862DE
:10C690008EE629C0E093723281E080937332F0E03D
:10C6A000EE0FFF1FE259FA4E659174914FE450E08E
:10C6B00086E69FE30E94F6E09F938F9385E394E1E3
:10C6C0009F938F938E010F5F1F4F1F930F930E94B5
:10C6D000ADE2C8010E94F8620F900F900F900F908A
:10C6E0000F900F9080E0C058DF4FCDBFDEBFDF91CD
:10C6F000CF911F910F9108950F931F93CF93DF93C5
:10C70000EC018DEE94E30E94CA4A882329F0098542
:10C710001A858B859C8511C023E333E34BEC51E4F0
:10C7200069857A858B859C850E9461D78B01AB01D9
:10C73000BC0149875A876B877C872C813D81F90131
:10C74000EE0FFF1FE20FF31FEE0FFF1FEE0FFF1F95
:10C75000EE0FFF1FEB54FA4EA591B491A801BC0156
:10C760004D935D936D937C931397F901EE0FFF1F2B
:10C77000E20FF31FEE0FFF1FEE0FFF1FEE0FFF1F65
:10C78000E255FA4E85919491888784E08F8380E00A
:10C79000DF91CF911F910F9108956FE375E10C9494
:10C7A000FAC06BE175E10C94FAC06FED74E10C9482
:10C7B000FAC06BEA74E10C94FAC06EE574E10C9473
:10C7C000FAC01F93CF93DF93EC0110E08881882398
:10C7D00011F18AE091E20E945E6145E050E0BE0105
:10C7E0008EE297E30E944FE16EE277E387E493E203
:10C7F0000E94BE5F80932137909322378DE197E3AB
:10C800000E94886042E063E080E00E9408631F5F4E
:10C8100026961D31D9F684E0DF91CF911F910895BE
:10C82000CF93DF93CDB7DEB7EC97CDBFDEBF8CE300
:10C83000E8E1F0E2DE01119601900D928A95E1F7B0
:10C84000CE0101960E94E163EC96CDBFDEBFDF9181
:10C85000CF910895CF93DF93CDB7DEB7AA97CDBF21
:10C86000DEBF8AE2E4E5F0E2DE01119601900D926E
:10C870008A95E1F7CE0101960E94E163AA96CDBFA9
:10C88000DEBFDF91CF910895CF93DF93CDB7DEB7B1
:10C890006E97CDBFDEBF8EE1EEE7F0E2DE011196CE
:10C8A00001900D928A95E1F7CE0101960E94E16315
:10C8B0006E96CDBFDEBFDF91CF910895CF93DF930A
:10C8C000EC0143E759E763E770E0498B5A8B6B8BC8
:10C8D0007C8B0E940D6142E063E080E00E9408636F
:10C8E000CE010E944464CE010E942A6420E731E315
:10C8F00040E0298B3A8B4B8BCE010E940D6142E0C8
:10C9000063E080E00E940863CE01DF91CF910C9438
:10C910001064FC0181859285A385B48583309105DF
:10C92000A105B105A0F480937632892B8A2B8B2B3D
:10C9300039F064E070E080E00E9439C680E008953C
:10C9400068E070E080E00E9439C680E008958EE6DD
:10C950000895FC0181859285A385B4858230910577
:10C96000A105B105A0F480937532892B8A2B8B2BFE
:10C9700039F060E170E080E00E9439C680E00895FF
:10C9800060E270E080E00E9439C680E008958EE6A3
:10C990000895FC0181859285A385B4858230910537
:10C9A000A105B105A0F480937432892B8A2B8B2BBF
:10C9B00039F060E470E080E00E9439C680E00895BC
:10C9C00060E870E080E00E9439C680E008958EE65D
:10C9D000089582E991E0089521E08934914008F0BA
:10C9E00020E0822F08959C012556314081E02932B4
:10C9F000310508F080E0089521E08636914008F086
:10CA000020E0822F0895CF92DF92EF92FF92CF9392
:10CA1000DF93EC01C984DA84EB84FC84A7019601DE
:10CA2000C701B6010E9482D881113CC0E894F7F892
:10CA30002FEF3FEF4FE75FE7C701B6010E9482D8B3
:10CA400081110AC02FEF3FEF4FE75FE7C701B60143
:10CA50000E94BCD4181634F18C819D81FC01EE0F2C
:10CA6000FF1FE80FF91FEE0FFF1FEE0FFF1FEE0F66
:10CA7000FF1FE355FA4EE491E3FF14C08DEE94E3FB
:10CA80000E94CA4A81110EC025E832E441E25DE30A
:10CA900069857A858B859C850E9461D769877A87AD
:10CAA0008B879C87DF91CF91FF90EF90DF90CF90A5
:10CAB000089580917332882349F010927332609107
:10CAC000723280E00E9441C680E0089583E00895BC
:10CAD000CF93DF93E091A63CF091A73C04C0E09394
:10CAE000A63CF093A73CEF018191982F9D7F903257
:10CAF000B1F38930A1F34FE750E0BE018AEA9EE32B
:10CB00000E944FE11092A23C1092A33C1092A43CD0
:10CB10001092A53C6881611105C08091843C81110F
:10CB20006FC039C0613221F4DF91CF910C94B955B7
:10CB3000653221F4DF91CF910C94BD556E3721F40D
:10CB4000DF91CF910C94C1556F3379F4FE010190C0
:10CB50000020E9F73197EC1BFD0B329780F021960E
:10CB6000C093A63CD093A73C4BC06B3741F481E007
:10CB70008093843CCE01DF91CF910C94827D70E054
:10CB800088E791E20E9424E1892B59F01092843CBD
:10CB9000CE010E9409BE6AEA7EE3DF91CF910C9438
:10CBA00071BF8091843C811109C0CE010E948570C3
:10CBB0006AEA7EE3DF91CF910C9471BF8AE091E243
:10CBC0000E945E61EC0127E633E640E0298B3A8B58
:10CBD0004B8B6091A63C7091A73C0E94616285E0FE
:10CBE0008F838091A63C9091A73C0E94857042E083
:10CBF00060E00E94086380E0DF91CF910C9429AB44
:10CC0000DF91CF910895FF920F931F93CF93DF93FE
:10CC10001F921F92CDB7DEB7F82EE0E7FCE32CEBB6
:10CC200032E0DF01C9011D920197E9F72FEE32E1F1
:10CC30002083318320932A3F30932B3F0CE51FE262
:10CC40002CED33E40093763C1093773C2093783CB2
:10CC50003093793C0CEE11E528E73FE300937A3CF2
:10CC600010937B3C20937C3C30937D3C81E080930F
:10CC70007E3C83E08093853C8F2D4A8369830E94AC
:10CC800051C66981862F0E945CC64A81842F0E940A
:10CC900067C6F0927132F0926F320F900F90DF9171
:10CCA000CF911F910F91FF900895CF93DF931F9223
:10CCB0001F92CDB7DEB780E6F82E01E010E00E94AB
:10CCC0000C798230E1F30E9413798230C1F30E9423
:10CCD000A94A863009F0D9C00E9434C480908B3CA8
:10CCE00090908C3CA0908D3CB0908E3C8616970620
:10CCF000A806B90620F70E9434C46C597F4F8F4FA5
:10CD00009F4F60938B3C70938C3C80938D3C9093B1
:10CD10008E3C0E948278D3CF0E94EFBC882329F0FA
:10CD20008CEC0E94EB4E823051F20E9412568230FF
:10CD300031F20E943C9E823011F20E94565D809337
:10CD4000B63F81112EC08091703C9091713C8F3E16
:10CD5000924109F0AAC080912A3F90912B3F8F3ECB
:10CD6000924109F0A2C097C00E9436828093B63FDC
:10CD7000811117C00E945EB38093B63F811111C02C
:10CD80000E9450708093B63F81110BC00E9460C515
:10CD90008093B63F811105C00E9456B4823031F4B1
:10CDA0008ECF0E94EB4E8230B9F789CF0E945BABE9
:10CDB000823009F484CF0E94ADAC823009F47FCF79
:10CDC0000E9469AD823009F47ACF09831A8368EA38
:10CDD0007CE3CE0101960E9476C68093A63C909398
:10CDE000A73C8F3F2FEF920739F48DE00E94D44E7D
:10CDF000823009F464CF04C0892B11F00E94686569
:10CE00000E949B8C823009F45ACF0E94856B82303D
:10CE100009F455CF0E94446E823009F450CF0E942D
:10CE20002B70823009F449CF0E94784C823009F48B
:10CE300044CF0E94EB828430F0F53FCF8091853C57
:10CE4000843038F484E08093853C0E94BD550E9474
:10CE5000D9A883E090E089839A8368EA7CE3CE01D5
:10CE600001960E9476C68093A63C9093A73C8F3F84
:10CE70002FEF920721F48DE00E94D44E1ECF892B14
:10CE800009F41BCF0E94686518CF0E94A94A82301E
:10CE900009F44BCF41CF1092B63F0E94A64E80932B
:10CEA000B63F882309F460CF7CCFF092B63F80E68E
:10CEB0000E94EB4E78CF8091E4299091E5290E9461
:10CEC000C6CF682F70E080E090E00E945ED520E041
:10CED00030E048E451E40E94BFD687FFEECE0E94C6
:10CEE0005965823009F0AACFE8CE809171328093E3
:10CEF0006F32089580936F32089580937032089551
:10CF0000CF93C82F80919323882379F040E050E09D
:10CF1000BA018C2F0E946350EC2FFF27E7FDF0959C
:10CF2000EE53FB4C81E080830AC06C2F85EB98E5C3
:10CF30000E94EF4BAB01BC018C2F0E9463504091CB
:10CF4000BA235091BB236091BC237091BD238C2FD9
:10CF50000E9429598BE499E680939423909395231A
:10CF600082E0CF910895CF92DF92EF92FF920F93DC
:10CF70001F93CF93DF93CDB7DEB7E097CDBFDEBF72
:10CF800098E17E01A9E1EA0EF11CF701A92F1192A7
:10CF9000AA95E9F7FE0131966F0111929A95E9F78A
:10CFA000F60194E08902E00DF11D1124408F518FAC
:10CFB000628F738F80E090E0A0E8BFE3808391836D
:10CFC000A283B38300932A3510932B3520932C35FD
:10CFD00030932D350E946E830E94C155B601C70162
:10CFE0000E948B538093B63F811101C082E0E0968E
:10CFF000CDBFDEBFDF91CF911F910F91FF90EF90DA
:10D00000DF90CF9008950F931F93E0918D23FF271A
:10D01000E7FDF095E956FD4C9381913099F400912C
:10D020009E2310919F232091A0233091A123409112
:10D03000A6235091A7236091A8237091A9230E9451
:10D04000B3671DC0E0918E23FF27E7FDF095E956F9
:10D05000FD4C9381913099F400919E2310919F2370
:10D060002091A0233091A1234091A6235091A72382
:10D070006091A8237091A92370580E94B36789E436
:10D0800098E6809394239093952382E01F910F91CB
:10D0900008950F931F93CF93C82F85E3C802F00123
:10D0A0001124ED56FC4C40815181628173818C2F9B
:10D0B0000E94295900919E2310919F232091A02323
:10D0C0003091A12340919A2350919B2360919C23FE
:10D0D00070919D238C2F0E94B36788ED98E6809312
:10D0E00094239093952382E0CF911F910F910895FF
:10D0F0000F931F9300919E2310919F232091A023B3
:10D100003091A1234091AA235091AB236091AC238D
:10D110007091AD230E94B36780E897E680939423D3
:10D120009093952382E01F910F9108950E946E8342
:10D130008091B3230E94CC4F8091B2230E94124F62
:10D140008091B4230E94164F8091B5230E9477539B
:10D150008091B6239091B723A091B823B091B923C1
:10D1600080932A3590932B35A0932C35B0932D3591
:10D1700064E08DEE94E30E94E74A0E946E5610929E
:10D18000BE3480E00895CF93C82F4091BA235091C8
:10D19000BB236091BC237091BD230E9429598C2F21
:10D1A0000E94966880E00E9429AB80EFCF9108959D
:10D1B0000F931F93E0918D23FF27E7FDF095E9562C
:10D1C000FD4C9381913039F083EC98E68093942361
:10D1D0009093952318C00091A2231091A32320912E
:10D1E000A4233091A5234091A6235091A7236091B9
:10D1F000A8237091A9230E94B36788E798E68093DB
:10D2000094239093952382E01F910F910895FF92AC
:10D210000F931F93CF93DF93CDB7DEB7C058D109DB
:10D22000CDBFDEBFF82E8AE091E20E945E618EEFF4
:10D23000F81205C08DE791E20E94F86219C08F2DA7
:10D240000E9403571F928F9323E53BE33F932F9355
:10D250008E010F5F1F4F1F930F930E94ADE2C80115
:10D260000E94F8620F900F900F900F900F900F9008
:10D2700042E062E080EF0E9408638F2D0E94966872
:10D2800080EFC058DF4FCDBFDEBFDF91CF911F9140
:10D290000F91FF9008954F925F926F927F929F92AD
:10D2A000AF92BF92CF92DF92EF92FF920F931F93B4
:10D2B000CF93DF938F3F09F045C02CEA35EC47E26E
:10D2C00057E36091253670912636809127369091EC
:10D2D00028360E94BFD618160CF469C12CEA35EC2A
:10D2E00047E257E360911D3670911E3680911F36DC
:10D2F000909120360E94BFD618160CF45DC12CEA1E
:10D3000035EC47E257E360912136709122368091E7
:10D310002336909124360E94BFD618160CF455C1BE
:10D320002CEA35EC47E257E36091293670912A36B2
:10D3300080912B3690912C360E94BFD618160CF493
:10D340003FC171C18230A1F52CEA35EC47E257E3C9
:10D3500060911D3670911E3680911F369091203657
:10D360000E94BFD618160CF427C12CEA35EC47E210
:10D3700057E3609121367091223680912336909147
:10D3800024360E94BFD618160CF41FC12CEA35ECC7
:10D3900047E257E36091293670912A3680912B3607
:10D3A00090912C360E94BFD618160CF409C131C1D9
:10D3B0008823D9F2813051F32CC17E018DEEE80E25
:10D3C000F11CF70180819181A281B381BC01CD0163
:10D3D0009F772CEA35EC47E257E30E94BCD487FDE7
:10D3E00046C06E01F1EFCF0ED11CF6014080518096
:10D3F0006280738020E030E0A901C301B2010E9485
:10D40000BCD487FD34C0FE01EF52FF4F2081318133
:10D4100042815381349760817181828193810E941E
:10D4200013D39B01AC015F77C301B2010E9414D3F7
:10D430002B013C019F772CEA35EC47E257E30E9431
:10D44000BCD487FD14C0AB2CAA0C8A2D0E94E9BC69
:10D4500080938B23992493949A0C892D0E94E9BC84
:10D4600080938C2320918B23822780FD02C08B2DFB
:10D47000DBC0B0928A23F80180819181A281B381BF
:10D48000BF7780939E2390939F23A093A023B09374
:10D49000A123F70140815181628173817F7740939D
:10D4A000A2235093A3236093A4237093A52320FF6A
:10D4B0002DC0A0928D2390928E2377FA709477F8E6
:10D4C000709440929A2350929B2360929C23709276
:10D4D0009D23F60180819181A281B3818093A6234F
:10D4E0009093A723A093A823B093A923CB50DF4FF9
:10D4F00088819981AA81BB818093AA239093AB23D1
:10D50000A093AC23B093AD238A2D2AC090928D2393
:10D51000A0928E2340929A2350929B2360929C2348
:10D5200070929D23F60180819181A281B381B058D0
:10D530008093A6239093A723A093A823B093A92315
:10D54000CB50DF4F88819981AA81BB81B0588093ED
:10D55000AA239093AB23A093AC23B093AD23892D42
:10D560000E94E9BC8D7F813039F08BE499E680938D
:10D5700094239093952369C080918E230E94E9BCE7
:10D58000811103C08FEF80938E238B2D0E941E5933
:10D590006093BA237093BB238093BC239093BD23E5
:10D5A00083E098E680939423909395234EC082E085
:10D5B00090E032E0B32E0DC080E090E0B12C09C0C5
:10D5C00083E090E023E0B22E04C081E090E0BB2431
:10D5D000B394FC01EE53FB4C108225E3289FE0013D
:10D5E000299FD00D1124C654DD4C8E0107511F4FC9
:10D5F000F80180819181A281B381BC01CD019F7727
:10D600002CEA35EC47E257E30E94BCD487FFD5CE25
:10D610002ECF81E08093C13486E998E680939423ED
:10D620009093952312C08EEFDF91CF911F910F91B0
:10D63000FF90EF90DF90CF90BF90AF909F907F9042
:10D640006F905F904F900C94076982E0DF91CF91CB
:10D650001F910F91FF90EF90DF90CF90BF90AF9010
:10D660009F907F906F905F904F900895CF93DF933E
:10D67000CBEED4E3888199810E94CA4A8093B22379
:10D68000888199810E94C54A8093B32388819981BA
:10D690000E94D44A8093B423888199810E94D94AF8
:10D6A0008093B523888199810E94E04A6093B623D4
:10D6B0007093B7238093B8239093B92381E00E949D
:10D6C000124F81E00E94164F80E00E94CC4F81E013
:10D6D0000E94775381E0809393238FEF80938A2376
:10D6E0008BE499E6809394239093952383E0809331
:10D6F000BE341092C13480E0DF91CF9108950E9432
:10D70000366B1092932380E008958091BE3483306D
:10D7100059F40E94DE4A813049F0E0919423F0915F
:10D72000952380918A23199483E0089582E00895D7
:10D7300080EA9BE68093CF239093D02382E00895E4
:10D740002F923F924F925F926F927F928F929F9211
:10D75000AF92BF92CF92DF92EF92FF920F931F93FF
:10D76000CF93DF93CDB7DEB7CA54D109CDBFDEBFAB
:10D7700098E19E01275E3F4F29AB3AABD901E92FD3
:10D780001D92EA95E9F7285131091901D9011D9235
:10D790009A95E9F724E08202F00111242B96EEAF6E
:10D7A000FFAF2B97E20DF31D80E090E0A0E8BFE310
:10D7B00080839183A283B383C090C723D090C82372
:10D7C000E090C923F090CA234090C3235090C42313
:10D7D0006090C5237090C6238090BF239090C02393
:10D7E000A090C123B090C223A5019401C301B2014E
:10D7F0000E94BCD418165CF080E090E0A0E8BFE383
:10D8000029968CAF9DAFAEAFBFAF29970AC080E01D
:10D8100090E0A0E8BFEB29968CAF9DAFAEAFBFAF55
:10D820002997A3019201C501B4010E9413D30E945C
:10D830002BD59B0177FF04C022273327261B370BEC
:10D84000B901882777FD8095982F0E945ED525968F
:10D850006CAF7DAF8EAF9FAF2597C0922A35D09227
:10D860002B35E0922C35F0922D350E946E830E946C
:10D87000C15520E030E040E050E425966CAD7DAD30
:10D880008EAD9FAD25970E94BFD618166CF0809183
:10D89000CB239091CC23A091CD23B091CE238BAFFD
:10D8A0009CAFADAFBEAFDBC02AE037ED43E25CE337
:10D8B00025966CAD7DAD8EAD9FAD25970E94BFD6F0
:10D8C00018162CF709E110E08AE0882E87ED982ED3
:10D8D00083E2A82E8CE3B82E412C512C32012B96DA
:10D8E000AEADBFAD2B97A20DB31D58962196AEAF2E
:10D8F000BFAF21974BAA5CAA6DAA7EAA8FAA98AE49
:10D90000A9AEBAAE29962CAD3DAD4EAD5FAD29970F
:10D910006FA978AD89AD9AAD0E9461D79B01AC012A
:10D920006091C3237091C4238091C5239091C62335
:10D930000E9414D32196EEADFFAD219760837183D1
:10D9400082839383C0922A35D0922B35E0922C3576
:10D95000F0922D35B101CE0149960E948B538093F0
:10D96000B63F8111AAC020E030E040E85FE36BA938
:10D970007CA98DA99EA90E9414D36BAB7CAB8DAB07
:10D980009EAB20E030E048EC51E40E94C3D49B0100
:10D99000AC0160E070E080E291E40E94C4D72B010A
:10D9A0003C018091CB239091CC23A091CD23B091C9
:10D9B000CE238BAF9CAFADAFBEAFC090C723D0908E
:10D9C000C823E090C923F090CA23A7019601BC01A7
:10D9D000CD010E9413D34B015C0120E030E040E216
:10D9E00051E4C301B2010E94C3D49B01AC01C50143
:10D9F000B4010E9461D79B01AC01C701B6010E942E
:10DA000014D36B017C012BA93CA94DA95EA9CA01C5
:10DA1000B9010E9414D320E030E048EC51E40E94A8
:10DA2000C3D49B01AC016FA978AD89AD9AAD0E94BA
:10DA300014D36FAB78AF89AF9AAF9B01AC01259639
:10DA40006CAD7DAD8EAD9FAD25970E94BFD61816EB
:10DA500034F4015011090115110509F053CF8BADB4
:10DA60009CADADADBEAD80932A3590932B35A09380
:10DA70002C35B0932D352B96EEADFFAD2B97E20DE7
:10DA8000F31D8091BF239091C023A091C123B09139
:10DA9000C223808F918FA28FB38FB101CE0149969F
:10DAA0000E948B538093B63F811107C084E79DE6A7
:10DAB0008093CF239093D02382E0C65BDF4FCDBF0E
:10DAC000DEBFDF91CF911F910F91FF90EF90DF901C
:10DAD000CF90BF90AF909F908F907F906F905F900E
:10DAE0004F903F902F900895CF93DF931F92CDB723
:10DAF000DEB789830E946E834091D9235091DA2347
:10DB00006091DB237091DC2389810E9429598091E7
:10DB1000D6230E94CC4F8091D5230E94124F809132
:10DB2000D7230E94164F8091D8230E94775380916B
:10DB3000D1239091D223A091D323B091D423809369
:10DB40002A3590932B35A0932C35B0932D3564E076
:10DB50008DEE94E30E94E74A0E946E561092BE3406
:10DB600089EA91E20E9457E280E00F90DF91CF9125
:10DB700008950F931F93CF93C82F0BEE14E3F80172
:10DB8000808191810E94CA4A8093D523F8018081C7
:10DB900091810E94C54A8093D623F80180819181AA
:10DBA0000E94D44A8093D723F801808191810E94FA
:10DBB000D94A8093D823F801808191810E94E04A5C
:10DBC0006093D1237093D2238093D3239093D42353
:10DBD0008C2F0E941E596093D9237093DA2380936F
:10DBE000DB239093DC2381E00E94124F80E00E94AF
:10DBF000164F80E00E94CC4F81E00E94775340E0B6
:10DC000050E060E271E44093C7235093C8236093CF
:10DC1000C9237093CA2385E3C89FF0011124ED57EF
:10DC2000FC4C40815181628173814093CB2350939E
:10DC3000CC236093CD237093CE236C2F85EB98E596
:10DC40000E94DC4B6093C3237093C4238093C5234D
:10DC50009093C6230E94F2596093BF237093C02310
:10DC60008093C1239093C223C093BE2388E99BE68F
:10DC70008093CF239093D02384E08093BE3480E0C0
:10DC8000CF911F910F9108958091BE34843059F443
:10DC90000E94DE4A813049F0E091CF23F091D023F9
:10DCA0008091BE23199483E0089582E00895E09165
:10DCB000DF23F0E0E956FD4C8381882341F082E7C1
:10DCC0009EE68093DD239093DE2382E008956CE24C
:10DCD00074E284E194E20E948B538093B63F8823E0
:10DCE00071F308951F93CF93DF93E091DF23F0E06A
:10DCF000E956FD4C81E09381913009F080E08093FA
:10DD0000C834C9ECD4E310E0812F0E945C97AB01CA
:10DD1000BC01812F0E946350612F8091EB34909160
:10DD2000EC340E94DC4B69937993899399931F5F3C
:10DD3000163051F783EB91E20E94827D8EED9EE6D4
:10DD40008093DD239093DE2382E0DF91CF911F91BA
:10DD500008951F93CF93DF930E946E838091E023F9
:10DD600080939732E091DF23F0E08091E123E95640
:10DD7000FD4C83870E9406BDC4EED3E210E04991BA
:10DD8000599169917991812F0E9429591F5F16300D
:10DD9000B1F78091E3230E94CC4F8091E2230E944F
:10DDA000164F64E08DEE94E30E94E74A0E946E569F
:10DDB0001092BE34DF91CF911F9108950E94A96EF9
:10DDC00080E008950F931F93CF93DF93CDB7DEB715
:10DDD000C058D109CDBFDEBF182F8AE091E20E9462
:10DDE0005E611E3F29F480EC91E20E94F86219C046
:10DDF000812F0E9403571F928F9381E89BE39F938B
:10DE00008F938E010F5F1F4F1F930F930E94ADE200
:10DE1000C8010E94F8620F900F900F900F900F9022
:10DE20000F9042E062E08AEF0E9408630E94A96EB0
:10DE30008AEFC058DF4FCDBFDEBFDF91CF911F917A
:10DE40000F910895FF920F931F93CF93DF9310923A
:10DE5000C83482E08093BE3404EE13E2C3E9D3E316
:10DE6000F12C8F2D0E941E59F801619371938193BB
:10DE700091938F01488159816A817B818F2D0E9406
:10DE800029596F2D8091EB349091EC340E94DC4B3A
:10DE9000F801648B758B868B978BF394E596F6E08F
:10DEA000FF12DFCF64E174E28CEF93E20E9437C18E
:10DEB0002AE43CE042E85EE30E94BCD487FF03C052
:10DEC0008EEF0E94E26EC8E0D4E213E0699179918E
:10DED000899199912C893D894E895F890E9413D33C
:10DEE0009F772CEA35EC47E257E30E94BFD618161D
:10DEF0001CF4812F0E94E26E1F5F163039F784E018
:10DF00008093DF238091A6328093E12381E0809388
:10DF1000A632809197328093E023109297320E942C
:10DF200006BD8091EB349091EC340E94C54A8093F9
:10DF3000E3238091EB349091EC340E94D44A809397
:10DF4000E22380E00E94164F80E00E94CC4F80E0E8
:10DF50000E9438AF87E59EE68093DD239093DE2311
:10DF600082E0DF91CF911F910F91FF9008950F9361
:10DF70001F93CF93DF938C01EB018091363588237B
:10DF800099F080912A3590912B35A0912C35B09144
:10DF90002D35BC01CD019F772CEA35EC47E257E3E4
:10DFA0000E94BCD487FD4FC088819981AA81BB8122
:10DFB000BC01CD019F772CEA35EC47E257E30E9484
:10DFC000BFD61816F4F48C819D81AE81BF81BC014F
:10DFD000CD019F772CEA35EC47E257E30E94BFD68C
:10DFE00018167CF488859985AA85BB85BC01CD016E
:10DFF0009F772CEA35EC47E257E30E94BFD618160C
:10E0000024F188E1F801A4E1B4E201900D928A952F
:10E01000E1F788E1FE01ACE2B4E201900D928A954D
:10E02000E1F788E1E9ECF4E3DF011D928A95E9F775
:10E0300082E08093C83482E29FE68093DD23909350
:10E04000DE2380E003C08EE801C086E8DF91CF9137
:10E050001F910F9108958091BE34823021F08091FC
:10E06000C834823049F40E94DE4A813039F0E091B0
:10E07000DD23F091DE23199483E0089582E0089572
:10E08000ECE2FFE380E2DF011D928A95E9F78FEE73
:10E0900092E180934A3F90934B3F80839183089510
:10E0A00080914A3F90914B3F8F3E924111F08CE519
:10E0B000089580912C3F90912D3F8F3E9241B9F76A
:10E0C00080E00895CF93DF93C82FCB01BA010E945F
:10E0D00010D827E0C29FE0011124C45DD04C0E94FB
:10E0E0002BD56D837E838F839887DF91CF910895A1
:10E0F00097E0899FF0011124E45DF04C6581768101
:10E10000878190850E945ED508952F923F924F920D
:10E110005F926F927F928F929F92AF92BF92CF92B7
:10E12000DF92EF92FF920F931F93CF93DF93CDB7C0
:10E13000DEB72797CDBFDEBF8C011B828091BD3437
:10E14000823009F440C7D801BC90B11069C780E0A3
:10E150006E01B3E0CB0ED11C3DC0F6018081811170
:10E1600008C0B72CD7011C926E01B3E0CB0ED11CB6
:10E1700054C7883239F4B72CF7011082FFEFCF1A59
:10E18000DF0A4BC78B33B9F3A82EB12CC5010E940F
:10E19000ABE0892B39F4B5018AEE91E20E9424E1CB
:10E1A000892B51F047018FEF881A980AC5010E9408
:10E1B000CFE0D7018C937401BFEFCB1ADB0AF701D4
:10E1C00080818111CACFB72CD8018C916E01B3E048
:10E1D000CB0ED11CF8011CC08E32E1F090E0C0974C
:10E1E0000A97A0F08181803391F4228130E020539E
:10E1F00031092A30310558F4DF01119611968C91BE
:10E2000011978D938111FACF808102C0818131965F
:10E210008111E2CFF601A080A11007C068C0D6012D
:10E220001196AC90BFEFCB1ADB0A76018A2C912CA9
:10E23000C4010E94BFE0892B91F7EBE7AE122FC01B
:10E24000D60111968C9190E00E94C7E08437910529
:10E2500031F5F601828190E00E94C7E08936910590
:10E26000F1F4D60113968C9190E00E94C7E08436B9
:10E270009105A9F4BE016F5F7F4FC60105960E940C
:10E2800027DD0E9430D56093A23C7093A33C80931D
:10E29000A43C9093A53CF601A0808A2C912CC4014B
:10E2A0000E94C7E08D369105A1F4D60111968C919C
:10E2B00090E00E94C7E08337910559F4F60182810E
:10E2C00090E00E94C7E08736910519F4F601339675
:10E2D00002C0FE013396AA2061F08A2DD70189324F
:10E2E00009F41C9211968C918111F9CF02C0FE01A4
:10E2F00033968FE2B81609F468C68081882319F036
:10E30000CF010E94B45580E1ECE4FFE3DF011D92F0
:10E310008A95E9F78BE5E6E1F6E3DF01982F1D9298
:10E320009A95E9F7EBEBF5E3DF011D928A95E9F7A2
:10E330008DEE94E30E94C24A8093BC35812C912CCF
:10E3400080E8A82E8FE3B82E5524539492E0492EEE
:10E3500024E0322E23C4C701B6010E9430D5862F97
:10E3600090E08F35910508F034C6FC01EC50FF4F6A
:10E370000C9407DD1092BC355092173680914D3FBA
:10E380008F5F80934D3F0AC45092BC355092173630
:10E3900080914D3F8F5F80934D3F00C44092BC35CC
:10E3A0005092173680914D3F8F5F80934D3FF6C35B
:10E3B00083E08093BC355092173680914D3F8F5F3C
:10E3C00080934D3FEBC38DE08093BB355092163662
:10E3D000E5C388E0B2C01092EB355092463680918A
:10E3E0004E3F8F5F80934E3FD9C35092EB35509292
:10E3F000463680914E3F8F5F80934E3FCFC3409211
:10E40000EB355092463680914E3F8F5F80934E3F62
:10E41000C5C31092EC35509247368091513F8F5FC3
:10E420008093513FBBC35092EC3550924736809158
:10E43000513F8F5F8093513FB1C3C701B6010E9426
:10E440007BD86C837D838E839F8320E030E040E225
:10E4500051E4C701B6010E9461D76B017C0120E045
:10E4600030E040E251E46C817D818E819F810E9489
:10E4700061D79B01AC01C701B6010E9413D30E9472
:10E4800030D5623001F128F4662341F0613089F023
:10E49000A0C56330E9F0643001F19BC5B5E0B093ED
:10E4A000BB355092163680914C3F8F5F80934C3F26
:10E4B00075C33092BB356093163680914C3F8F5FA9
:10E4C00080934C3F6BC35092BB355092163666C357
:10E4D0004092BB355092163661C383E08093BB35C2
:10E4E000509216365BC3C701B6010E947BD86C837D
:10E4F0007D838E839F8320E030E040E251E4C701BA
:10E50000B6010E9461D76B017C0120E030E040E25F
:10E5100051E46C817D818E819F810E9461D79B0136
:10E52000AC01C701B6010E9413D30E9430D5662307
:10E5300019F0613061F04DC587E08093BB35509292
:10E54000163680914C3F8F5F80934C3F27C3E6E0A7
:10E55000E093BB356093163680914C3F8F5F80937C
:10E560004C3F1CC3C701B6010E947BD86C837D83DE
:10E570008E839F8320E030E040E251E4C701B60182
:10E580000E9461D76B017C0120E030E040E251E461
:10E590006C817D818E819F810E9461D79B01AC013E
:10E5A000C701B6010E9413D30E9430D5623009F032
:10E5B00010C58EE08093BB3550921636EFC2509254
:10E5C000EE3550924936EAC25092ED3550924836B7
:10E5D0008091553F8F5F8093553FE0C24092ED356B
:10E5E000509248368091553F8F5F8093553FD6C2F9
:10E5F00083E016C03092ED35509248368091553FF9
:10E600008F5F8093553FCAC2F5E0F093ED3550928D
:10E6100048368091553F8F5F8093553FBFC286E05B
:10E620008093ED35509248368091553F8F5F8093AF
:10E63000553FB4C2C701B6010E947BD86C837D836D
:10E640008E839F8320E030E040E251E4C701B601B1
:10E650000E9461D76B017C0120E030E040E251E490
:10E660006C817D818E819F810E9461D79B01AC016D
:10E67000C701B6010E9413D30E9430D5662319F05A
:10E68000613059F0A6C41092F03550924B3680910B
:10E69000563F8F5F8093563F81C26093F035609301
:10E6A0004B368091563F8F5F8093563F77C24092A2
:10E6B000F03550924B368091563F8F5F8093563F96
:10E6C0006DC23092BC355092173680914D3F8F5FAE
:10E6D00080934D3F63C2C701B6010E947BD86C8313
:10E6E0007D838E839F8320E030E040E251E4C701C8
:10E6F000B6010E9461D76B017C0120E030E040E26E
:10E7000051E46C817D818E819F810E9461D79B0144
:10E71000AC01C701B6010E9413D30E9430D5662315
:10E7200019F0613059F055C41092F13550924C36C1
:10E7300080914F3F8F5F80934F3F30C21092F235F0
:10E7400060934D3680914F3F8F5F80934F3F26C23D
:10E75000C701B6010E947BD86C837D838E839F8323
:10E7600020E030E040E251E4C701B6010E9461D7E9
:10E770006B017C0120E030E040E251E46C817D815E
:10E780008E819F810E9461D79B01AC01C701B601B8
:10E790000E9413D30E9430D5662319F0613059F0DE
:10E7A00018C45092F13550924C3680914F3F8F5F94
:10E7B00080934F3FF3C16093F23560934D36809163
:10E7C0004F3F8F5F80934F3FE9C1C701B6010E9461
:10E7D0007BD86C837D838E839F8320E030E040E292
:10E7E00051E4C701B6010E9461D76B017C0120E0B2
:10E7F00030E040E251E46C817D818E819F810E94F6
:10E8000061D79B01AC01C701B6010E9413D30E94DE
:10E8100030D5613089F028F06230A1F06330C1F06A
:10E82000D8C399E09093BB355092163680914C3FF7
:10E830008F5F80934C3FB2C1AAE0A093BB35609339
:10E840001636ACC1BBE0B093BB3550921636A6C1AC
:10E85000ECE0E093BB3550921636A0C11092E6353D
:10E86000509241368091503F8F5F8093503F96C1C8
:10E870005092E635509241368091503F8F5F8093A1
:10E88000503F8CC1C701B6010E9430D5862F90E061
:10E890008D33910508F09BC3FC01ED5AFE4F0C949B
:10E8A00007DD1092BD35509218368091573F8F5F2B
:10E8B0008093573F73C15092BD3550921836809166
:10E8C000573F8F5F8093573F69C15092F835509200
:10E8D00053368091593F8F5F8093593F5FC140927B
:10E8E000F835509253368091593F8F5F8093593F4E
:10E8F00055C11092F835509253368091593F8F5F31
:10E900008093593F4BC15092F5355092503646C1D5
:10E910005092F6355092513680915A3F8F5F8093D6
:10E920005A3F3CC15092F7355092523680915A3F2F
:10E930008F5F80935A3F32C11092F7355092523612
:10E9400080915A3F8F5F80935A3F28C15092E9359A
:10E950005092443680915B3F8F5F80935B3F1EC136
:10E960001092E9355092443680915B3F8F5F8093DF
:10E970005B3F14C15092E7355092423680915B3F25
:10E980008F5F80935B3F0AC15092013650925C3694
:10E9900080915B3F8F5F80935B3F00C1C701B601F1
:10E9A0000E947BD80E9430D56093F43550924F3648
:10E9B000F5C0C092DA35D092DB35E092DC35F092CA
:10E9C000DD358092353690923636A0923736B09249
:10E9D0003836E4C0C0920236D0920336E092043654
:10E9E000F092053680925D3690925E36A0925F3648
:10E9F000B0926036D3C0C092F935D092FA35E09229
:10EA0000FB35F092FC358092543690925536A092A8
:10EA10005636B0925736C2C0C092C235D092C33576
:10EA2000E092C435F092C53580921D3690921E3624
:10EA3000A0921F36B0922036B1C0C092C635D09297
:10EA4000C735E092C835F092C93580922136909250
:10EA50002236A0922336B0922436A0C0C092CA3586
:10EA6000D092CB35E092CC35F092CD3580922536E0
:10EA700090922636A0922736B09228368FC0C09248
:10EA8000CE35D092CF35E092D035F092D13580920C
:10EA9000293690922A36A0922B36B0922C367EC020
:10EAA000C092D235D092D335E092D435F092D5359C
:10EAB00080922D3690922E36A0922F36B09230361C
:10EAC0006DC0C092D635D092D735E092D835F0924D
:10EAD000D9358092313690923236A0923336B09248
:10EAE00034365CC0C0920A36D0920B36E0920C36B7
:10EAF000F0920D368092653690926636A092673617
:10EB0000B09268364BC0C0920E36D0920F36E0926B
:10EB10001036F09211368092693690926A36A09241
:10EB20006B36B0926C363AC0C0921236D092133621
:10EB3000E0921436F092153680926D3690926E36D1
:10EB4000A0926F36B092703629C0C0920636D0922D
:10EB50000736E0920836F09209368092613690923C
:10EB60006236A0926336B092643618C0C701B6010F
:10EB70000E9430D56093BE357093BF358093C03509
:10EB80009093C13581E090E0A0E0B0E08093193629
:10EB900090931A36A0931B36B0931C36D8012C9054
:10EBA000222009F424C2822D90E00E94B6E0892B35
:10EBB00009F42FC23801BFEF6B1A7B0AF80181817B
:10EBC000803349F48281883531F40E5F1F4FC12CA8
:10EBD000D12C760100C2BE016F5F7F4FC3010E943E
:10EBE00027DD6B017C0109811A816016710609F02D
:10EBF000F2C111C28091E6350E947753182F01C0EF
:10EC000010E06091353670913636809137369091AC
:10EC100038360E9430D5662359F06091DA3570910C
:10EC2000DB358091DC359091DD350E944653182FFD
:10EC30006091393670913A3680913B3690913C36EE
:10EC40000E9430D5662371F06091DE357091DF351A
:10EC50008091E0359091E1350E9430D5862F0E9459
:10EC60002255182F60913D3670913E3680913F3687
:10EC7000909140360E9430D5662371F06091E23564
:10EC80007091E3358091E4359091E5350E9430D55F
:10EC9000862F0E946155182F609154367091553619
:10ECA00080915636909157360E9430D5662359F0A0
:10ECB0006091F9357091FA358091FB359091FC3572
:10ECC0000E946CAF182F6091583670915936809120
:10ECD0005A3690915B360E9430D5662371F0609170
:10ECE000FD357091FE358091FF35909100360E9480
:10ECF00030D5862F0E94A055182F80914F3688233B
:10ED000029F08091F4350E94DF53182F80915036FE
:10ED1000882329F08091F5350E941354182F809193
:10ED20005336882329F08091F8350E9438AF182F88
:10ED300080915136882329F08091F6350E944854FD
:10ED4000182F80915236882329F08091F7350E9440
:10ED50007C54182F80914236882329F08091E73522
:10ED60000E94F754182F80914336882329F0809110
:10ED7000E8350E943655182F80915C36882329F09B
:10ED8000809101360E947555182F80914436882352
:10ED900029F08091E9350E94EF54182F8091BB35FE
:10EDA0008D3029F0809146368823A9F00FC06091FC
:10EDB00002367091033680910436909105360E9498
:10EDC0007F538093B63F882369F32FC18091EB3541
:10EDD0000E940E4F182F80914736882329F080918A
:10EDE000EC350E94124F182F80914836882329F065
:10EDF0008091ED350E94CC4F182F80914B3688239F
:10EE000029F08091F0350E947B53182F80914C3669
:10EE1000882329F08091F1350E94164F182F4091D8
:10EE2000BB3550E04F30510508F0B6C0FA01E0574D
:10EE3000FE4F0C9407DD0E94C852182FADC06DE143
:10EE400076E382EC95E30E94D352182FA5C00E946E
:10EE50000753182FA1C06DE176E382EC95E30E9481
:10EE60001253182F99C00E94366B182F95C06DE170
:10EE700076E382EC95E30E949250182F8DC00E9499
:10EE80007F6B182F89C06DE176E382EC95E30E94D9
:10EE9000B76F182F81C06091023670910336809150
:10EEA0000436909105360E9430D5862F2DE136E349
:10EEB00042EC55E36091EA350E941A4F182F6CC05E
:10EEC0006DE176E382EC95E30E940F51182F64C048
:10EED0000E94C251182F60C00E942952182F5CC096
:10EEE0000E946052182F58C06091EE358DEE94E369
:10EEF0000E945D4B8091BC35843038F48230D8F468
:10EF0000882349F0813079F047C0843009F044C04B
:10EF10008093F13441C06DE176E382EC95E30E9489
:10EF20009852182F39C06DE176E382EC95E30E9488
:10EF30008B53182F31C0A0901236B0901336C0906A
:10EF40001436D0901536E0900E36F0900F360091C2
:10EF500010361091113620910A3630910B364091BF
:10EF60000C3650910D368F93809109368F93809196
:10EF700008368F93809107368F93809106368F9352
:10EF80006DE176E382EC95E30E94FE84182F0F90EA
:10EF90000F900F900F900F9060E08DEE94E30E9421
:10EFA0005D4B80911836813061F48091BD358111BF
:10EFB00004C00E94A156812F38C00E94D256812FD2
:10EFC00034C0812F32C08BEC30C083E02EC084E887
:10EFD0002CC083E82AC0822D90E0FC01E154F109A5
:10EFE000EA31F105B0F7E156FE4F0C9407DD1092BF
:10EFF000B63F6091BE357091BF358091C03590911C
:10F00000C1350E94F74A80914136882309F4F8CD32
:10F01000F1CD85E60AC086E608C0D8018C91DAC831
:10F0200068018B2D78017B2CA4C82796CDBFDEBF4D
:10F03000DF91CF911F910F91FF90EF90DF90CF90D4
:10F04000BF90AF909F908F907F906F905F904F9008
:10F050003F902F900895CF93DF93EC016AEA7EE30F
:10F060000E9461628093B63F811102C095E09F8348
:10F07000DF91CF910895FC018789908D0C94857064
:10F0800083FF06C0E0918F32F091903290E2958339
:10F0900082FF06C0E0919132F091923290E2958326
:10F0A00081FF06C0E0919332F091943290E2958313
:10F0B00080FF06C0E0919532F091963280E2858320
:10F0C000089583FF06C0E0918F32F091903290E274
:10F0D000968382FF06C0E0919132F091923290E2E5
:10F0E000968381FF06C0E0919332F091943290E2D2
:10F0F000968380FF06C0E0919532F091963280E2CF
:10F10000868308958091863C811107C084E00E9427
:10F11000407881E08093863C089584E00E94617885
:10F120001092863C0895CF92DF92EF92FF920F9358
:10F130001F93CF93DF93C12C26E0D22EC0927F3253
:10F14000D092803230EAE32E36E0F32EE092813224
:10F15000F092823200E816E00093833210938432FA
:10F16000C0E6D6E0C0938532D0938632C092873213
:10F17000D0928832C0938932D0938A3200938B32F6
:10F1800010938C32E0928D32F0928E322DEC3CEC6A
:10F190004CED50E40E94BFD6C0928F32D092903294
:10F1A000E0929132F092923218164CF4C09393325E
:10F1B000D0939432009395321093963208C0009306
:10F1C000933210939432C0939532D0939632DF915C
:10F1D000CF911F910F91FF90EF90DF90CF90089506
:10F1E0000E9466D260E070E080E091E40E94937833
:10F1F0000C9485D281E080938F3C089520E093E0C9
:10F2000088ED08B618BE84BF9093800020918200DC
:10F2100021FDFCCF08BEFFCF80918F3C81110E9461
:10F22000FE7883E008958091903C882341F0F89423
:10F2300061E089E790E00E9468D282E0089583E06F
:10F240000895CF93DF93CDB7DEB7AD97CDBFDEBFC7
:10F2500021E2EDEEF1E2DE01119601900D922A9588
:10F26000E1F722E02093CA01DE019296E8E0F0E0A7
:10F2700024912D933196EE30F105D1F72DE228A798
:10F28000E0E1F0E0E491EF7121E030E02C0F3D1F70
:10F290002E0F311DF901208129A7E2E1F0E0E49170
:10F2A000EF719E012E0F311DF90121812AA7E4E1A2
:10F2B000F0E0E491EF719E012E0F311DF9012181E3
:10F2C0002BA71CA61092CA0125E0FC012783BE01D2
:10F2D0006E5D7F4F0E9461628093B63FAD96CDBF59
:10F2E000DEBFDF91CF91089581E08093903C80E074
:10F2F0000895CF93DF93EC0120E030E040E051E44B
:10F3000069857A858B859C850E94BFD618166CF01E
:10F31000CE010E943C5F69857A858B859C850E9421
:10F3200093780E9406BD80E001C08DE6DF91CF9109
:10F33000089561E27CE30C94FAC063E07CE30C94F2
:10F34000FAC066EE7BE30C94FAC068EC7BE30C94A5
:10F35000FAC064EB7BE30C94FAC0CF93DF9387E6AB
:10F3600097E49F938F93CEE6DCE589818F93888124
:10F370008F930E94D2E181E395E49F938F938981DB
:10F380008F9388818F930E94D2E189EA94E49F93BE
:10F390008F9389818F9388818F930E94D2E18FED23
:10F3A00093E49F938F9389818F9388818F930E9499
:10F3B000D2E10E94D9A88DB79EB740968DBF9EBF5F
:10F3C00080E0DF91CF910895CF93DF938AEB93E4B0
:10F3D0009F938F93CEE6DCE589818F9388818F930D
:10F3E0000E94D2E18CE492E49F938F9389818F9362
:10F3F00088818F930E94D2E181EC90E49F938F9358
:10F4000089818F9388818F930E94D2E189EA94E465
:10F410009F938F9389818F9388818F930E94D2E1EC
:10F420008FED93E49F938F9389818F9388818F933E
:10F430000E94D2E18DB79EB744968DBF9EBF80E0FB
:10F44000DF91CF910895CF93DF9380EA90E49F936B
:10F450008F93CEE6DCE589818F9388818F930E941C
:10F46000D2E182E29DE39F938F9389818F9388817C
:10F470008F930E94D2E18FED93E49F938F938981C4
:10F480008F9388818F930E94D2E18DB79EB70C969F
:10F490008DBF9EBF80E0DF91CF910895CF93DF9322
:10F4A0008AEF9CE39F938F93CEE6DCE589818F936F
:10F4B00088818F930E94D2E189E89CE39F938F9388
:10F4C00089818F9388818F930E94D2E18FED93E49D
:10F4D0009F938F9389818F9388818F930E94D2E12C
:10F4E0008DB79EB70C968DBF9EBF80E0DF91CF9108
:10F4F0000895CF93DF9386E69CE39F938F93CEE6A8
:10F50000DCE589818F9388818F930E94D2E18DE31E
:10F510009CE39F938F9389818F9388818F930E941F
:10F52000D2E18FED93E49F938F9389818F938881AC
:10F530008F930E94D2E18DB79EB70C968DBF9EBF70
:10F5400080E0DF91CF9108952F923F924F926F927A
:10F550007F928F929F92AF92BF92CF92DF92EF9263
:10F56000FF920F931F93CF93DF93CDB7DEB76D97C5
:10F57000CDBFDEBF3C016F8B788F1B861C861D863E
:10F580001E8680915F3F8F5F80935F3F833008F0DE
:10F5900099C2FB0101900020E9F73197E61BF70BB8
:10F5A000E130F24008F090C2DB018C91882379F1C0
:10F5B0007B01BFEFEB1AFB0A8B0191E020E02111E8
:10F5C00018C021E0883209F020E0992321F081322F
:10F5D000C0F08F37B1F06801EFEFCE1ADE0A90E08D
:10F5E0002D8F0E94C7E0D8018C93860190E02D8D6D
:10F5F00008C021E0893209F420E0F80180830F5F20
:10F600001F4FD7018D917D018111D9CF02C00F8984
:10F61000188DF80110821092B63F22E2222E2AE3C2
:10F62000322E412C3CE2832E3DE7932EA12CEF8815
:10F63000F88C82E29CE2ABE7B0E08F839887A987E1
:10F64000BA872A8A3B8A4C8A8F86988AA98A86E05A
:10F65000EEE0F2E2DE01119601900D928A95E1F75B
:10F66000D7016C91662309F473C170E0CE0107964F
:10F670000E9424E1892B09F46BC1C3010E946560DB
:10F680008701075F1F4F6F8A788E37016301BFEFD5
:10F690006B1A7B0AF601608170E0CE0107960E942A
:10F6A00024E1892B61F4860163016F88788C7601EF
:10F6B00098012E5D3F4F0F8B188F890109C0D7012C
:10F6C0008C91882309F444C160167106F9F600C2D2
:10F6D0006701BFEFEB1AFB0AF601608170E0CE0113
:10F6E00042960E9424E1892B01F10F89188DD601E1
:10F6F0001C9293012F5E3F4F2F8B388F46E050E0D6
:10F70000B801C9010E944FE16F89788D87E493E2C7
:10F710000E94BE5F898F9A8FD30114968D939C931C
:10F720001597019631F484E6D8C1E016F10681F60A
:10F73000FACF86010F5F1F4F7601EAE0EE0EF11C53
:10F740006B8E7C8E3801D801BD908D01CB2CD12CD5
:10F75000C6010E94ABE0892B59F4B601CE01019697
:10F760000E9424E1892B21F40E151F0559F7DBCFE8
:10F7700073016B8C7C8CBEE6BB1649F0E2E2BE12D4
:10F7800009C0D70111968C91823209F04AC0F30169
:10F790001782C0C0C601C0970A9718F0FDE2BF12D9
:10F7A00035C0E98DFA8DEE0FFF1F298D3A8DE20FDE
:10F7B000F31FEE0FFF1FEE0FFF1FEE0FFF1FE355AE
:10F7C000FA4EE491E4FF17C0BE016B5E7F4FC701A4
:10F7D0000E9427DDD30119966D937D938D939C93A1
:10F7E0001C978D899E898E159F0509F473C184E04D
:10F7F00017968C938FC0C7010E94ACDFF30161871D
:10F8000072878387948782E0878384C0FBE7BF1277
:10F8100054C087E0D30117968C93BFEFEB1AFB0A15
:10F8200099C0B7016F5F7F4F85E0F3018783C70100
:10F830008F579F4FFB01DB0120812C3531F4318143
:10F840003232A1F43C93319612C0223279F41C92E8
:10F850007F012FEFE21AF20AD7010D900020E9F79D
:10F860001197AE19BF09139740F41FC02C9331961E
:10F870001196A817B90701F72FC181818033A9F428
:10F880008281883791F440E050E060E070E0C70189
:10F890000E9498DED30119966D937D938D939C936E
:10F8A0001C9783E017968C9335C0C3010E94616258
:10F8B0008093B63F882371F146C0B4E7BB120CC0F9
:10F8C00081E0F301878381E090E0A0E0B0E08187F0
:10F8D0009287A387B4871EC0F6E6BF120AC081E0F4
:10F8E000D30117968C93F301118612861386148622
:10F8F00011C0FBE5BF12ECC086E0D30117968C93D4
:10F90000B701C3010E9461628093B63F81111BC0A1
:10F9100087E6E3C0BE01615F7F4FC7010E9469E1D6
:10F920007C01009709F4D4C0FC0180818D3729F453
:10F93000818197012F5F3F4F79018C3259F03FEF62
:10F94000E31AF30A07C0843008F0C7C0833011F40B
:10F9500080E0C3C08B85882349F043E050E0BE01BE
:10F96000655F7F4FC3010D960E944FE1D30114964E
:10F970008D919C9115970E94F364882371F08F8973
:10F98000988D0E949C5F882341F043E050E06F898E
:10F99000788DCE010B960E944FE1F3018481958111
:10F9A00020910237309103378217930711F42EEF1D
:10F9B00027830E94B35F882309F456C0D30157966A
:10F9C0000D911C915897F80160816B3729F4B801AB
:10F9D000C3010E94A47A48C070E088E791E20E94C7
:10F9E00024E1892B61F180915D3F811103C0AEE874
:10F9F000B7E402C0A0E8B7E4BF93AF930E9433E23C
:10FA00000F900F9082E08093843CC8010E9409BE51
:10FA100011E01093843CAEE7B7E4BF93AF930E942C
:10FA200033E280E090E00E945E611093603FD3017A
:10FA300012968D919C9113970F900F903FC087E67F
:10FA400093E6A0E0EF89F88D80839183A283C801BB
:10FA50000E9485706AEA7EE30E9471BFD30112960C
:10FA60008D919C9113972AC0F30187818F3F19F4E0
:10FA70008281938123C0811105C0C3010E94335C40
:10FA8000F30112C08091BD34823069F0C3010E943D
:10FA9000095CC3010E94865CF30106C027812F3FE9
:10FAA00061F0FC0101C0F301828193810097B1F7FD
:10FAB00082B193B1612C712C01C03F01892B09F0F7
:10FAC000B8CD46CF82E709C08BE68093B63F05C02C
:10FAD0008FE603C086E601C081E76D96CDBFDEBF2D
:10FAE000DF91CF911F910F91FF90EF90DF90CF901A
:10FAF000BF90AF909F908F907F906F904F903F906E
:10FB00002F900895CF93DF93EC011092603F1092F5
:10FB10005F3F8AE091E20E945E61BE010E94A47A8A
:10FB200042E060E00E94086381E0DF91CF910C9495
:10FB300029AB2F923F924F925F926F927F928F925A
:10FB40009F92AF92BF92CF92DF92EF92FF920F936C
:10FB50001F93CF93DF935C011B018A01060F171FD0
:10FB6000DC0116969C908091603FEB0121968823E2
:10FB700021F08CE2FB01808303C08BE7DB018C93D7
:10FB800090E0412C4BE7642E55E0752E68E1C62EBF
:10FB900062E2D62E74E1E72E72E2F72EECE28E2EB0
:10FBA000FDE75F2EF50187818E5F823008F4E5C0A6
:10FBB000992311F08882219680915D3F811113C0B5
:10FBC000C50141969F938F93FF92EF92DF93CF935E
:10FBD0000E9484E2C80FD91F0F900F900F900F90D2
:10FBE0000F900F9012C0C50141969F938F93DF92A3
:10FBF000CF92DF93CF930E9484E2C80FD91F0F905A
:10FC00000F900F900F900F900F90D50117968C9139
:10FC1000811103C0EEE1F2E2A0C0823019F5D501F6
:10FC20001C968C911C978F931B968C911B978F938E
:10FC30001A968C911A978F9319968C918F93A3E2B1
:10FC4000B2E2BF93AF93DF93CF930E9484E2C80FD9
:10FC5000D91FD50117968C91EDB7FEB73896EDBF39
:10FC6000FEBF84C0833019F5D5011C968C911C977A
:10FC70008F931B968C911B978F931A968C911A9742
:10FC80008F9319968C918F93A7E2B2E2BF93AF93B3
:10FC9000DF93CF930E9484E2C80FD91FD501179636
:10FCA0008C91EDB7FEB73896EDBFFEBF5FC08530D3
:10FCB00059F4D50158968C9158978F9357968C91FB
:10FCC0008F93AFE2B2E209C08630C9F4F501808DAE
:10FCD0008F9387898F93A4E3B2E2BF93AF93DF93AF
:10FCE000CF930E9484E2C80FD91FD50117968C913B
:10FCF0000F900F900F900F900F900F9037C084309F
:10FD000091F4C5010E940365F50141855285638523
:10FD100074852085CE010E942BC3C80FD11DD5014B
:10FD200017968C9123C0813009F5F5018185928564
:10FD3000A385B485892B8A2B8B2B69F4E9E3F2E246
:10FD4000DE0186E001900D928A95E1F72596D501B6
:10FD500017968C910BC0EFE3F2E2DE01872D019044
:10FD60000D928A95E1F72496F5018781873021F479
:10FD70006882219690E001C091E0C017D10718F089
:10FD80008FEF9FEF48C0D5011296AD90BC901397AE
:10FD9000A114B10441F0F50186812FEF240D8415E3
:10FDA0002CF0482EFFCE9414A4F01EC0FE01D50105
:10FDB000CF010196EC01508216964C9016973FEFBA
:10FDC000320F42161CF4232FFC01F2CF5D0191E0AB
:10FDD000E9CEFE012DE7CF010196EC0120834A9484
:10FDE000941414F4FC01F7CF8091603F882329F02C
:10FDF0001092603F8DE7888321968DE79AE0A0E01E
:10FE000088839983AA8322960C171D0708F4B8CF1C
:10FE1000CE0182199309DF91CF911F910F91FF902D
:10FE2000EF90DF90CF90BF90AF909F908F907F909A
:10FE30006F905F904F903F902F90089540E052E078
:10FE40006AEA7CE30E94997D8AEA9CE39F938F9300
:10FE50000E9421E20F900F900895BF92CF92DF92FF
:10FE6000EF92FF920F931F93CF93DF93CDB7DEB73F
:10FE70006297CDBFDEBFB82E80915C3F882309F426
:10FE8000FFC08FE6B81214C08AE091E20E945E6162
:10FE90006AEA7EE38091A63C9091A73C0E940BC346
:10FEA000BC018CE091E20E94BF620DE117E332C019
:10FEB0008091BD340DE117E3882361F1FF24FA94AA
:10FEC000C8010E942560882329F1823029F480919D
:10FED000653F811119C016C0843029F48091623FBA
:10FEE000811112C00FC0853079F48091643F88235E
:10FEF00049F0F8014185528563857485452B462B71
:10FF0000472B11F0F801F782F801028113810115E6
:10FF10001105B1F6C090A23CD090A33CE090A43C67
:10FF2000F090A53CC701B6010E945CD52CEA35ECE7
:10FF300047E257E30E94BFD6181654F14EC0F801AD
:10FF4000028113810115110519F581E70E945FA84F
:10FF50008091A23C9091A33CA091A43CB091A53C7F
:10FF600089B99AB9ABB9BCB984E799E6A4E6B0E01F
:10FF700081BB92BBA3BBB4BB82E087B916B840E09B
:10FF800052E06AEA7CE384E097E30E94997D78C0BE
:10FF9000F80187818F3F99F6C186D286E386F48681
:10FFA00084E799E6A4E6B0E0818B928BA38BB48BB7
:10FFB00082E087831682028113810FC0F8010281DB
:10FFC00013810115110549F440E052E06AEA7CE32F
:10FFD00084E097E30E94997D53C0F80187818F3FA9
:10FFE00069F78091773281111AC08091A93C8F9373
:10FFF0008091A83C8F931F92BF9284E492E29F93DA
:020000021000EC
:100000008F93CE0101967C01FF928F930E9484E230
:100010001092A83C1092A93CCDBFDEBF13C00E9435
:1000200060C81F928F931F92BF928CE492E29F93BD
:100030008F93CE0101967C01FF928F930E9484E200
:10004000CDBFDEBFB701C8010E946162F801168210
:1000500086E0878386E690E0818B928B1282138202
:1000600040E052E06AEA7CE384E097E30E94997DF5
:100070008AEA9CE39F938F930E9421E20F900F9056
:100080006296CDBFDEBFDF91CF911F910F91FF90A0
:10009000EF90DF90CF90BF900895613019F06230FB
:1000A00029F0089584E097E30C941E7F0C942D7F33
:1000B000FC0181859285A385B48586309105A105D3
:1000C000B10580F580935C3F1092613F1092623FD2
:1000D0001092633F1092643F1092653F0097A10514
:1000E000B10511F121E02093613F81309105A10517
:1000F000B105D1F02093623F82309105A105B10591
:1001000099F02093633F83309105A105B10561F01B
:100110002093643F0597A105B10531F42093653F15
:1001200080E008958EE6089580E0089563E278E423
:100130000C94FAC06CEC77E40C94FAC068E977E4AC
:100140000C94FAC0BF92CF92DF92EF92FF920F937E
:100150001F93CF93DF93CDB7DEB76897CDBFDEBFD8
:100160006B0128E1FC01DE01119601900D922A95A8
:10017000E1F78EE7E82E83E3F82E8E010F5F1F4F25
:10018000B12CF7018081823029F4F80110821182AC
:10019000128213828091F05A8B1114C02091035B5C
:1001A0003091045B4091055B5091065BF8016081E2
:1001B0007181828193810E9461D7F601608371838E
:1001C0008283938380910F5B8B1114C02091225BFB
:1001D0003091235B4091245B5091255BF801608155
:1001E0007181828193810E9461D7F6016483758356
:1001F0008683978380912E5B8B1114C02091415B85
:100200003091425B4091435B5091445BF8016081C7
:100210007181828193810E9461D7F6016087718725
:100220008287938780914D5B8B1114C02091605B16
:100230003091615B4091625B5091635BF80160813A
:100240007181828193810E9461D7F60164877587ED
:1002500086879787B394F5E3EF0EF11C0C5F1F4F71
:1002600086E0B8128ECF6896CDBFDEBFDF91CF910A
:100270001F910F91FF90EF90DF90CF90BF90089566
:10028000F8940E94F0780E9497810E9485D20E9483
:100290001EC50E94A3B30E9440700E9406BD0E942A
:1002A00040A640E060E080E00E9403660E94A661F4
:1002B0000E9485810E944A830E9402500E947DD242
:1002C0008091A20084608093A2008091A20082604D
:1002D0008093A2008091A20081608093A200789414
:1002E0000E94D9A80E9408BE0E945566FDCFE82F43
:1002F000F0E0EE0FFF1FE15BF74B659174914FE467
:1003000050E086E69FE30C94F6E08091833C8230D7
:1003100041F440E060E081E00E94036680E00E94DA
:100320007D670C9459C9682F81E00C94FBC510922D
:10033000B73F1092B83F1092B93F1092BA3F08955C
:10034000CF93DF93EC018C819D81880F991F880FDB
:10035000991F2091B93F3091BA3F820F931F80932C
:10036000BB3F9093BC3F44E050E061EC7FE30E94D0
:100370007DD14091C13F5091C23F6091C33F709188
:10038000C43F49875A876B877C8780E0DF91CF9194
:1003900008950F931F93CF93DF93EC018091BE34A8
:1003A000882339F089E0DF91CF911F910F910C9450
:1003B0005FA849855A856B857C854093BD3F5093E6
:1003C000BE3F6093BF3F7093C03FCE010E94A081AB
:1003D0008093B63F811141C00091BD3F1091BE3F57
:1003E0002091BF3F3091C03F49855A856B857C8500
:1003F000401751076207730739F10093C13F10930B
:10040000C23F2093C33F3093C43F8C819D81880FAE
:10041000991F880F991F2091B93F3091BA3F820FE1
:10042000931F8093BB3F9093BC3F44E050E061EC4E
:100430007FE30E940ED23091BD3F2091BE3F90914C
:10044000BF3F8091C03F04C0342F252F962F872FA8
:1004500039872A879B878C8780E0DF91CF911F9116
:100460000F9108950E941EB980E008958091C53FC4
:100470009091C63F8F3E924111F08EE50895809194
:10048000EB3F9091EC3F8F3E9241B9F78091ED3F69
:100490009091EE3F8F3E924181F7809176579091F7
:1004A00077578F3E924149F78091785790917957CD
:1004B0008F3E924111F780910B5990910C598F3ECC
:1004C0009241D9F680E0089594E0899FF0011124CB
:1004D000EB53F04C4283538364837583089594E017
:1004E000899FF0011124E858F84A45AB56AB67AB39
:1004F00070AF08955F926F927F928F929F92AF92AA
:10050000BF92CF92DF92EF92FF920F931F93CF9300
:10051000DF93CDB7DEB76097CDBFDEBFBE016F5FA3
:100520007F4F8DEA97E50E94A280CE0101964C0193
:1005300085E2A82E88E5B82E95E3C92E98E5D92E38
:1005400025E4E22E28E5F22E05E618E537E8632ECD
:100550003BE5732E512CF4014191519161917191C0
:100560004F01F50141935193619371935F01F6013E
:1005700041935193619371936F01F70141935193AB
:10058000619371937F01852D0E946270F801119231
:100590001192119211928F01F30110821182128235
:1005A00013825394F8E16F0E711C84E05812D3CF7C
:1005B0006096CDBFDEBFDF91CF911F910F91FF906D
:1005C000EF90DF90CF90BF90AF909F908F907F90F3
:1005D0006F905F9008958091EF3F08951F93CF93A0
:1005E000DF938BE897E1EDEEFFE3DF019C011D92C5
:1005F00021503040E1F78FEE92E18093ED3F9093F0
:10060000EE3F8093765790937757C6EFDFE3C09322
:10061000F03FD093F13FC093F23FD093F33FC093AC
:10062000F43FD093F53F81E090E06AEB76E520E07F
:1006300030E01CEB129FA001139F500D1124FA0112
:10064000E351F04CD90111961A9F90011B9F300D78
:1006500011242A50304C2387348761877287BA016E
:100660006A50704C9C0101968032910519F78CEB11
:10067000829FF001839FF00D1124E351F04CC3875A
:10068000D4876187728780E28093EF3FDF91CF91BB
:100690001F910895CF93DF93E8E7F7E585E991E0AF
:1006A000DF01EC011D922197E9F7A5ECBFE388E299
:1006B000ED0119928A95E9F78FEE92E18D939C9363
:1006C0008093EB3F9093EC3F8083918380930B5911
:1006D00090930C59DF91CF910C94EE820E94678D1C
:1006E0000E94EE8280E00C94AC4AE091F03FF091E1
:1006F000F13F848581111BC02281338180819181EA
:100700004CEBDF011D924A95E9F722833383808306
:10071000918381E084878091EF3F81508093EF3F08
:10072000828193818093F03F9093F13F05C08CE1EB
:100730000E945FA8E0E0F0E0CF010895A2EFBFE3E0
:10074000ED91FC911197858781E0878782E084870E
:10075000828193818D939C9381E00E9460AC0C9484
:1007600064B6EF92FF920F931F93CF93DF9300D065
:100770001F92CDB7DEB78C014B835C8369837A838C
:100780000E947583FC014B815C8169817A810097AD
:1007900061F48EE02496CDBFDEBFDF91CF911F9133
:1007A0000F91FF90EF900C94EB4E83E0858782E3EE
:1007B00092E884839583068317838B017A0126E070
:1007C000D8014D915D916D917D918D01CF0185593C
:1007D0009F4FDC014D935D936D937C931397D701ED
:1007E0004D915D916D917D917D01418B528B638B1C
:1007F000748B215034962111E3CF83E02496CDBF32
:10080000DEBFDF91CF911F910F91FF90EF900C947D
:100810009E83CF92DF92EF92FF926B017C010E9448
:100820007583009739F48EE0FF90EF90DF90CF90C2
:100830000C94EB4E2CE834E8FC0124833583E55618
:10084000FF4FC082D182E282F38221E0FC01278740
:1008500082E00E949E8380E0FF90EF90DF90CF9037
:1008600008958091F43F9091F53FFC0124853EEF7F
:10087000320F323018F424E024870895243011F028
:1008800080E090E00895E091F43FF091F53F2281FF
:100890003381808191814CEBDF011D924A95E9F70C
:1008A0002283338380839183E091F43FF091F53F7D
:1008B0000280F381E02DE093F43FF093F53F8485CF
:1008C000823011F483E084878091EF3F8F5F8093C3
:1008D000EF3F8FEF0E9460AC81E04091F03F50917C
:1008E000F13F2091F43F3091F53F4217530709F053
:1008F00080E00895BC016F5E7F4FDC011696ED919C
:10090000FC91179785599F4F19950E944384811137
:100910000E946E5680E0089585569F4F20E034E295
:1009200044E759E4FC0160817181828193810E94D6
:1009300061D70E9430D50E945CD50E9428B90E94E0
:10094000438481110E946E5680E008958091F43FA7
:100950009091F53FFC0124853EEF320F323018F4C0
:1009600024E024870895243011F080E090E0089579
:10097000CF93DF93C091F43FD091F53F8C859EEFEC
:10098000980F923018F484E08C8705C0843019F0F9
:1009900080E090E010C02097D9F3DE011296ED912F
:1009A000FC9113978785882329F0EC17FD0711F038
:1009B000DF01F4CFCD01DF91CF910895CF93DF9385
:1009C000EC012A813B81888199814CEBFB01DE019E
:1009D00001900D924A95E1F72A833B83888399839E
:1009E000DF91CF9108958FEE92E180930D5990930E
:1009F0000E598093CA599093CB5908952F923F92E4
:100A00004F925F926F927F928F929F92AF92BF921E
:100A1000CF92DF92EF92FF920F931F93CF93DF93CA
:100A2000CDB7DEB76A97CDBFDEBF4C011B012901F0
:100A30003A01E986FA860B871C871A2D0B2DE8A848
:100A4000B9A8AAA82BA9298380913635882399F0C3
:100A500080912A3590912B35A0912C35B0912D3570
:100A6000BC01CD019F772CEA35EC47E257E30E94A9
:100A7000BCD487FD11C78091613690916236A091F8
:100A80006336B0916436BC01CD019F7731E03D8380
:100A90002CEA35EC47E257E30E94BFD6181614F053
:100AA0001D8210C02DEC3CEC4CEC5DE360910636F1
:100AB0007091073680910836909109360E94BCD417
:100AC00087FDECC6F10180819181A281B381BC01D7
:100AD000CD019F77F1E0FD872CEA35EC47E257E343
:100AE0000E94BFD618160CF01D86F10184819581F5
:100AF000A681B781BC01CD019F77F1E0F98B2CEA8B
:100B000035EC47E257E30E94BFD618160CF0198A5D
:100B1000F10180859185A285B3852091653630915C
:100B2000663640916736509168362E8B3F8B488FE2
:100B3000598F2091693630916A3640916B365091C9
:100B40006C362A8B3B8B4C8B5D8B40916D36509174
:100B50006E3660916F3670917036F0903735F110C7
:100B600021C01092555981E08093565982E08093BC
:100B700057593D81332341F04D85411195C659891F
:100B8000511192C68CE9C1C6CB01BA019F772CEAFC
:100B900035EC47E257E30E94BFD618160CF089C621
:100BA0008BE9B3C6BC01CD019F77A1E0AA8F2CEAE7
:100BB00035EC47E257E30E94BFD618160CF01A8EA8
:100BC000B1E0FB1216C01092555982E0809356593D
:100BD000F0925759ED81EE2339F0FD85F11164C68D
:100BE0002A8D222379F260C66A897B898C899D8946
:100BF000CDCF32E0F31217C081E080935559F092C7
:100C00005659109257594D81442341F05989511139
:100C10004BC68A8D882309F4B5CF46C66E897F8975
:100C2000888D998DB3CFB101C4010E94FB4C9D8189
:100C3000992309F451C02091F2343091F33440915A
:100C4000F4345091F5346091473570914835809176
:100C5000493590914A350E9413D39F772CEA35ECA1
:100C600047E257E30E94BCD487FF36C02091F63498
:100C70003091F7344091F8345091F93460914B350C
:100C800070914C3580914D3590914E350E9413D323
:100C90009F772CEA35EC47E257E30E94BCD487FFEC
:100CA0001BC02091FA343091FB344091FC345091B8
:100CB000FD3460914F357091503580915135909150
:100CC00052350E9413D39F772CEA35EC47E257E365
:100CD0000E94BCD487FDE4C58CA98093F1348DEECD
:100CE00094E30E94034B86E5EDEEF4E3A4E7B9E557
:100CF00001900D928A95E1F788E1E7E4F5E3A0E140
:100D0000B9E501900D928A95E1F78091383581110E
:100D1000D5C523E333E34BEC51E46E2D7B2D8A2DB7
:100D200099810E9461D74B015C0160934059709397
:100D30004159809342599093435923E333E34BEC59
:100D400051E4C301B2010E9461D7609328597093A6
:100D5000295980932A5990932B5923E333E34BEC81
:100D600051E469857A858B859C850E9461D7609363
:100D70002C5970932D5980932E5990932F5923E31A
:100D800033E34BEC51E4612F702FC6010E9461D711
:100D9000162F072F412F502FBC01409330595093ED
:100DA0003159609332597093335980910236909142
:100DB0000336A0910436B0910536BC01CD019F7772
:100DC0000E9499D50E9430D5609351597093525921
:100DD0008093535990935459A0915559A98BB09130
:100DE0005659BA8BEB2FF0E0ED83FE837F01EE0CBA
:100DF000FF1CEE0CFF1CF101EE0DFF1D80819181A7
:100E0000A281B381BC01CD019F772CEA35EC47E28A
:100E100057E30E94BCD4D82EDD1CDD24DD1C3989AB
:100E2000232F30E029833A838901000F111F000F1F
:100E3000111FF101E00FF11F80819181A281B38127
:100E4000BC01CD019F772CEA35EC47E257E30E94C5
:100E5000BCD4881F8827881F8D21809350592CEA85
:100E600035EC47E257E3C501B4019F770E94BFD636
:100E700018160CF0F9C0F801EE50FB4CD801A95B34
:100E8000BA4C2D913D914D915C916081718182812F
:100E900093810E9413D36B017C01ED81FE81EE0FE3
:100EA000FF1FEE0FFF1FEE50FB4CAD81BE81AA0F5E
:100EB000BB1FAA0FBB1FA95BBA4C2D913D914D9151
:100EC0005C9160817181828193810E9413D36987D3
:100ED0007A878B879C87A5019401C501B4010E9484
:100EE00061D720E030E040E850E40E9461D76D8790
:100EF0007E878F87988BA7019601C701B6010E9454
:100F000061D72B013C0129853A854B855C85CA0157
:100F1000B9010E9461D79B01AC01C301B2010E94DB
:100F200014D39B01AC016D857E858F8598890E94C5
:100F300013D32B013C0120E030E0A9010E94BFD671
:100F40001816C4F4C301B2010E943AD82B013C0127
:100F500029853A854B855C85C701B6010E94CCD6B0
:100F60009B01AC01C301B20190580E94C3D42B0174
:100F70003C0103C0412C512C32018091F13483306B
:100F800021F477FA709477F8709420E030E0A901AA
:100F9000C501B4010E94BCD487FF04C077FA7094E5
:100FA00077F8709409811A81000F111F000F111F2B
:100FB000A801435F564A5A01A301920169857A85C7
:100FC0008B859C850E9461D79B01AC01C701B6014E
:100FD0000E9413D320E030E040E05FE30E9461D73D
:100FE000D5015B966D937D938D939C935E97AD80B9
:100FF000BE80AA0CBB1CAA0CBB1CF501E35FF64A21
:101000004F01A3019201C701B6010E9461D79B0164
:10101000AC0169857A858B859C850E9414D320E07C
:1010200030E040E05FE30E9461D7D4015B966D93AE
:101030007D938D939C935E97E0915759F0E0EE0F6E
:10104000FF1FEE0FFF1FE35FF64A138E148E158EFF
:10105000168EB0914059B987E0914159ED872090A3
:1010600042593090435925C05701F701E35FF64AD2
:10107000838D948DA58DB68D9C01AD015058F801DE
:10108000E35FF64A838D948DA58DB68DBC01CD01AD
:1010900090580E94CCD69B01AB01BC0140934059B3
:1010A00050934159609342597093435929873D8722
:1010B0001C01D801A35FB64A5B96CD90DD90ED9000
:1010C000FC905E97E981FA81EE0FFF1FEE0FFF1F84
:1010D000E758F64A13962D913D914D915C911697E4
:1010E00060817181828193810E9413D3A70196014F
:1010F0000E9413D369837A838B839C83D501A35F7A
:10110000B64A5B964D905D906D907C905E97ED81B8
:10111000FE81EE0FFF1FEE0FFF1FE758F64A1396F2
:101120002D913D914D915C911697608171818281E5
:1011300093810E9413D3A30192010E9413D36D8364
:101140007E838F8398879B01AC0169817A818B8133
:101150009C810E94CCD629853D85A1010E9413D394
:101160004B015C01E894B7F820E030E040E85FE331
:10117000C501B4010E94BFD618160CF4C3C32AE0FF
:1011800037ED43EA5BE3C501B4010E94BFD61816F0
:1011900094F42AE037ED43E25CE369857D85C10183
:1011A0000E9461D79B01AC01C501B4010E94BFD66A
:1011B00018160CF4A7C3A30192015058C701B60139
:1011C00090580E9487D34B015C016093385970930B
:1011D000395980933A5990933B59809137358130F2
:1011E00039F4412C512C30E8632E3FEB732E06C0AE
:1011F000412C512C20E8622E2FE3722E8091505901
:101200008823D1F16091515970915259809153596D
:10121000909154590E945CD56B017C012CEA35EC0D
:1012200047E257E30E94BCD487FD10C01091F1340F
:101230002BED3FE049EC50E4C701B6010E9461D7B5
:101240009B01AC01C12CD12C7601B9C081E090E0AA
:10125000A0E0B0E08093515990935259A093535914
:10126000B09354591091F1342BED3FE049EC50E428
:10127000C12CD12C7601A3C02D813E814F81588590
:1012800069817A818B819C810E9487D369837A836B
:101290008B839C8360933C5970933D5980933E5956
:1012A00090933F59A50194010E9413D36B017C01D7
:1012B0009F772CEA35EC47E257E30E94BCD487FFC6
:1012C00018C01091F1346091515970915259809128
:1012D0005359909154590E945CD52BED3FE049EC55
:1012E00050E40E9461D79B01AC01C12CD12C760146
:1012F00066C029813A814B815C81C501B4010E949D
:10130000BFD61816F4F42BED3FE049EC50E4C301CE
:10131000B2010E9461D79B01AC0169817A818B8106
:101320009C810E9414D360933C5970933D598093E3
:101330003E5990933F59A50194010E9413D36B012C
:101340007C011091F134133099F0609151597091F2
:10135000525980915359909154590E945CD52BED6C
:101360003FE049EC50E40E9461D79B01AC0127C0EB
:101370002BED3FE049EC50E4C301B2010E9461D77C
:101380009B01AC01C701B6010E9413D37B018C0104
:10139000609151597091525980915359909154597B
:1013A0000E945CD52BED3FE049EC50E40E9461D7F0
:1013B0009B01AC01C701D8016C017D010BC012304B
:1013C00049F4C301B2010E9461D7A70196010E94AE
:1013D00014D30AC0C301B2010E9461D79B01AC01C2
:1013E000C701B6010E9413D37B01AB01BC0140933E
:1013F00044595093455960934659709347598C010D
:1014000050905759A52DB0E0FD01EE0FFF1FEE0FD4
:10141000FF1FE758F64AAA0FBB1FAA0FBB1FA35F07
:10142000B64A13962D913D914D915C91169760812E
:101430007181828193810E9413D34B015C0160937F
:1014400048597093495980934A5990934B59970141
:10145000A80169857D85C1010E9461D76B017C016E
:1014600060934C5970934D5980934E5990934F59B6
:10147000A50194010E94CCD669837A838B839C83D7
:1014800060933459709335598093365990933759F6
:1014900080913635811117C0F0912A35FD83409037
:1014A0002B3520912C352E8B30912D353A8F109283
:1014B0002A3510922B3510922C3510922D3581E063
:1014C0008093363512C020912A3530912B354091CA
:1014D0002C3550912D3569817A818B819C810E94B8
:1014E000C3D46D83472E8E8B9A8F598945E3549FC1
:1014F000F0011124E158FC4C20813181428153815B
:10150000C701B6010E94C3D4662E072F182F792E6B
:101510002D81342D4E895A8D0E94BCD487FF04C082
:101520006D80042D1E897A8C9A8985E3989FF0013D
:101530001124E158FC4C2081318142815381C70143
:10154000B6010E94C3D46B017C019B01AC01662DE6
:10155000702F812F972D0E94BFD6181624F06C2C67
:101560000D2D1E2D7F2C862D902FA12FB72D809312
:10157000585990935959A0935A59B0935B5920E008
:1015800030E0A901C501B4019F770E94BFD61816AB
:1015900084F5A5E35A9EF0011124E158FC4C20810A
:1015A000318142815381C501B4010E94C3D44B01F2
:1015B0005C01E894B7F8A5019401662D702F812F86
:1015C000972D0E94BFD6181614F4A72C04C0682CBF
:1015D000092D1A2DAB2C862D902FA12FBA2D80937B
:1015E000585990935959A0935A59B0935B59B62CB6
:1015F00002C0B62CA72CC090C032D090C132E0906F
:10160000C232F090C33220E030E040E850E4C7013D
:10161000B6010E9461D72B013C0129853D85A101BE
:1016200069857D85C1010E9414D3A70196010E949E
:1016300013D39B01AC01C301B2010E9461D70E9488
:101640003AD82B013C0120EC31EE44E65CE46B2DF2
:10165000702F812F9A2D0E9461D720E030E44CE159
:1016600056E40E94C3D46B017C012091C9323091B1
:10167000CA324091CB325091CC3269817A818B81D0
:101680009C810E94C3D44B015C01A301920169813A
:101690007A818B819C810E94C3D487017601A50148
:1016A00094010E9413C20E9499D57B018C0120E015
:1016B00030E040E85FE30E94BFD618163CF4B70163
:1016C000C8010E942BD54B015C0108C0812C912CD4
:1016D00054018394E12CF12C00E81FE3C701D801E9
:1016E00080935C5990935D59A0935E59B0935F5974
:1016F0009701A801609158597091595980915A5990
:1017000090915B590E94C3D46093A9597093AA59D0
:101710008093AB599093AC598092605990926159E3
:10172000A0926259B09263599701A80160914459FF
:101730007091455980914659909147590E94C3D460
:101740006093645970936559809366599093675973
:101750009701A801609148597091495980914A595F
:1017600090914B590E94C3D4609368597093695902
:1017700080936A5990936B59809038599090395959
:10178000A0903A59B0903B59C501B4010E9430D89D
:10179000C0904059D0904159E0904259F09043593F
:1017A0000091555910E0000F111F000F111F035F2A
:1017B000164AA70196010E9461D79B01AC01F8016E
:1017C00063817481858196810E9413D360936C59E3
:1017D00070936D5980936E5990936F59C501B40100
:1017E0000E94C0D49B01AC010091565910E0000F3B
:1017F000111F000F111F035F164AC701B6010E9497
:1018000061D79B01AC01D80113966D917D918D91AB
:101810009C9116970E9413D36093705970937159DD
:101820008093725990937359A0915759B0E0FD017C
:10183000EE0FFF1FEE0FFF1FE758F64AAA0FBB1F60
:10184000AA0FBB1FA35FB64A13968D919D910D9071
:10185000BC91A02D80839183A283B3831092B63F65
:101860008091345990913559A0913659B09137599A
:10187000BC01CD019F772CEA35EC47E257E30E948B
:10188000BCD487FD0FC00E94615682E080930F593F
:101890000E945E4C80E039C08EE837C08EE935C0CA
:1018A0008FE933C089EC31C0B101C4010E94FB4C07
:1018B000C2C9B101C4010E94FB4C0ECA8E2D9B2DE2
:1018C000AA2DB9818093405990934159A0934259D0
:1018D000B0934359409228595092295960922A59FD
:1018E00070922B5929853A854B855C8520932C591C
:1018F00030932D5940932E5950932F594C015D012F
:10190000C60148CA8BE98093B63F6A96CDBFDEBF59
:10191000DF91CF911F910F91FF90EF90DF90CF90CB
:10192000BF90AF909F908F907F906F905F904F90FF
:101930003F902F9008958F929F92AF92BF92CF9237
:10194000DF92EF92FF92CF93DF9380910F5988231C
:1019500009F4B1C00E94EB82843010F482E0ACC084
:101960002091645930916559409166595091675959
:10197000609138597091395980913A5990913B59F9
:101980000E9414D36B017C016093385970933959CC
:1019900080933A5990933B590E9430D88090405997
:1019A00090904159A0904259B0904359C0915559D7
:1019B000D0E0CC0FDD1FCC0FDD1FC758D64AA501E4
:1019C00094010E9461D79B01AC0160916C597091A8
:1019D0006D5980916E5990916F590E9414D368830C
:1019E00079838A839B83C701B6010E94C0D49B017F
:1019F000AC01C0915659D0E0CC0FDD1FCC0FDD1FDC
:101A0000C758D64AC501B4010E9461D79B01AC01F9
:101A10006091705970917159809172599091735978
:101A20000E9414D3688379838A839B83C09157591A
:101A3000D0E0CC0FDD1FCC0FDD1FC758D64A209158
:101A400068593091695940916A5950916B59688130
:101A500079818A819B810E9414D3688379838A83E8
:101A60009B8384E799E50E947D9788E1E9E7F9E5A2
:101A7000A0E1B9E501900D928A95E1F78091605956
:101A800090916159A0916259B09163590197A10950
:101A9000B1098093605990936159A0936259B093B2
:101AA0006359181619061A061B060CF457CF109224
:101AB0000F5980E001C083E0DF91CF91FF90EF905C
:101AC000DF90CF90BF90AF909F908F90089510922D
:101AD0000F5908954F925F926F927F928F929F92CB
:101AE000AF92BF92CF92DF92EF92FF92CF93DF93AC
:101AF000CDB7DEB76497CDBFDEBF69837A838B83B2
:101B00009C8369017A0120E030E040E751E40E94C3
:101B100061D74B015C0120E030E040E751E4C701B0
:101B2000B6010E9461D79B01AC01C501B4010E94BE
:101B300013D36D877E878F87988B20E030E040E25B
:101B400051EC69817A818B819C810E9461D74B0124
:101B50005C0120E030E040E251E4C701B6010E94A0
:101B600061D79B01AC01C501B4010E9414D3698BFC
:101B70007A8B8B8B9C8B20918D5830918E58409115
:101B80008F585091905860E070E080E89FE30E9489
:101B9000C3D44B015C0120E030E040EC50EC6981A3
:101BA0007A818B819C810E9461D72B013C0120E0CE
:101BB00030E040EC50E4C701B6010E9461D79B01C0
:101BC000AC01C301B2010E9414D3A50194010E948B
:101BD00061D7A50194010E9461D7A50194010E94DB
:101BE00061D7A50194010E9461D7A50194010E94CB
:101BF00061D76B017C01A50194016D857E858F8580
:101C000098890E9461D7A50194010E9461D7A5011E
